:020000040000FA
:10000000021F4E022003FFFFFFFFFF02200BFFFF36
:10001000FFFFFF022013FFFFFFFFFF02201BFFFF78
:10002000FFFFFF022023FFFFFFFFFF02202BFFFF48
:10003000FFFFFF022033FFFFFFFFFF02203BFFFF18
:10004000FFFFFF022043FFFFFFFFFF02204BFFFFE8
:10005000FFFFFF022053FFFFFFFFFF02205BFFFFB8
:10006000FFFFFF022063FFFFFFFFFF02206BFFFF88
:10007000FFFFFF022073FFFFFFFFFF02207BFFFF58
:10008000FFFFFF022083FFFFFFFFFF02208BFFFF28
:10009000FFFF70DFFFFF040000000002000000C847
:1000A000030002030369A5020269A532730000017F
:1000B00000000000000400FFFFFFFFFFFFFFFF0440
:1000C00003090424035400650078006100730020D4
:1000D0000049006E0073007400720075006D0065C9
:1000E000006E007400730024035400490020004394
:1000F000004300320035003300310020005500532A
:10010000004200200043004400430000035F005F02
:100110000030005800000000000000000000000057
:1001200000000000000000000000000000000000CF
:100130000000000000303132333435363738394171
:1001400042434445463C1C911C911C911C911C99B6
:100150001C74F8121BD6900391E060159003027492
:10016000FEF0900304744DF0A37405F07A011207B9
:100170000C7F01021D7B74F8121BD674FF121EC582
:100180007E00801F851882851983E064FE700690CA
:1001900003877401F0851882851983E0F890038441
:1001A000E068F07901AA18AB191210DFE9700302B8
:1001B000027E851882851983E064EF70027E07E075
:1001C000C0E0900387E0F8900385E0FAE82AF8E4BD
:1001D000340012075BD0E0F0900387E060A6146063
:1001E0000E14602A14603A14605014606680A69061
:1001F0000384E4F0851882851983E0900386F0C3B8
:1002000094809003874003E4808A74028086851876
:1002100082851983E0900382F090038774030201C2
:1002200094851882851983E0900383F0900386E01B
:1002300060199003877404020194900385E004F030
:10024000F8900386E06860030201959003877405C7
:10025000020194900385E4F0900387F0900384E01A
:10026000F8851882851983E0686003020195900380
:1002700082E0644D60030201951203B68002EEF93C
:100280007401121E4602017174F7121BD674FB1220
:100290001EC5EAFEEBFF7508047509007808121EFA
:1002A000DF7402121F467A907B0079041218F274F0
:1002B00002121E461206FE121F97E0687003A3E0AA
:1002C000697012851882851983E0F47003A3E0F445
:1002D00060030203917404121F3E1207678A088BA1
:1002E00009A808A9097402121F97E8F0A3E9F0749D
:1002F00004121F97E0600879011201510203AA85D8
:100300001882851983E0687003A3E0697076851808
:1003100082851983E0F47003A3E0F470197402126B
:100320001F977410F0A37420F085188285198374C8
:1003300010F0A37420F07508017509007808121EEA
:10034000DF7402121F467A247B0812197774021296
:100350001E467508047808121EDF7402121F467AC2
:10036000907B0079041218F27402121E461206FEE7
:10037000121F97E0687003A3E06970047902800699
:100380007904800279031201518E828F83741E805A
:10039000058E828F83E4F01206FE121F97E06870CC
:1003A00003A3E06970047901800279007405121ECC
:1003B000467F02021D7B74ED121BD674F8121EC517
:1003C000900307E0FA900306E0FB8B08EAF8E4C824
:1003D000F9EB28FEE93408FF751001880C750D064D
:1003E0008F0974027808121F2BC39508F8E4950949
:1003F000F9740228F50E740339F50F8E088F09740D
:10040000097808121F5DE508F511EE2410F508E4DF
:100410003FF509EEF50AEF5401F50B900383E01464
:1004200060541470030204EB147003020566146038
:100430001024FE70030206211470030206D1020686
:10044000E1750D03794E1213B29003071206F4748E
:1004500002F0A374401206F274081206F2F0A3F040
:10046000751012AA10A90C12070CA90D7408121EFF
:10047000467F0C021D7B750D04794E1213B2EE45BA
:100480000B7005A9111219DDC3EE9425EF940850E5
:100490003CC3E5089424E50994084031E50E249610
:1004A000F8E50F3420F988828983E0701BA3AA82C3
:1004B000AB83E070139003887401F08882898374A1
:1004C000A5F08A828B838004900388E4F07508107D
:1004D0007509007808121EDF7C087D03EEFAEFFB39
:1004E0001219777402121E46020463750D05E51198
:1004F000C394794006750C010204637512407513AC
:10050000007812121EDF7C097D037402780A121F24
:100510002BAA0AAB0BA9111218F27402121E4690F4
:100520000307E0A3F0900306E0A3F0751043C3EEC9
:100530009425EF94084003020463C3E5089424E57E
:100540000994085003020463900388E070030204D6
:1005500063E50E2497F8E50F3420F988828983E457
:10056000F0A3F00204637508047509007808121EF0
:10057000DF7402121F467A907B0079041218F2741D
:1005800002121E467402121F97E0F8A3E0F98518C4
:1005900082851983E0687003A3E069851882851954
:1005A00083700BE0F47003A3E0F470578009E0F46B
:1005B0007003A3E0F4700D8518828519837410F020
:1005C000A37420F01206FE121F97E8F0A3E9F0755D
:1005D00008017808121EDF7402121F467A247B0875
:1005E0001219777402121E467508047808121EDF6D
:1005F0007402121F467A907B0079041218F274027A
:10060000121E461206FE121F97E0687003A3E069EF
:100610007006750D01020463750D02750C07020466
:10062000639003D6E0600764026003020463EAFF9C
:100630007A01790012070CE060030206C5800312FC
:10064000117B121162E970F77404121F971206E60B
:100650007404121F977808121F7B85080C85090DFA
:10066000850A0E850B0F9003C2780C121F057404C7
:10067000121F97780C121F6CE5084509450A450BB7
:1006800070CE8EC2E5C554E04FF5C57404121F97B5
:100690001206E67404121F977808121F7B85080C57
:1006A00085090D850A0E850B0F9003C2780C121F69
:1006B000057404121F97780C121F6CE50845094554
:1006C0000A450B70CE7A01790012070C79080204F2
:1006D0006CEB900391F07003020463750D09020442
:1006E00063790602046CE4F0A37426F0A3E4F0A39B
:1006F000F022F0A3E4F0A3F0A3F0A3F0A322851866
:1007000082851983E0F8A3E0F974022274F6121BC3
:10071000D6EAFE900305E0D2E7F0E9A3F0EE9003FD
:1007200003F08E0A74042AFE7A028004E0620A0A48
:10073000EAF83395E012075B8E08C3E89508E99460
:1007400000A2D265D03340E4E50AF0740128F97ABA
:10075000027B0312111D7F03021D7BF9740228F531
:1007600082740339F5832274E9121BD675820075F1
:1007700083FE121E288A168B177514007515008AC1
:10078000828B83E4F09003D6E07006D2AAD2AF80C9
:1007900004640270057900120151750C00750D207A
:1007A000750E00750F009003D6E0600464027015AA
:1007B00012117B120176E9F874096860030208A33C
:1007C0007900120151E064027007A292400302080E
:1007D0007E7508007509027808121EDF7402121F68
:1007E00046850C08850D09AA08E5095407FB850E06
:1007F0000A850F0B740B7808121E96A9081218F2BE
:100800007402121E467E007F009003CAC0828E10C2
:10081000EFF5113395E0F512F513850C08850D09F8
:10082000850E0A850F0B78087910121F189003C6E1
:100830007808121F05758303D0827808121E0950AC
:100840001D851882851983E5822EF582E5833FF5A3
:1008500083E0F9AA14AB151208D28A148B150EEE98
:1008600070010FC3EF940240A09003CE780C121FCA
:10087000059003D2780C121E0940030207A67900E6
:10088000AA14AB151208D279001208D28B15900366
:10089000D6E07004C2AFC2AAEA451570277AA57BDC
:1008A000A58021E870030207C5740668700302077B
:1008B000C574076870030207C5851682851783749F
:1008C00001F080BA758200758302121E287F100223
:1008D0001D7BC008C0097C088A088B09740F780842
:1008E000121F5DEA25E0FAEB33FBE9A2E75004743E
:1008F000014AFAE508A2E0500874216AFA74106B04
:10090000FBE9C333F91CEC70CFD009D0082274F78F
:10091000121BD6120F2860030209E9A3E0F8A3E036
:1009200060030209E9A3E064027002A3E06003022D
:1009300009E99003B8E02480600914604F14605CFA
:100940000209E9E860030209E99003B2E060047873
:1009500001800278009003C0E8F0A3E4F09003B1B6
:10096000E0600A9003C0E04402F0A3E4F09003A624
:10097000E0640460149003B374C0F0A37403F0A3A4
:10098000E4F0A37402120F8AF002100A90039FE0B1
:10099000640470559003C0E4F0A380D0E8547FF560
:1009A0000890039FE064047040E508C39406503942
:1009B000749F2508F582E43403F583E854806018B9
:1009C000A3A3A3A3A3A3A3E06403700478018002FC
:1009D00078009003C0E88091E582240CF5825002F3
:1009E0000583E0640370E980E39003A674048098B3
:1009F00074F7121BD6E9FE9003BE120F2B600302A0
:100A00000AD190039FE06404600B9003BC120F2B8B
:100A10006003020AD19003B8E0541F6009146030EB
:100A2000146020020AD19003BAE064017022EE90B3
:100A300003B1F060047905800279067A00121BD4B4
:100A4000020AD79003BCE0547FFA9003BAE0600535
:100A50007900020AD9EAC394065076EA90620EF051
:100A6000749F2AF8E43403F99003BCE05480602CAE
:100A7000EE6004741080027440906211F0EE600425
:100A800074038001E488828983A3A3A3A3A3A3A3FF
:100A9000F0EE6004790880307907802CEE600474F1
:100AA0002080027480906214F0EE60047403800170
:100AB000E4C0E0E8240CF582E439F583D0E0F0EE00
:100AC0006004790A80027909121BD490620EE480D6
:100AD000059003A67404F0790102100A7900120946
:100AE000F0E97003121BC32279011209F0E97003C7
:100AF000121BD222C082C0839003BC120F2B701530
:100B0000A3120F2B700F9003BA120CD05480FAE985
:100B1000FBEA4B60079003A67404801AE890620019
:100B2000F090039F6009E06402700C74038007E09A
:100B3000640370037402F0D083D0822274F3121B1A
:100B4000D69003BAE0FAA3E01460081460101460B1
:100B500039805712175F120CADA37B80804179005A
:100B6000121781120CAD7B80E92402F9E43AFA12E3
:100B70001E7CFC1919E0FAA3E92403F9E43AFA12FD
:100B80001E7CF9ECA3F0A3E9801CEAF91217EF90A0
:100B900003B3EAF0A3EBF0A3E4120CBCA37B0012B6
:100BA0001E7CA3F0A3E4F0020C679003B3E4F0A36F
:100BB000F0A3F0F50B90047DE0FAA3E0FB020C42F9
:100BC00075090074037808121F2BEA2508F8EB3525
:100BD00009F99003BA120CC6E493C0E0EFFCD0E030
:100BE0006C705DA3E4936E70579003BC120CC6A3A7
:100BF000A3E493C0E0EFFCD0E06C7044888289836A
:100C0000A3A3A3E4936E703888828983A3A3A3A3CC
:100C1000E493F508740193F5099003B3E508F0A394
:100C2000E509F0A37480F088828983A3A3A3A3A31A
:100C3000A3E493F8740193F99003B6E8F0A3E9F004
:100C4000050B850B0890047F120CD0C39AF50CE9B4
:100C50009BF50D7403780C121F5DC3E508950CE439
:100C6000950D5003020BC09003B3E0FCA3E0FDA37D
:100C7000E0FEEC4D4E9003A6700474048029E064FD
:100C80000460259003BEE0FAA3E0FB9003B6E0F811
:100C9000A3E0F9C3EA98EB9950089003B6EAF0A3F1
:100CA000EBF09003A67401F07F06021D7B9003B366
:100CB000EAF0A3EBF0A37480120CBC22F09003B313
:100CC000E0F9A3E0FA22E0FEA3E0FF888289832214
:100CD000E0F8A3E0F9E82274EE121BD6EA2404F847
:100CE000E43BF9880889098882F583E493602590BC
:100CF0000481120CD0FEE9FF8007EE2404FE5001AF
:100D00000F8E828F83E493F8740193F9EA6870027E
:100D1000EB6970E6750C00803F9062147490F0747B
:100D200010120E2A7003750D408E828F83A3A3A329
:100D3000E49355106006E50DD2E0F50DE50D9062E7
:100D400015F0EA906213F0EC240CF582E43DF58393
:100D5000E4F090620EF0050C850882850983E49327
:100D6000F8E50CC3984003020E257A0079051216A7
:100D7000F28A0E8B0FEA450F60DCEA2402F8E435B4
:100D80000FF9880A890B8882F583E493540FF512D2
:100D900090620EF0750D008A828B83A3A3A3A3E457
:100DA000932407F510A3E4933400F511740378102D
:100DB000121F5DAA10851210749F2510F8E43403E9
:100DC000F9E8FCE9FD751001751100E512781012C3
:100DD0001F2BE50E2403F8E4350FF9850A82850BF5
:100DE00083E493A2E74003020D199062117448F066
:100DF0007408120E2A7003750D408E828F83A3A390
:100E0000E49355106006E50DD2E0F50DE50D906216
:100E100012F0EA906210F08C828D83A3A3A3A3A3A7
:100E2000A3A3020D507F0B021D7BF088828983E40F
:100E3000935403640122C082C083120F287010A350
:100E4000120F2B700AA3E064017002A3E060079008
:100E500003A67404800C9003B374A0F0A37403126F
:100E60000F80F0020B3774F4121BD690039FE064DE
:100E70000260149003BC120F2B700CA3120F2B7086
:100E8000069003BBE060099003A67404F0020F23F0
:100E90007A007901121BD49003BAE060717A00F9EC
:100EA0001217818A088B09EA4509605A90039F74DA
:100EB00004F09003BAE09003A0F0750C008508825E
:100EC000850983A3A3A3A3E493F8E50CC398504C2E
:100ED000850C0A74A1250AF8E43403F9E8FEE9FF59
:100EE0008E828F83E4F07A0079041216F28A828B64
:100EF00083A3A3A3E493F88E828F83E06870E71244
:100F00000CD7050C80B79003A67404F0800E9003F4
:100F1000A0F090039F7403F0F91216587A0079023A
:100F2000121BD47F05021D7B9003BAE0F8A3E0F901
:100F3000E8492274F6121BD690039FE064047019EE
:100F40009003B8E064817011120F28700C9003BEFA
:100F5000E064017002A3E060079003A67404801AA5
:100F60009003BCE024A1F508A3E03403F509900345
:100F7000B3E508F0A3E509120F80F07F03021D7BA3
:100F8000F0A3E4F0A304120F8A22F0A3E4F090038C
:100F9000A6042274F7121BD690039FE064047064C9
:100FA0009003B8E06401705C9003BE120F2B705484
:100FB0009003BAE0FB9003BCE0FA9003A0E0F912C2
:100FC00017B98A088B09AE08AF09EE4F6036900357
:100FD000BCE0FA7903121BD49003BAE0C0E090039E
:100FE000BCE024A1F8A3E03403F988828983D0E02F
:100FF000F0EEFAEFFB120CD79003BCE0FA79041282
:101000001BD480069003A67404F07F02021D7BC0EF
:1010100082C0838003121A39A2E840F9A823E85459
:101020000460097823E654FBF6121402A823E8545E
:101030001060097823E654EFF6121420A823E8A2E2
:10104000E05005782354FCF690620EE0FA7404F048
:10105000906214E0A2E0503AE5A8F8C2AF906216A0
:10106000E0F9A3E0E9FBE8A2E792AF8017906228DD
:10107000E0C0E0900393E0F8121112D0E0F090038A
:1010800093E004F0EBFC74FF2C1B0470E0906214FE
:10109000E4F0EA90620EF0E0FD7404F0906211E07A
:1010A000A2E04031900395E0F8900394E068602559
:1010B0007A40900394121155E0906228F0900394C6
:1010C000E004F008900395E06860041AEA70E39089
:1010D00062117401F0ED90620EF0D083D082227420
:1010E000F8121BD6E9FE79008012121112E08A82F2
:1010F0008B83F0900392E00412114A09900392E06E
:10110000F8900393E0686005E9C39E40DD7F01022B
:101110001D7B748528F582E43404F58322C082C0E7
:1011200083E9FC80188A828B83E0C0E090039512EB
:101130001155D0E012114A900395E004F0ECF874D8
:10114000FF281C0470DF79018090F08A828B83A3D2
:10115000AA82AB8322E0F8748528F582E43405F591
:101160008322C082C083900395E0F8900394E068E6
:1011700060047901800279000210DA02100F74FB1A
:10118000121EC57E009006857808121F7B794A12D0
:1011900013B29006857401F0A3F0A37469F0A374F0
:1011A000A5F09003D77808121EF070030E801590FA
:1011B00003DB7808121EF06008E59D541864107077
:1011C00003022000EEF9121329C280D291EEA2E0B0
:1011D00050030212DCAA18AB19120288E97003024C
:1011E00012DCC291851882851983E0C3943C500EAD
:1011F000E0F8743CC398F50895E0F5098006750899
:1012000000750900E4F50AF50B9003DF780C121F56
:101210007B7808790C121ADA790612015112100F34
:10122000120176E9F8740968700779061201518095
:10123000277407686016A2935012E8600874066865
:1012400060030212DCA292400F0212DC75080075E6
:101250000900750A00750B0085080C85090D850AC3
:101260000E850B0F9003C27808121F05E50C450D83
:10127000450E450F70A7D2807907120151800312E5
:10128000100F121162E970F77E007F007401121FC7
:1012900097E4F0A37426F0A3E4F0A3F07401121F06
:1012A000977808121F7B85080C85090D850A0E8525
:1012B0000B0F9003C2780C121F057401121F977850
:1012C0000C121F6CE5084509450A450B70CEA29229
:1012D00050FCA29350F81213AD022000D280D2919C
:1012E000794E1213B2750800750900750A00750B66
:1012F00000790512015112100F120176E9F87409F4
:101300006860EE74016870EE12100F9003E37808C5
:10131000121F059003E77808121E0950EB1213AD57
:101320000220007405121E462274F8121BD6E9FE34
:1013300053BEFBE59DA2E650FA0078F8790100E87B
:1013400024FF18E934FFF9E84970F375C68074800A
:10135000659E70FA43BE049062707408F01213A286
:10136000EE700853F4FEC29043FE017403F5D57588
:10137000D489900396E4F0A374C2F0A37401F0A39F
:10138000E4F0A3F0A3F0A37408F01213C87AFF7B73
:10139000FF1219F453F4FED29043FE011213A2027D
:1013A000110DD28043FD01C29143FE0222D280C2C0
:1013B0009122781075B60FE5B4A2E750FAE5BBC3E9
:1013C0009940F118E870ED22C082C0837A0079015B
:1013D0001217818A828B83A3A3A3A3A3A3A3E4935D
:1013E000A2E69003B2500474018001E4F09003B1CE
:1013F000E4F090620F7403F0E0A2E750FBD083D0DA
:101400008222C082C08390039F7402F0A3E4F09014
:1014100003A6F0790312165875210075220080DDAD
:1014200074F6121BD690620EE0FEE4F0906211E0BA
:10143000FFA2E4501D7480F09003A67407F0E5212C
:1014400045226009852182852283121FA69003A66A
:10145000E4F0EFA2E2500B906211E4F09003A6F0EA
:1014600080669003A6E0F87402687045906216E00A
:10147000FF9003B3121DBBEFF97A207B6212168C2A
:101480007403121E468F089003B612163C121634CF
:101490002F121647E0F8A3E0F9E849600474408091
:1014A000027448906211F0E849600302162A02169D
:1014B000067406687009852182852283121FA69012
:1014C00003A6E060030215B1EFA2E0400302162A72
:1014D0007508B8750903750A007808121EDB7908CB
:1014E0007A207B6212168C7403121E4675210075D9
:1014F00022009003B8E054E0601D24E07003021560
:101500008D24E0607224C0604824E07003021598C6
:1015100024E0606E0215A3A3E014602624FE601D83
:1015200024FE600A24FC601F24FE60208075120ADD
:10153000F49003A6E06404707274608070120AE88C
:1015400080EF120ADC80EA120E6680E5120F9380AB
:10155000E0A3E0600E24FA600F24FE601024FE6019
:1015600011804012090E80C9120B3C80C4120E3645
:1015700080BF120F3380BA7521BF75221B121BBFAB
:1015800080AF7521C175221B121BC180A475215A21
:1015900075221B121B5A809975218A75221B121BFA
:1015A0008A808E9003A67404F0808E74409062113D
:1015B000F09003A6E0F874016870617F029003B6B2
:1015C000E0F8A3E0F9C3E89420E994005007E8F5B7
:1015D0000A7F0A8003750A209003B3121DBBA90A73
:1015E0007A207B621216B77403121E46850A08120F
:1015F0001634250812164712163CEF906211F0E5DA
:101600000AC394205024E521452260098521828562
:101610002283121FA69003A6E4F0800E7405687062
:1016200009852182852283121FA6EE90620EF07F2B
:1016300003021D7B9003B31216E4E922C3E0950870
:10164000F0A3E09400F022F9E43AFA9003B3E9F051
:10165000A3EAF0A3EBF0A32274F7121BD678007470
:10166000A728F582E43403F583E9F008E8C394057C
:1016700040ED780074AC28F582E43403F583E9F09A
:1016800008E8C3940540ED7F02021D7B74F8121B2D
:10169000D6EAFCEBFDE9F87408121F971216DF601A
:1016A000118C828D83E0121EAFE9240109E43AFA1D
:1016B000D8EF7F01021D7B74F8121BD6EAFCEBFD0C
:1016C000E9F87408121F971216DF6011121E7C8C45
:1016D000828D83F0E9240109E43AFAD8EF80D3122D
:1016E00016E4E822E0F9A3E0FAA3E0FB22D083D0DD
:1016F0008222C082C083E9FCEAFD7A007B0080037D
:1017000012173D90039DE0F8A3E0F990047BE06898
:101710007003A3E069602490039EE0F5838882A3B0
:10172000E493F8EC68700D90039DE0FAA3E0FB12DF
:10173000173D8007ED6870C8ED60C580B090039DCF
:10174000E0F8A3E0F5838882E493F890039DE02815
:10175000F8A3E03400F990039DE8F0A3E9F022C07B
:1017600082C0831217707A0079011216F20216ED08
:10177000900479E0F8A3E0F990039DE8F0A3E9F084
:101780002274F7121BD6E9FEEAFF1217707A00796D
:10179000021216F2EA4B601CEE60108A828B83A361
:1017A000A3A3A3A3E4936E70E48009EFF874FF2869
:1017B0001F0470D97F02021D7B74F5121BD6EAFF4D
:1017C0008B087A001217817A0279041216F2EA4B1A
:1017D00060188A828B83A3A3E4936F70EA8A828B5A
:1017E00083A3A3A3E493650870DD7F04021D7B74CB
:1017F000F7121BD674F0121EC5E97A007B00600C4C
:101800001460101460141460180218DB7AF37B0360
:101810000218DB7AF77B030218DB7A1B7B040218C1
:10182000DB90043FE060030218D79003EB740812CA
:101830001F467408121DE8750808F5097808121E7D
:10184000DF7402121F467AE87B07797F1218F27460
:1018500002121E467808121EDF740A121F46740216
:10186000121F3E121C997402121E468B09EA45098A
:1018700070197509007808121EDF7C0C7D787402DF
:10188000121F3E121D357402121E467C287D0085F3
:101890001882851983E5822DF582E43583F583E08E
:1018A000FF743F2CF8E43404F9EF1218E3888289BE
:1018B00083F0EFC41218E3C0E0E824FEF582E934B7
:1018C000FFF583D0E0F00D74FC2CFCEDC3940840D0
:1018D000BE90043F742AF07A3F7B047410121E46B7
:1018E0000217B4540FFA74692AF582E43404F583BC
:1018F000E02274F5121BD68908740F5508F50A7595
:101900000B00740B780A121F2BEA2400F8EB3480CA
:10191000F9E82400E9350BF9E5C7F509A2AFE4338E
:10192000F50AC2AFE508C4540FFAE5C754F84AF502
:10193000C7740B121F97E0FAA3E0FB801C88828912
:1019400083E08C828D83F088828983A3A882A98317
:101950008C828D83A3AC82AD83EAFEEBFFEE24FF85
:101960001AEF34FFFBEE4F70D48509C7E50AA2E0F9
:1019700092AF7F04021D7B74F7121BD6ED90038992
:10198000F0ECA3F0A37462F0A37473F0A3E0541F0F
:10199000F07409121F97E0F508A3E0F509E5083394
:1019A0003354FC90038EF074067808121F5DE5082E
:1019B00090038DF090038F7412F0A37442F075D1F0
:1019C000FE75D601EA906271F0EBA3F0906270E0D0
:1019D000D2E1F0E0A2E740FB7F02021D7BC082C0A3
:1019E00083E9C333906272F0906270E0D2E0F0D08D
:1019F00083D0822274F7121BD675230075240075DC
:101A000025008A268B27EA90620BF08A088B0974DE
:101A1000047808121F5DE508906207F08A088B09B8
:101A200074097808121F5DE508543E906209F0754C
:101A30008B00C2E87F02021D7B74F7121BD6E59D66
:101A4000A2E650FA906206E0FAA2E25035A826E833
:101A500090620BF0F50885270974047808121F5D61
:101A6000E508906207F0852608852709740978083B
:101A7000121F5DE508543E906209F0906201E0D2C9
:101A8000E0F07823EA46F6906202E0F50875090076
:101A900074047808121F2B7823E50846F608E50938
:101AA00046F6906204E0F50875090074097808129A
:101AB0001F2B7824E50946F6EAA2E05003752501BC
:101AC00074065A6003752500E58BA2E55006758BF8
:101AD000DF752500121BD5021A2F080808EAC0E09E
:101AE000EBC0E086F0E7A4FA180986F0E7A42AFA2A
:101AF000180986F0E7A42AFA180986F0E7A42AFA5A
:101B00001986F0E7A4FBE5F02AFA190886F0E7A4A5
:101B10002BFBE5F03AFA190886F0E7A42BFBE5F079
:101B20003AFA18180986F0E7A4C5F02BFBE43AFA54
:101B30001908E7C5F0C6A426F6E5F03BFBE43AFA3F
:101B40001886F0E7A4F6E5F00826F6E43B08F6E48C
:101B50003A08F6D0E0FBD0E0FA22C082C0839003BE
:101B6000B9E0F874226870089003A6E0701A80113A
:101B70007420689003A6700DE0700D121BB19003E5
:101B8000A6740280027404F08043C082C083900374
:101B9000B9E064219003A67013E07013121BB1A387
:101BA0007407F0A3E4F09003A60480027404F080AC
:101BB0001C9003B37496F0A37403F0A3E4F02280A6
:101BC000028000C082C0839003A67404F0D083D04A
:101BD000822280EF22222518C582C0E0E51934FF59
:101BE000C583C0E0E518C3958224F910AF0885834A
:101BF000198582188008858319858218D2AFCEF0A6
:101C0000A3E520F0A37808E608F0A3DEFAEFF0A33E
:101C1000E58124FBF8E608F0A3E608F0A30808E64F
:101C200008F0A3E608F0A315811581D0E0FED0E00E
:101C3000F815811581E8C0E0EEC0E0221201000233
:101C4000020000205104A816090001020301090244
:101C50004300020100801909040000010202010092
:101C600005240010010424020205240600010524B5
:101C70000100010705820340004009040100020A37
:101C80000000000705840240000007050402400030
:101C900000571C00007A1C000074F5121BD6740B50
:101CA000121F97E0F8A3E08015A3AA82AB838C8271
:101CB0008D83A3AC82AD83E824FF18E934FFF9E8F3
:101CC00049601F8C828D83E0F5088A828B83E0F562
:101CD0000AE508650A60D2E50AC39508FA95E0FBB3
:101CE00080047A007B007F04021D7BE47921780761
:101CF000B800028004F709D8FCE490030278C179A7
:101D0000018002F0A3D8FCD9FA7AC27B0390008E3E
:101D100078C479018015E493A3AD82AE838A828B67
:101D200083F0A3AA82AB838D828E83D8E9D9E71290
:101D3000117E121FA174F7121BD6EAF8EBF9740991
:101D4000121F97E0FEA3E0FF80188C828D83E0884D
:101D5000828983F0A3A882A9838C828D83A3AC821D
:101D6000AD838E088F09E50824FF1EE50934FFFFC7
:101D7000E508450970D47F02021D7B85198385180B
:101D800082E0A3FEE0A3F5207808E0A3F608DFFADE
:101D9000E0A3FFE0A3C0E0E0A3C0E0E0A3C0E0E078
:101DA000A3C0E010AF08858218858319800885825A
:101DB00018858319D2AFD083D0822274038000CCDF
:101DC000C0E0EDC0E0E518C39CCCAD1950011D107A
:101DD000AF068C188D1980068C188D19D2AF121D84
:101DE000E8D0E0FDD0E0FC22CAC0E0E0A3C582CC90
:101DF000C582C583CDC583F0A3C582CCC582C5830A
:101E0000CDC583DAE6D0E0CA22C008C3E096F50863
:101E100008A3E096420808A3E096420808A3E096CB
:101E200045087001D3D00822C5822518C582C58314
:101E3000351910AF07F5198582188007F5198582C5
:101E400018D2AFC5832200C0D0251810AF08F518EE
:101E5000500C05198008F51850020519D2AFD0D0E2
:101E6000222518F58210AF08F518400C15198008C6
:101E7000F51840021519D2AF85198322BB0102E77C
:101E800022C082C08389828A83BB0003E08002E48F
:101E900093D083D082226016080808C6C313C618E0
:101EA000C613C618C613C618C613C6D5E0EA22BBA9
:101EB000000EC082C0838A838982F0D083D08222C0
:101EC000BB0101F722251810AF08F518400C1519B1
:101ED0008008F51840021519D2AF227403800474EB
:101EE000028000C0E0F404121E61D0E0121F8A22BA
:101EF000E066701008A3E066700A08A3E06670044C
:101F000008A3E06622E026F608A3E036F608A3E080
:101F100036F608A3E036F622E627F60809E637F695
:101F20000809E637F60809E637F622700422600D44
:101F300018C6C333C608C633C6D5E0F41822251820
:101F4000FAE43519FB222518FCE43519FD2275D079
:101F50000075813F751802751903021CEB600C08AF
:101F6000C6C313C618C613C6D5E0F422E6F008A30C
:101F7000E6F008A3E6F008A3E6F022E0F608A3E006
:101F8000F608A3E0F608A3E0F622CAC0E0E6F0A354
:101F900008DAFAD0E0FA222518F582E43519F5833B
:101FA0002200000080FBE473FFFFFFFFFFFFFFFF45
:101FB000FFFFFFFFFFFFFFFFFFFFFFFFFFFFFFFF31
:101FC000FFFFFFFFFFFFFFFFFFFFFFFFFFFFFFFF21
:101FD000FFFFFFFFFFFFFFFFFFFFFFFFFFFFFFFF11
:101FE000FFFFFFFFFFFFFFFFFFFFFFFFFFFFFFFF01
:0A1FF600850609433886000000004C
:020000040003F7
:01FFF000F020
:020000040000FA
:10200000022DA8022221FFFFFFFFFFFFFFFFFFFFBE
:10201000FFFFFFFFFFFFFFFFFFFFFFFFFFFFFFFFD0
:10202000FFFFFFFFFFFFFFFFFFFFFF022A6CFFFF25
:10203000FFFFFF022244FFFFFFFFFFFFFFFFFFFF45
:10204000FFFFFFFFFFFFFFFFFFFFFFFFFFFFFFFFA0
:10205000FFFFFF02215DFFFFFFFFFFFFFFFFFFFF0D
:10206000FFFFFFFFFFFFFFFFFFFFFF022A44FFFF0D
:10207000FFFFFFFFFFFFFFFFFFFFFF022895FFFFAE
:10208000FFFFFF0221BD01FFFFFFFFFFFFFFFFFF7B
:102090001020102001FF01010503010F10FEFFA217
:1020A0004F000000003A4F00000000FF000000FF5A
:1020B00000010000873B00000000D93AD13C213BE1
:1020C0003B3C00000F3B000000000000000000004F
:1020D0000000000000000000000000000000FF0100
:1020E0000100AA07000000E803FFFF250803E8033A
:1020F00064006400B8010202000800000502070441
:1021000001051E02051E020A0A0103B80B02803EE9
:102110000102FEFFE8030A050001FFFF0A01E000DB
:1021200020FD000206FFFF00035F005F0030005843
:10213000000000000000000000000000000000009F
:10214000000000000000000000000000000000008F
:1021500000B5260A270A270A270A271227C0E07493
:10216000F2122656A2AFE433FED2AFE5A7FFE5A1F7
:10217000F5085F5410600612467975A1EFE5085F17
:102180005408600812467F75A1F78024E508A2E094
:1021900092F0EFA2E082F05017906198E0F8900A78
:1021A00009E0C398A2D265D0335002E8F075A1FED1
:1021B000751A00EEA2E092AF7F01022712C0E07410
:1021C000F2122656A2AFE433FED2AF9061A4E0F83B
:1021D000759B00E59158540860087591F71246C741
:1021E0008023E59158541060087591EF1246CD8018
:1021F00014E591A2E092F0E8A2E082F05007E0C27C
:10220000E0F01248239061A3E0F8E5E95854046037
:102210000E1247F975E9FB906193E0A2E640F28067
:102220008FC0E074F2122656A2AFE433FED2AF9014
:1022300061A5E0F8E5BF585404600675BFFB12487D
:102240003B0221B0C0E074F1122656E59DA2E65093
:10225000FA906206E0FAA2E25035A82CE890620BF0
:10226000F0F508852D0974047808122DB8E508905A
:102270006207F0852C08852D0974097808122DB89D
:10228000E508543E906209F0906201E0D2E0F078F7
:1022900029EA46F6906202E0F508750900740478B0
:1022A00008122D447829E50846F608E50946F69017
:1022B0006204E0F50875090074097808122D447865
:1022C0002AE50946F6EAA2E05003752B0174065A86
:1022D0006003752B00E58BA2E55006758BDF752B2F
:1022E000001249EB758B00C2E87F02022712C3E49B
:1022F00098F8E499F912232F8026C3E49AFAE49B14
:10230000FBE920E7E912232FE498F8E499F922C3C6
:10231000E498F8E499F912232FE498F8E499F9C3C2
:10232000E49AFAE49BFB22EB20E7CFE920E7E0B94F
:102330000010BB0008E88AF084F8AAF022E4FBC889
:10234000FA22EB70227B10C833C8C933C933500757
:10235000C39AC3DBF280069A50012ADBEAC833F441
:10236000C8C933F4C9FA2275F008E4C833C8C933C0
:10237000C933C99AC99B5004C92AC93BD5F0ECFBA3
:10238000C833F4C8E4C9FA2274F51225F074FA12BD
:102390002C187508047509007808122B567404125D
:1023A0002BFA7AF87B0779031245537402122B84B7
:1023B0009080FC7808122DD67402122E2D78081207
:1023C0002C4470497508027509007808122B567460
:1023D00002122BFA7AF67B07790312455374021224
:1023E0002B84851882851983E0F47003A3E0F460E0
:1023F0001C851882851983E0F8A3E0F98882898317
:102400007402F0A3F0A37469F0A374A5F0C2AF75D1
:10241000D69F0200007406122B847F040228D8087D
:102420000808EAC0E0EBC0E086F0E7A4FA180986E5
:10243000F0E7A42AFA180986F0E7A42AFA18098610
:10244000F0E7A42AFA1986F0E7A4FBE5F02AFA19C6
:102450000886F0E7A42BFBE5F03AFA190886F0E7C6
:10246000A42BFBE5F03AFA18180986F0E7A4C5F0AA
:102470002BFBE43AFA1908E7C5F0C6A426F6E5F006
:102480003BFBE43AFA1886F0E7A4F6E5F00826F6F6
:10249000E43B08F6E43A08F6D0E0FBD0E0FA22127A
:1024A0002E22B900030224FFE47921780DB800023E
:1024B0008004F709D8FCE49004D178ED790C80020F
:1024C000F0A3D8FCD9FA781A9020867A01BA0002D3
:1024D0008007E493A3F608DAF97ABD7B1090209484
:1024E00078CA79018015E493A3AD82AE838A828B8A
:1024F00083F0A3AA82AB838D828E83D8E9D9E77556
:10250000820D7583B27406122B307582CD75834CA3
:102510007400122B30E4CFC0E0E4CEC0E0E4CDC0C4
:10252000E0E4CCC0E075F020E626F608E633F608D5
:10253000E633F608E633F6181818EC33FCED33FDF5
:10254000EE33FEEF33FFC3EC9709ED9709EE9709E1
:10255000EF97191919400FFFEC97FC09ED97FD094A
:10256000EE97FE191906D5F0BFECF709EDF709EE65
:10257000F709EFF7191919D0E0FCD0E0FDD0E0FE23
:10258000D0E0FF222518C582C0E0E51934FFC583DD
:10259000C0E0E518C3958224F810AF08858319853B
:1025A00082188008858319858218D2AFCEF0A3E502
:1025B00020F0A37808E608F0A3DEFAEFF0A3E581A7
:1025C00024FAF8E608F0A3E608F0A3E608F0A3086A
:1025D00008E608F0A3E608F0A315811581D0E0FE17
:1025E000D0E0F8158115811581E8C0E0EEC0E02249
:1025F0002518C582C0E0E51934FFC583C0E0E518A1
:10260000C3958224F910AF08858319858218800844
:10261000858319858218D2AFCEF0A3E520F0A37888
:1026200008E608F0A3DEFAEFF0A3E58124FBF8E664
:1026300008F0A3E608F0A30808E608F0A3E608F00F
:10264000A315811581D0E0FED0E0F815811581E851
:10265000C0E0EEC0E022C0D02518C582C0E0E51978
:1026600034FFC583C0E0E518C3958224F310AF089A
:102670008583198582188008858319858218D2AFD1
:10268000C8F0A3E9F0A3EAF0A3EBF0A37908E70907
:10269000F0A3D8FAECF0A3EDF0A3EEF0A3EFF0A3D3
:1026A000D0E0F0A3D0E0F0A3D0E0F0A3E520F0A3C9
:1026B000E5F0F0A32212010002020000205104A85C
:1026C00016090001020301090243000201008019FA
:1026D0000904000001020201000524001001042485
:1026E00002020524060001052401000107058203FA
:1026F00040004009040100020A00000007058402AE
:1027000040000007050402400000D0260000F32628
:102710000000851983851882E0C0E0A3E0F9A3E0FA
:10272000FAA3E0FBA37808E0F608A3DFFAE0FCA335
:10273000E0FDA3E0FEA3E0FFA3E0C0E0A3E0C0E073
:10274000A3E0F5D0A3E0F520A3E0A3F5F010AF08D7
:102750008583198582188008858319858218D2AFF0
:10276000D082D083D0E0F8D0E032E47375F0108EE0
:10277000218F22858226858325851882851983E00D
:10278000CEA3E0CF852682852583EBC9EAC8EDCBB1
:10279000ECCAC3E833C8E933C9EA33CAEB33CBC365
:1027A000EA9EF524EB9FF523B35004AB23AA24EC57
:1027B00033CCED33CDD5F0DAAE21AF2222D083D0A9
:1027C00082ECC0E0EDC0E0E493A3FCE493A3FDED54
:1027D0004C600D122918EC24FFFCED34FFFD80EF56
:1027E000E493A3FCE493A3FDED4C600D1229EFEC00
:1027F00024FFFCED34FFFD80EFD0E0FDD0E0FCE4F1
:1028000093A3C0E0E493C0E022851983851882E099
:10281000A3FEE0A3F5207808E0A3F608DFFAE0A322
:10282000FFE0A3C0E0E0A3C0E0E0A3C0E0E0A3C0FD
:10283000E0E0A3C0E010AF08858218858319800806
:10284000858218858319D2AFD083D082022B36D0EF
:1028500083D082E9C0E0E493A3C386F0C5F095F08D
:10286000F908E493A386F0C5F095F0700BE493A308
:10287000C3994005E9048002A3E475F002A425820F
:10288000F582E5F03583F583D0E0F9E493A3C0E069
:10289000E493C0E022C0E074F2122656A2AFE43303
:1028A000FED2AFE58AA2E250079009CAE0D2E0F07A
:1028B000E58AA2E350079009CAE0D2E1F0758A00E8
:1028C000C2EB7A107B009009C6E0F9123E63EEA2DB
:1028D000E092AF7F01022712851983851882E0A359
:1028E000FEE0A3F5207808E0A3F608DFFAE0A3FFF6
:1028F000E0A3C0E0E0A3C0E0E0A3C0E0E0A3C0E04C
:1029000010AF088582188583198008858218858311
:1029100019D2AFD083D08222C0E0C3E4939608746A
:1029200001939618400FE49366700808740193664B
:102930001870007019A3A3C3E493960874019396CA
:1029400018A3A3400DD0E0D0E0D0E00227F9A3A364
:10295000A3A3A3A3D0E022D083D082C5F0E493A3A5
:10296000C5F0C395F0F5F0E493A3C395F04005E5F9
:10297000F0048001E475F002A42582F582E5F035CB
:1029800083F583E493A3C0E0E493C0E02274048061
:10299000087403800474028000CCC0E0EDC0E0E560
:1029A00018C39CCCAD1950011D10AF068C188D19A1
:1029B00080068C188D19D2AF122AB2D0E0FDD0E07B
:1029C000FC2274028000CCC0E0EDC0E0E518C39C9E
:1029D000CCAD1950011D10AF068C188D1980068CD6
:1029E000188D19D2AF122A90D0E0FDD0E0FC22C0A1
:1029F000E0C0F088F0E493667008087401936618EC
:102A00007000A8F0A3A3700BD0F0D0E0D0E0D0E02D
:102A10000227F9A3A3D0F0D0E022D083D082CCC08B
:102A2000E0E493A36006122AD31470FAE493A3603F
:102A300006122C021470FAD0E0FCE493A3C0E0E488
:102A400093C0E022C0E074F2122656758900C2C518
:102A50009010B5E0700E7A007B1090071EE0F9121E
:102A60003E638003124B2F7F01022712C0E0C0D0CB
:102A7000E8C0E0E9C0E0E5A8D2AFC2C7751A00A27D
:102A8000E7A2E792AFD0E0F9D0E0F8D0D0D0E032C2
:102A9000CAC0E0E493A3C582CCC582C583CDC583FB
:102AA000F0A3C582CCC582C583CDC583DAE5D0E06D
:102AB000CA22CAC0E0E0A3C582CCC582C583CDC509
:102AC00083F0A3C582CCC582C583CDC583DAE6D0A9
:102AD000E0CA22C0E0E493A3D39C5010E493A3C3C4
:102AE0009C400AD0E0D0E0D0E0022A37A3A3A3D0D4
:102AF000E0227009080808226016181818C6C333A7
:102B0000C608C633C608C633C608C633C6D5E0EA0B
:102B100022C008C3E096F50808A3E096420808A37F
:102B2000E096420808A3E09645087001D3D0082239
:102B3000C09FF59FE473D09F22D083D082C09FE4D2
:102B400093C0E0740193C0E0740293F59F22740473
:102B5000800A74038006740280027401C0E0F404E9
:102B6000122B69D0E0122DE5222518F58210AF084E
:102B7000F518400C15198008F51840021519D2AF48
:102B80008519832200C0D0251810AF08F518500C05
:102B900005198008F51850020519D2AFD0D022BB14
:102BA0000102E722C082C08389828A83BB0003E0DE
:102BB0008002E493D083D082226016080808C6C33E
:102BC00013C618C613C618C613C618C613C6D5E052
:102BD000EA22C3E0C696F608A3E0C696F608A3E08C
:102BE000C696F608A3E0C696F6222518F8E435192D
:102BF000F9222518FAE43519FB222518FCE43519C9
:102C0000FD22C0E0E493A36C7009D0E0D0E0D0E0F6
:102C1000022A37A3A3D0E022251810AF08F51840E8
:102C20000C15198008F51840021519D2AF22BB0007
:102C30000EC082C0838A838982F0D083D08222BB77
:102C40000101F722E066701008A3E066700A08A38D
:102C5000E066700408A3E06622C3E09608A3E0964D
:102C600008A3E09608A3E096A2D265D03322E766D7
:102C700070100809E766700A0809E7667004080919
:102C8000E76622C3E096F008A3E096F008A3E0967A
:102C9000F008A3E096F022C3E4939608740193969B
:102CA0000874029396087403939622C3E697F60875
:102CB00009E697F60809E697F60809E697F622E08E
:102CC00026F608A3E036F608A3E036F608A3E036B9
:102CD000F622E657F60809E657F60809E657F60819
:102CE00009E657F622E056F608A3E056F608A3E0F8
:102CF00056F608A3E056F622E056F008A3E056F098
:102D000008A3E056F008A3E056F022E627F60809EB
:102D1000E637F60809E637F60809E637F622E02630
:102D2000F008A3E036F008A3E036F008A3E036F0A0
:102D300022E647F60809E647F60809E647F60809D5
:102D4000E647F622700422600D18C6C333C608C6D3
:102D500033C6D5E0F41822E4C396F608E496F608E4
:102D6000E496F608E496F622C6F4C608C6F4C60849
:102D7000C6F4C608C6F4C622600D08C6A2E713C68C
:102D800018C613C6D5E0F322C3E7960809E79608EC
:102D900009E7960809E79622C3E09608A3E096089B
:102DA000A3E09608A3E0962275D00075813F7518C0
:102DB000D17519040002249F600C08C6C313C618FD
:102DC000C613C6D5E0F422E6F008A3E6F008A3E6B1
:102DD000F008A3E6F022E0F608A3E0F608A3E0F688
:102DE00008A3E0F622CAC0E0E6F0A308DAFAD0E0D1
:102DF000FA22EAF0A3EBF0A3ECF0A3EDF022E0FA64
:102E0000A3E0FBA3E0FCA3E0FD22E0F8A3E0F9A32C
:102E1000E0FAA3E0FB22E8F0A3E9F0A3EAF0A3EBD9
:102E2000F022E5C754F84401F5C77901222518F5C9
:102E300082E43519F58322122B39DCAC02122B39CE
:102E40000CAD02122B39A5AE02122B3961AF021262
:102E50002B3919B002122B396EB002122B39D1B0B6
:102E600002122B390FB102122B3939B102122B3950
:102E7000C5B102122B391EB202122B397FB20212D7
:102E80002B39BEB402122B3992B602122B3971B70C
:102E900002122B39AAB802122B395DBB02122B3950
:102EA00070BE02122B397FBE02122B390BBF0212E9
:102EB0002B39C1BF02122B3908C002122B3951C065
:102EC00002122B398DC002122B3903C102122B3989
:102ED0006FC102122B398BC102122B39BCC10212F5
:102EE0002B39FBC102122B39FCC202122B39ABC3A6
:102EF00002122B393CC602122B3995C702122B390C
:102F000028C802122B39B2C802122B39D6C80212B5
:102F10002B3987C902122B3938CA02122B39B5CB8B
:102F200002122B3940CC02122B397FCC02122B39E2
:102F3000F5CC02122B394ACE02122B39EDCE0212F9
:102F40002B3921CF02122B3939CF02122B39DCCF8A
:102F500002122B3966D202122B3907D402122B39F6
:102F600025D402122B3943D402122B3913D5021265
:102F70002B3968D802122B39008003122B395A8062
:102F800003122B39C48003122B394D8103122B39C4
:102F9000098203122B39518203122B398C820312BE
:102FA0002B39E28203122B394A8303122B39CE8349
:102FB00003122B39E78303122B390C8403122B39AC
:102FC0002B8403122B39698403122B39B884031222
:102FD0002B39E18403122B39308503122B39DC8520
:102FE00003122B39A48603122B39098703122B39BC
:102FF000D68703122B391C8803122B393888031209
:103000002B396A8803122B39128A03122B39E98A69
:1030100003122B39158B03122B394B8B03122B39CF
:103020006C8B03122B397B8B03122B39868B03128B
:103030002B393A8C03122B39AD8C03122B391F8D8F
:1030400003122B39278D03122B39A28D03122B3932
:10305000FB8D03122B393E8E03122B39D0900312B5
:103060002B39169203122B39A69403122B398E9505
:1030700003122B39C19503122B39839603122B3976
:10308000329703122B397A9703122B39DC970312EC
:103090002B39019803122B39129803122B398A9875
:1030A00003122B39129903122B39769903122B39FB
:1030B0005B9A03122B39809A03122B39A19B0312BE
:1030C0002B39BF9B03122B39D29B03122B39459C02
:1030D00003122B39549C03122B39DC9C03122B391D
:1030E000249D03122B39319D03122B393A9D031273
:1030F0002B393A9F03122B398EA003122B399EA035
:1031000003122B39BAA103122B3933A203122B3924
:1031100069A303122B39ABA303122B39E7A30312C4
:103120002B39BBA503122B3920A803122B3934A845
:1031300003122B393EA803122B3948A803122B394E
:1031400052A803122B395CA803122B3975A803125D
:103150002B397FA803122B3989A803122B3993A886
:1031600003122B39C2A803122B39EAA803122B39F8
:10317000F5A803122B393FA903122B3949A90312D1
:103180002B3954A903122B3978A903122B399CA986
:1031900003122B39FDA903122B3948AA03122B392C
:1031A00064AA03122B39CEAA03122B391AAB0312CD
:1031B0002B3962AB03122B39DDAB03122B3977AC01
:1031C00003122B393BAE03122B39A9AE03122B3954
:1031D000DBAF03122B3901B003122B3971B103128B
:1031E0002B3925B503122B3925B703122B39FDB81E
:1031F00003122B3996B903122B39A8BB03122B39B2
:103200006ABC03122B39B6BC03122B391CBD031246
:103210002B392EBD03122B397EBF03122B396DC003
:1032200003122B39ACC103122B39FEC103122B3907
:10323000A3C203122B395EC403122B398FC50312AC
:103240002B39ADC503122B3902C603122B3900C727
:1032500003122B3928C703122B398BC703122B39C2
:103260008CC803122B39FFC803122B392DCA031245
:103270002B3998CA03122B3988CB03122B39EECD88
:1032800003122B391CCE03122B3917CF03122B3903
:10329000B5D003122B3905D103122B39BDD103123E
:1032A0002B3972D203122B39D6D203122B398FD37A
:1032B00003122B392FD403122B3993D403122B3939
:1032C000DDD403122B391AD503122B3982D60312FF
:1032D0002B39798101122B39BB8101122B39B6842C
:1032E00001122B39098501122B394F8501122B3917
:1032F000908601122B39F58601122B393587011280
:103300002B39788801122B39BA8B01122B39E38CB7
:1033100001122B39249801122B39C49801122B3930
:10332000B79B01122B39EE9C01122B39649D0112BF
:103330002B398E9E01122B39DE9F01122B39C5A02D
:1033400001122B392EA301122B393CA501122B3966
:10335000CDA501122B39A1A601122B392DA70112DF
:103360002B3937A701122B395FA701122B390CA873
:1033700001122B39F7A801122B39CAA901122B39D6
:1033800057AA01122B396DAA01122B39D1AA0112A9
:103390002B39FAAA01122B3927AB01122B396CAD4C
:1033A00001122B3947AE01122B398BAE01122B398A
:1033B000FCAE01122B39B5AF01122B39E7AF011268
:1033C0002B392EB001122B3961B001122B39C6B046
:1033D00001122B3915B101122B391AB101122B39F7
:1033E0006EB101122B39B8B101122B39B4B20112EE
:1033F0002B3919B301122B3977B301122B39C1B60E
:1034000001122B3995B701122B3922B901122B3930
:10341000FCBB01122B39AFBC01122B39D6BE0112F5
:103420002B397BBF01122B39B9BF01122B3989C14E
:1034300001122B399CC101122B39A5C101122B3964
:10344000AEC101122B39C3C101122B39E2C10112E5
:103450002B3917C401122B396AC401122B3974C4D9
:1034600001122B397EC401122B39D9C401122B3918
:1034700035C501122B394DC601122B39AEC60112CA
:103480002B39FDC701122B3946C801122B391EC931
:1034900001122B3949CA01122B39FFCA01122B39EB
:1034A00001CC01122B3903CD01122B39E8CD0112C9
:1034B0002B39FFCD01122B393CCE01122B3946CED0
:1034C00001122B3950CE01122B395BCE01122B3950
:1034D00079CE01122B39BBCE01122B3919CF011233
:1034E0002B393ECF01122B3958CF01122B39E5CFA2
:1034F00001122B391ED001122B396ED101122B393A
:10350000C5D101122B39DFD201122B3915D301128B
:103510002B39B1D301122B392DD401122B399DD562
:1035200001122B39B8D601122B397ED701122B3953
:1035300028D801122B39ADD801122B3915D9011217
:103540002B39CAD901122B391CDA01122B3991DA25
:1035500001122B395ADB01122B397DDB01122B3979
:1035600041DC01122B3965DC01122B3987DC011299
:103570002B39E8DC01122B3933DF01122B390EE035
:1035800001122B39B8E001122B39F9E201122B3963
:1035900047E301122B398AE301122B39E2E30112CE
:1035A0002B3940E401122B396AE401122B398EE4E5
:1035B00001122B39BFE401122B39E9E401122B3936
:1035C00030E501122B398EE501122B39EAE50112A3
:1035D0002B39EBE601122B3955E801122B3993E810
:1035E00001122B39BCE801122B394DE901122B399C
:1035F00097E901122B39BBE901122B3911EA0112AB
:103600002B392CEA01122B39E7EA01122B3911EB85
:1036100001122B3954EB01122B39AAEB01122B3971
:10362000AFEE01122B39E2EE01122B399FEF01129E
:103630002B397AF001122B390AF101122B394BF197
:1036400001122B39DFBE05122B3917BF05122B399A
:1036500038BF05122B397ABF05122B39DEBF051290
:103660002B39E8BF05122B39F8BF05122B392FC0B3
:1036700005122B39D8C305122B39A0C505122B39D9
:1036800094C705122B3932C805122B39B9C8051257
:103690002B394D8004122B39F68004122B39D58139
:1036A00004122B39F08204122B39108304122B39A7
:1036B000328404122B39CF8504122B393C86041234
:1036C0002B39128704122B39188804122B397D8864
:1036D00004122B39B98804122B39128904122B39A0
:1036E0004B8904122B39948904122B39268A04122F
:1036F0002B39C38A04122B39988B04122B39658C11
:1037000004122B39F28C04122B39188D04122B3928
:10371000458D04122B39768D04122B394B8E0412F1
:103720002B395B8E04122B39AE8E04122B39BB8ED3
:1037300004122B39C88E04122B39D18E04122B3966
:10374000358F04122B39938F04122B39DE8F04121C
:103750002B39F98F04122B39209004122B393D900C
:1037600004122B39499004122B39ED9104122B3994
:10377000069204122B39829204122B39959204126C
:103780002B39A59204122B394B9304122B39BB947D
:1037900004122B39CE9504122B396E9604122B3954
:1037A000789604122B39E69604122B39F7960412F8
:1037B0002B39369704122B39649704122B39319820
:1037C00004122B39889804122B39CD9804122B3906
:1037D000239904122B39419904122B398F99041221
:1037E0002B395D9A04122B39AB9A04122B39ED9ABE
:1037F00004122B39709B04122B399A9B04122B391B
:10380000D09B04122B39DF9B04122B393D9C0412F0
:103810002B39B59C04122B39F69C04122B39459D8B
:1038200004122B39709D04122B398A9D04122B39F6
:10383000A49D04122B39799E04122B39839E041205
:103840002B39BE9E04122B39CE9E04122B39D79EE3
:1038500004122B39289F04122B393C9F04122B3958
:103860005AA004122B396DA004122B3984A0041223
:103870002B3999A004122B3933A104122B39B2A190
:1038800004122B3955A204122B3960A204122B39D1
:10389000ADA304122B39C9A304122B3921A404129D
:1038A0002B398FA404122B39DBA404122B39F5A475
:1038B00004122B3955A504122B39F3A504122B3908
:1038C0003EA604122B39A1A804122B3939A90412DF
:1038D0002B39B0A904122B39F6AB04122B390EACDC
:1038E00004122B3911AC04122B391DAC04122B39E4
:1038F00031AC04122B3939AC04122B3970AC0412E0
:103900002B3964AD04122B39EEAD04122B3970AE95
:1039100004122B39E5AE04122B39BDAF04122B393A
:10392000DFAF04122B3976B004122B3982B00412A7
:103930002B39DFB004122B39E2B004122B390FB14E
:1039400004122B3924B104122B3993B104122B39F0
:10395000DFB204122B39F2B304122B397DB40412F6
:103960002B3990B504122B395AB604122B398BB669
:1039700004122B39B1B604122B39BAB604122B3902
:10398000E9B604122B3999B704122B3949B804123D
:103990002B39BCB804122B396EB904122B39E1B99A
:1039A00004122B3920BA04122B3969BA04122B39AC
:1039B0009EBA04122B39D0B105122B393BB2051235
:1039C0002B3982B205122B39F8B205122B3948B3C4
:1039D00005122B39CCB305122B3910B605122B3931
:1039E0003BB805122B3918BC05122B3995BC0512B2
:1039F0002B39D0BC05122B39EEBC05122B394EBD2C
:103A000005122B3976BD05122B39A6BD05122B39AF
:103A1000D7BD05122B3904BE05122B395DBE051228
:103A20002B39A8BE05122B390CF201122B3988F262
:103A300001122B39AEF201122B39E5F201122B39AA
:103A40003EF401122B395AF401122B399FF4011262
:103A50002B392FF501122B3987F501122B395CF622
:103A600001122B393AF701122B3984F701122B3945
:103A7000E5F701122B3969F801122B3992F801127E
:103A80002B39D3F801122B3981FA01122B3951FB52
:103A900001122B3918FC01122B39EBFC01122B39C6
:103AA00025FD01122B397DFD01122B399FFD0112DD
:103AB0002B3933FE01122B39E6FE01122B397F8D93
:103AC00006122B39E48D06122B398B8E06122B39F8
:103AD000C38E06122B39C1A305122B396CA4051213
:103AE0002B3909A605122B3985A605122B39BDA63F
:103AF00005122B39A8A905122B393AAB05122B391F
:103B0000A4AB05122B39DCAE05122B397DB00512A2
:103B10002B39E6B906122B390EBA06122B39FABA2E
:103B200006122B396AE805122B39EDE805122B39FC
:103B300004E905122B3977E905122B39DDE9051265
:103B40002B3906EA05122B398BEA05122B392DEB9E
:103B500005122B3990EB05122B39F5EB05122B3999
:103B600015EC05122B3945EC05122B3961EC0512C9
:103B70002B3990EC05122B39C0EC05122B39F6ECE1
:103B800005122B3956ED05122B399BF304122B39F4
:103B90006BF404122B3990F404122B39B0F4041294
:103BA0002B39C4F404122B392CF504122B3950F59F
:103BB00004122B39CEF604122B39F4F704122B39E8
:103BC000D5F804122B3939F904122B3965F904128E
:103BD0002B39E9F904122B393AFA04122B395BFA22
:103BE00004122B39D3FA04122B39F8FA04122B39A8
:103BF0005BFB04122B39EBFC04122B39B8FD0412C9
:103C00002B39EFFD04122B3914FE04122B3934FE2C
:103C100004122B395AFE04122B396EFE04122B3972
:103C2000D7FE04122B392BFF04122B39B0AD06122C
:103C30002B39BAAD06122B39DBAD06122B392C9479
:103C400005122B39469705122B39739805122B391B
:103C50004E9A05122B39D89A05122B398C9B0512D6
:103C60002B39B59B05122B39EA9B05122B39989CF1
:103C700005122B39289D05122B399B9D05122B39D6
:103C80001D9E05122B39209E05122B39239E0512ED
:103C90002B39269E05122B39469E05122B39499E3B
:103CA00005122B39629E05122B39C69E05122B393F
:103CB000B89F05122B391DA702122B393AA1051204
:103CC0002B3941A205122B3913A305122B39F5D636
:103CD00003122B392DD703122B39EBDB03122B39AF
:103CE000BDDC03122B3944DD03122B3975DD0312C1
:103CF0002B39A3DD03122B39F7DD03122B3925DE17
:103D000003122B3946DF03122B3974DF03122B39D0
:103D1000A2DF03122B39D8DF03122B39A0AC021219
:103D20002B39ABE003122B390AE103122B3980E265
:103D300003122B391AE303122B390BE403122B392C
:103D4000E8E403122B3932E503122B3981E5031223
:103D50002B39EDE503122B3955E603122B39A2E678
:103D600003122B3912E703122B3923E803122B39E4
:103D700017E903122B39C8E903122B39FDE90312A5
:103D80002B3952EA03122B39F4EA03122B3922EBB6
:103D900003122B39A7EC03122B392CED03122B390C
:103DA0006CED03122B39ABED03122B39C4ED03126A
:103DB0002B3973EE03122B393DEF03122B39E4EF4D
:103DC00003122B3978F003122B391EF103122B3911
:103DD00088F103122B3913F203122B39A6F20312C6
:103DE0002B39C4F203122B3997F303122B3955F4F4
:103DF00003122B390BF503122B39A9F503122B39BA
:103E000073F902122B39B4F902122B391DFA02127E
:103E10002B393EFA02122B3957FA02122B3911FBB9
:103E200002122B391AFB02122B396BFB02122B39AF
:103E300094FB02122B39ABFB02122B390FFC02123E
:103E40002B39A1FC02122B39D2FC02122B392EFD88
:103E500002122B3994FD02122B39C8FD02122B39A4
:103E60003BFE02122B397DFE02122B39BDFE0212DF
:103E70002B39F5FE02122B3907FF02122B3919FFDD
:103E800002122B394AFF02122B398AFF02122B39F8
:103E9000B3FF02122B39B8F805122B39FBF90512C2
:103EA0002B3921FA05122B3932FA05122B394AFC2B
:103EB00005122B3969FC05122B39BDFD05122B3972
:103EC000F3FD05122B393EFE05122B398AFF051230
:103ED0002B39008005122B393E8105122B397A814E
:103EE00005122B393F8305122B39698305122B39B3
:103EF000EF8505122B392F8605122B39C487051241
:103F00002B39598805122B39B78805122B39488966
:103F100005122B39808905122B39C28905122B39DC
:103F20003C8B05122B39C58C05122B39FB8E0512E3
:103F30002B39298F05122B39558F05122B395E8F9E
:103F400005122B39B48F05122B39449005122B39E9
:103F50004B9305122B39CF9305122B3981C30612CF
:103F60002B3997C306122B39A1C306122B39F1C383
:103F700006122B39038506122B391C8506122B39A4
:103F8000C18506122B39018606122B391A860612B4
:103F90002B394E8606122B399B8606122B39CF867B
:103FA00006122B39118706122B39E78806122B3996
:103FB000528906122B3963BC06122B39B8BC061283
:103FC0002B3911BD06122B39E3C206122B3925C33A
:103FD00006122B3967C306122B3977C306122B3909
:103FE00006BB04122B3961BB04122B3901BC04122D
:103FF0002B3919BD04122B3905BE04122B39D2BE40
:1040000004122B39E7BE04122B3931BF04122B39AD
:1040100088BF04122B39F4BF04122B3907C00412D5
:104020002B395FC004122B39CEC004122B39E6C0E5
:1040300004122B397DC304122B3979C404122B3995
:10404000D4C404122B3928C504122B3944C70412D6
:104050002B3994C704122B3915C804122B39E7C821
:1040600004122B3920C904122B393FC904122B39F1
:104070008AC904122B39A0C904122B39B7C90412FA
:104080002B39E6C904122B39F8C904122B39E7CAB7
:1040900004122B39F2CA04122B3977CB04122B39B4
:1040A000CFCB04122B391BCC04122B3952CD041266
:1040B0002B3983CD04122B39FFCF04122B3930D08A
:1040C00004122B394BD104122B397AD104122B391B
:1040D000F2D104122B39B4D204122B39E8D20412D3
:1040E0002B3958D304122B3935D404122B396ED402
:1040F00004122B3978D404122B397BD404122B39B7
:1041000085D404122B39A1D404122B391DD50412E5
:104110002B3956D504122B3972D504122B399ED562
:1041200004122B39D9D504122B39F4D504122B39AA
:10413000FED504122B392DD604122B3943D6041286
:104140002B395FD604122B398ED604122B39AED6FA
:1041500004122B39F7D604122B3940D704122B390D
:104160004AD804122B399CBF06122B39ADBF061258
:104170002B3936C006122B3942E105122B3991E159
:1041800005122B394FE305122B3922E505122B3985
:1041900060E505122B3936E605122B393BE705128F
:1041A0002B395DE705122B39B9E705122B393AE8AF
:1041B00005122B39885200122B39AA5200122B39C2
:1041C000FC5300122B39455400122B39BE540012F7
:1041D0002B39395500122B39A25500122B39E955CC
:1041E00000122B39575600122B39FC5600122B396E
:1041F000825700122B39BE5700122B39125C001265
:104200002B39205E00122B39535E00122B39925E3F
:1042100000122B399F5F00122B39886200122B3954
:10422000326300122B39DD6400122B391066001244
:104230002B39266700122B399B6700122B396768D0
:1042400000122B39FE6800122B390E6900122B392F
:10425000C56900122B39FB6A00122B393F6D001221
:104260002B39E26F00122B39C07000122B39FD710F
:1042700000122B39427500122B39527500122B395E
:10428000897600122B393C7700122B396D78001299
:104290002B39DB7800122B39127A00122B39677A0E
:1042A00000122B3995D904122B393CDA04122B3920
:1042B000AEDA04122B39BEDA04122B3940DB0412B9
:1042C0002B3997DB04122B398CDC04122B39B3DC2D
:1042D00004122B3958DD04122B39A7DD04122B39B7
:1042E00005DE04122B3960DE04122B393BE1041287
:1042F0002B39F4E104122B3959E204122B39ECE387
:1043000004122B398CE404122B3925E504122B39C5
:1043100082E504122B39F8E504122B39F4E6041275
:104320002B39E7E704122B3940E804122B3956E801
:1043300004122B3977E804122B39B6E804122B3912
:1043400046E904122B3989EA04122B3946EC04128F
:104350002B3990ED04122B39CAEE04122B39D5EF0C
:1043600004122B3975F004122B39E4F004122B39A6
:1043700001F204122B3986D802122B39EFD802121F
:104380002B3937D902122B397BD902122B39EED9AE
:1043900002122B3948DA02122B3983DA02122B3936
:1043A0001DDB02122B3977DB02122B39E3DC021200
:1043B0002B395CDD02122B3986DD02122B399ADE95
:1043C00002122B39A8DF02122B39D0DF02122B394F
:1043D000CEE002122B39DFE002122B39F5E0021297
:1043E0002B39F6E102122B3919E202122B39E6E2DF
:1043F00002122B390EE302122B3925E302122B395C
:104400004BE302122B3986E302122B39A6E3021288
:104410002B39CDE302122B39E5E302122B39C2E42A
:1044200002122B3925E502122B39A8E602122B398C
:1044300037E702122B395BE702122B3972E70212BF
:104440002B3946E802122B39E2E802122B3908E92F
:1044500002122B395DEA02122B397BEA02122B3948
:10446000F6EA02122B392CEB02122B3969EB0212FD
:104470002B39F5EB02122B3961EC02122B3945ED89
:1044800002122B3923EF02122B39F8EF02122B39CB
:1044900044F002122B397CF102122B39C9F20212BC
:1044A0002B393FF402122B394DF402122B3947F508
:1044B00002122B39EEF502122B3937F602122B3984
:1044C0004CF602122B395BF702122B3974F80212E8
:1044D0002B39D2F802122B3992F305122B39CFF374
:1044E00005122B3968F405122B3973F505122B3997
:1044F000BBF705122B3937F805122B390C99061228
:104500002B393A9A06122B39029B06122B39579BEC
:1045100006122B39DA9B06122B3989B206122B3977
:1045200078C106122B3989C106122B3929C206120D
:104530002B39DDFF02122B39EEFF01122B398FC010
:1045400006122B399FC006122B39B7C006122B3921
:104550006BC106122B3998BE06122B391DBF0612ED
:104560002B3983BF06122B393FFF04122B3942FF30
:1045700004122B397BFF04122B39CEFF04122B3986
:10458000E0FF04122B39E3FF04122B397D91061250
:104590002B398B9106122B39049206122B39D992A2
:1045A00006122B39989406122B39FD9406122B39DA
:1045B000609506122B39F87F00122B39FDAF0612D9
:1045C0002B3935B006122B3986B106122B390AB2B7
:1045D00006122B3903AB06122B39A4AB06122B396A
:1045E000D5AB06122B3920AC06122B39E4AC0612DF
:1045F0002B3917AD06122B393DAD06122B394FADB5
:1046000006122B3963AD06122B3971AD06122B3908
:104610000AEE05122B3936EE05122B39DDF00512A4
:104620002B3932F105122B396EF105122B3982F13B
:1046300005122B399BF105122B398EF205122B39FD
:104640006AF305122B397EF305122B3916B70612C1
:104650002B393AB706122B3953B706122B3992B7BA
:1046600006122B39C5B706122B39F5B706122B39AE
:10467000FFB706122B3967B806122B396AB8061233
:104680002B3974B806122B3981B806122B395DA864
:1046900006122B3985A806122B39C6A806122B390B
:1046A000E4A806122B39FFA806122B3967A90612B7
:1046B0002B3973A906122B39D2A906122B39F6A968
:1046C00006122B39B7AA06122B39C4AA06122B39A7
:1046D000D5AA06122B399FC406122B39B7C406126D
:1046E0002B39DDC406122B39448006122B398D81FB
:1046F00006122B39938106122B39AA8106122B3907
:10470000CB8106122B39E18106122B39F581061275
:104710002B39748206122B39D98206122B39618308
:1047200006122B39DA8306122B39B38406122B3981
:10473000C38406122B39D28406122B394AC20612C0
:104740002B396EC206122B3996C206122B39BEC205
:1047500006122B399EA506122B390AA606122B39F2
:1047600029A606122B398FA606122B39D5A20612BE
:104770002B39EEA206122B3905A306122B390EA3F4
:1047800006122B392CA306122B3936A306122B390D
:1047900040A306122B3953A306122B39E0A30612AD
:1047A0002B394FA406122B397DA406122B39CEA427
:1047B00006122B391AA506122B3935A506122B39EC
:1047C0003FA506122B3950A506122B3993A50612C8
:1047D0002B3926C506122B3971C506122B396EF6F8
:1047E00003122B399AF603122B39B8F603122B3920
:1047F000CBF603122B39E6F603122B3945F70312D9
:104800002B3973F703122B397FFB03122B39C1FCB1
:1048100003122B39F3FC03122B395EFD03122B39E3
:10482000E2FE03122B390AFF03122B391FFF03127A
:104830002B392FFF03122B396FFF03122B39B1FFD6
:1048400003122B39C1FF03122B392BBB06122B3954
:104850003BBB06122B3959BB06122B3974BB06120F
:104860002B399BBB06122B39BCBB06122B39D6BB8E
:1048700006122B390EBC06122B3931BC06122B390D
:104880003AFF01122B3980FF01122B397495061261
:104890002B39849506122B39A29606122B39D49601
:1048A00006122B39F69606122B391E9706122B3953
:1048B000379706122B39739706122B39DC9706129D
:1048C0002B39189806122B395F9806122B398C98C1
:1048D00006122B39B89806122B3987B506122B39D8
:1048E000BEB506122B39E6B606122B39E9B606120A
:1048F0002B3985BD06122B39F7BD06122B3935BE73
:1049000006122B3976BE06122B39E2D105122B394D
:10491000E8D105122B392FD205122B393BD40512C1
:104920002B396BD405122B39D5D405122B3990D5E0
:1049300005122B39D7D505122B390AD605122B397A
:1049400094D605122B39ABD605122B39B8D60512E1
:104950002B39C2D605122B3962D805122B3954D9FE
:1049600005122B39B2D905122B3965C905122B391D
:104970007BC905122B392DCA05122B3957CB0512CD
:104980002B394CCC05122B39E3CC05122B391ECD1B
:1049900005122B3990CD05122B39EECD05122B398E
:1049A000FECD05122B3925CE05122B3977CE0512F7
:1049B0002B39E6CF05122B39EBCF05122B390DD051
:1049C00005122B391FC406122B394DC406122B3980
:1049D00082C406122B3984C406122B3986C40612EF
:1049E0002B3997C406122B3999C406122B399CC453
:1049F00006122B39FEB306122B396CB406122B3972
:104A00008EB406122B39C6B406122B39FCB406122A
:104A10002B39AC9F06122B39EF9F06122B390DA0B4
:104A200006122B3940A206122B3974A206122B391A
:104A30009FA206122B397DC506122B39EBD9051220
:104A40002B39CEDA05122B39B6DB05122B39C7DB31
:104A500005122B39D8DB05122B3924DC05122B3932
:104A600013DE05122B396EDF05122B399EDF05127E
:104A70002B3969E005122B39C6E005122B395F8905
:104A800006122B397D8906122B39C18906122B3962
:104A9000E78906122B39098A06122B39218A061258
:104AA0002B39398A06122B39518A06122B39F78A8B
:104AB00006122B39398B06122B39438B06122B39F0
:104AC000588B06122B395F8C06122B397A8C061202
:104AD0002B39838C06122B398C8C06122B39958C32
:104AE00006122B399F8C06122B391C8D06122B397E
:104AF000237B00122B39687F00122B39847F001230
:104B00002B39897F00122B396C9C06122B39829C21
:104B100006122B39039E06122B392D9E06122B39B5
:104B2000749E06122B397D9F06122B398BB8061204
:104B30002B39EBC506122B3910C606122B39BEA62F
:104B400002122B392FA502122B39BDA402122B39C8
:104B500089A402122B395EA402122B393AA4021244
:104B60002B395DA302122B3927A302122B39E7A29E
:104B700002122B39B5A202122B3926A202122B39AE
:104B8000D8A002122B395EA002122B399B9F021271
:104B90002B39919E02122B39489E02122B39229EEC
:104BA00002122B395E9D02122B39A89B02122B395F
:104BB000489B02122B39199B02122B39169B0212A9
:104BC0002B39DC9902122B39C89802122B3988979D
:104BD00002122B39BA9602122B398CAC02122B39E5
:104BE00078AC02122B3964AC02122B3950AC021291
:104BF0002B39BCAB02122B39D4AA02122B394CAA86
:104C000002122B39329602122B39529502122B398D
:104C1000B99402122B39139402122B3999A902125A
:104C20002B39D59302122B393B9302122B39FA926E
:104C300002122B399D9202122B3985E003122B3977
:104C40006A9202122B3948A702122B39FE910212E6
:104C50002B39CB9102122B39709102122B393F91D3
:104C600002122B39088E02122B391A8D02122B399F
:104C7000D48B02122B39808B02122B39748B0212C7
:104C80002B39DB8A02122B39A98902122B39FA86B9
:104C900002122B399D8402122B39518402122B39B6
:104CA000368302122B39CB8202122B39F381021286
:104CB0002B39008002122B39AF8102122B396B8005
:104CC00002122B39328002122B39EDA005000000B0
:104CD00080FB8F0001009B09870001009A092400D6
:104CE00002001711250002001911260002001B11F5
:104CF000270002001D11280001001F1129000100DA
:104D000020118400040021118600010025112A00D1
:104D1000010026112B00010027112C0001002B118E
:104D20002D00080082092E0001002C112F00010027
:104D30002D11300001002E11310001002F11320021
:104D400001008A09330001008B0934000100301191
:104D5000360001008C0938000100311139000100D2
:104D60002A118300020043116300010097096400C7
:104D7000010028116500010029116D00010098094A
:104D8000710008007A096600010042114300010029
:104D90003311440002003411450001003611460071
:104DA00002003711470008008F094800010039113F
:104DB0004B0001003A11040001004511A10001005F
:104DC0004711370001004611880001009C093C0092
:104DD00001008D093D0001003211490002003B1124
:104DE0006700010099094D0002003D114E000100CD
:104DF0003F114F00020040113E0001008E090000EB
:104E0000000000000001363601010001020100012E
:104E10000301000104010606050200000701003439
:104E20000801000F090401010D0100FF0E08000038
:104E300017020000190100FF1A0100011B0100FE0A
:104E40001C0100081D0200001F01000120010001DB
:104E5000210200002301000F2402000026010001AE
:104E600027010008280200FF2A0100072B01024049
:104E70002C0100002D0100012E0100012F0100FF77
:104E800030010B1C310800003A0100083B01000F03
:104E90003C0100013D0100FF3E040000420400000F
:104EA000460400004A0400004E04000052040000C2
:104EB000560400005A0400005E20FFFF3600010087
:104EC000060000000F0000000000000000000000CD
:104ED000000003FFFF00000403FFFF0000FFFF0FBF
:104EE000F4010005C4040320000100000B000000D1
:104EF000000000000003010F00000000000000009F
:104F000000000000000000000000000000000000A1
:104F10000000000000000000000000000000000091
:104F20000000000000000000000000000000000081
:104F300000000000000000000000010371030103F5
:104F40000103010301030103220302030103100310
:104F500000030003000300030003000300034203F7
:104F600000032403060300030003040312032503C4
:104F700023032503230304030403000300030003A6
:104F800044030003000323030003650321003503EA
:104F9000810300030503000300030003000325034E
:104FA0002303030071003001600011007000310222
:104FB0002003500480001000610000001400630012
:104FC000730072006200430000001300060000003E
:104FD00000000400120000000000000000000400B7
:104FE0000400370037003C024400000000000000CD
:104FF0000000650000003500810000000500000091
:105000008300000001017101010101011101010191
:105010003101010101018001100161013B00140017
:105020006301730172016201430100011301060172
:105030003D013500040112010001000100010001E1
:1050400004010401330133013C0144013201360003
:105050000001000165010001350081010001050129
:10506000820183010001030271023001600211021A
:1050700070020102020202028002100261023A0082
:1050800041006302730272026202430200021302D1
:1050900038000002000204021202000200020002B4
:1050A000000204020402370037003C0244020002FE
:1050B000390000020002650200023502810200028E
:1050C00005028202830200020304710402046004E8
:1050D00011047004020402040104020410046104B7
:1050E000000414046304730472046204430400049F
:1050F0001304060400040004040412040004000461
:10510000000400045104640000040004000444048A
:105110000004000400040004650400043504810454
:10512000640005040004830400040000E34213004B
:1051300053420100E3420200D5410300DB41040079
:10514000E1410500E7410600F3413000174231001C
:105150001142320023423300294235002F423400ED
:10516000354236003B421100474214004D421500C3
:1051700005421F000B42FFFF0000011733064D33AD
:105180000847330B65331081320A7733021D33052C
:105190003B330723330CFF320D0B33648330FF00A6
:1051A0000007ECFDFDFDECDCDCCCBCACAC9C9C8CCD
:1051B0007C7C6C6C5C5C5C4C4C3C3C2C2C1C1C0368
:1051C000EAF5E5D5D5C5B5A595958585757565656A
:1051D000555545453535252515150500160F000093
:1051E0000B150B020002220F3300000E010305070E
:1051F000090B0D0F00020406080A0C0D5A696742DC
:105200006565416C6C69616E6365303930301718C3
:105210001921301B1D1F30303016181920231A1C7D
:105220001E3000034A49434E181A25050200011991
:1052300016181616182303000C0E020B040B0A078F
:1052400008000F00393D3F373C3C362C442D02040A
:1052500002010101010902E803000000BE040A7F07
:10526000003C00000000000E00E8033C0008100CA9
:105270000A0C03150900040009FF1E1E0305010C9A
:105280000504040810080328C082C08390081DE4A8
:10529000F0A3F07CD57D047A8E7B07124901123091
:1052A00089124CAF12308F02706374F3122584742C
:1052B000F5122C1889098A088B0AE9705F74026557
:1052C00008703E9007AD7408F0750C00780C122B36
:1052D0005AECF50C780C122B5AEBF50C780C122BBF
:1052E0005A90112112298D901125E0F97C8F7D09AA
:1052F0009011431270741230B37407122B8402534E
:10530000BC7401650860030253BF9007AD7408F0D8
:105310007B00AA0AA90A1230F50253BC7401650980
:1053200060097402650960030253BFEA60067403F2
:10533000650870409007AD74021253E0122DFE1202
:1053400030A19007B5E0A2E34010E9700D9008216C
:10535000E004F0640470031253EA74036508705C9F
:10536000900822E0F8740128F0E8C39405404D123B
:1053700053EA804874016508704574016509900717
:10538000AD702E740AF07401122E2DE4F074021226
:105390002E2D7403F004122E2DE4F0A3F0A3F0A33D
:1053A000F07408122E2DE4F0AA18AB1912332980DC
:1053B00025740A1253E0122DFE1230D7E9601790BF
:1053C000810012298D7A017B009007AAE0F9123F33
:1053D000897404122B84740B122B847F0502280914
:1053E000F0901125E0F990112122901121E4F0A311
:1053F00074F8F0A374FFF0A37407F02274F612257A
:1054000084E9FFEAFE7AD1F9123E3F8A828B83E576
:10541000824583702A7A027B00123E21EA4B700E8D
:105420007A107B009007AAE0F9123E6380148A820A
:105430008B8374D1F0EFA3F0EEF9123E2D8003EFD1
:10544000A3F002565274F7122584890890070712B8
:105450007730FF901112E0F47003A3E0F4703690FF
:10546000071EE0901112F0A3E4F080298E828F8352
:10547000A3A3127B1E60168E828F83A3A3A3E0F5E5
:10548000838882A3127B1EFAA9081241BD8E828FE7
:1054900083127A46FFEE4F70D3901112E0F470033E
:1054A000A3E0F4600A901112E0FAA9081241BD12BB
:1054B0003431900778125BC312342B02786874F190
:1054C000122584890A8C08750900750B00740F1267
:1054D0002E2D12631C7411122E2D125BEA8049AE20
:1054E0000E12558AF50CA3E0F50DAE0BEE2EFEE480
:1054F00033FFEA2EF582EB1268D5650C7004A3E049
:10550000650D7019AE09EE2EFEE433FFEC2EF58228
:10551000ED3FF583E50CF0A3E50DF00509050EE57B
:105520000EC3950840B9050BE50BC3950A500575E8
:105530000E0080EBA909026F8074F4122584890B98
:105540007D00740C122E2D12631C80010DEDC3958D
:105550000B5032750A008002050AE50AC39C50EC24
:10556000ED25E0FEE433FFEA2EF582EB3F12559A7B
:10557000F509AE0A12558A65087004A3E065097042
:10558000D7790180027900026D27EE2EFEE433FF09
:10559000E82EF582E93FF583E022F583E0F508A3E4
:1055A000E02274F612258412563D7003A3E06D705C
:1055B000177508B37509077808122B56EEFA1242D0
:1055C000E97402122B84801F75080275098078081F
:1055D000122B568C088D097808122B561256301251
:1055E000430D7404122B84806974F61225841256BC
:1055F0003D7003A3E06D70177508C0750907780842
:10560000122B56EEFA1242EF7402122B84801F7591
:1056100008037509807808122B568C088D097808C4
:10562000122B5612563012430D7404122B84802212
:10563000125F8BF583E0FD7C801269A9221268DE7F
:10564000127A58FCE439FD900778E06C227402125B
:105650002B847F0202280974F612258474FE122C12
:1056600018EAFEEBFF851882851983E4F0A3125E29
:105670001A1268F5E0FCA3E0FBECFA88828983A3A8
:10568000A3E0F9750900750800600574FF697005ED
:10569000750882803D900778E06A7003A3E06B7024
:1056A0001AAA18AB191239F5E9F509851882851976
:1056B00083126D32701C750883801790099AE06020
:1056C00004640170057508818008E0640270037548
:1056D0000880851882851983125BEAA908EEFAEF23
:1056E000FB1242F5E5096011851882851983126D58
:1056F00032600612706E123EC902564D74F21225C7
:1057000084EAFEEBFF750A00750B0012576E123427
:1057100031EA65087003EB65097012123A07E91463
:10572000F50A79017AE97B07123A0D8003750B803F
:105730001268CFF50C780C122B5A750CE9750D0711
:10574000780C122B56780A122B5A7808122B56E531
:105750000BF5087808122B5A1267901268D2F97A62
:10576000057B801242FB7407122B840264D81279E5
:105770009112632088828983127A57F508E439F5FB
:10578000092274F6122584E9FE7F0080298A828B23
:105790008312559CF8E4C8F9E50828E439F509EFC7
:1057A00025E0F8E433F9EC28F582ED125F94EA2461
:1057B00002FA50010B0FEFC39E40D202565274E81A
:1057C00012258474FB122C188A168B178518828573
:1057D0001983E4F07403122E2DE4F0A3F004122ECA
:1057E0002DE4F0A3F012630D3517125DECF50B8577
:1057F0000A82F583127A53FEE439FF850A82850B0B
:1058000083A3A3E0FA850A82850B83A3A3A3E0F90F
:10581000EAF508E439F509E50A2404F50A50020519
:105820000BEEFAEFFB1234CDE964016016EEFAEFED
:10583000FB1234CDE9703D900778E06E7003A3E071
:105840006F6031126AEC122B5AE4F508F5097808FA
:10585000122B567808122B5A900778122995750842
:10586000807808122B5A125BC91242FB7407122B64
:1058700084025BB9125BF08810602B12766D123EC9
:10588000C37403122E2D125BC37403122E2D126DDE
:105890003260137403122E2D125BE2A9101241ED37
:1058A0008A0A8B0B8003751000125BF0880F60274B
:1058B00012766D123EC37401122E2D125BC3740159
:1058C000122E2D126D32600F7401122E2D125BE21A
:1058D000A90F1241ED8003750F00900707805D85C9
:1058E0000A82850B83A3A3A3A3A3A3A3A3E4F0A38A
:1058F000F0AA0AAB0B851482851583A3A3125C0062
:10590000127B1EF9123E2D851282851383E0C0E0C2
:10591000851882851983E0F874E928F582E4340754
:10592000F583D0E0126D3604F0E511A2E05007AA2D
:1059300012AB13123EC9851482851583E0F514A3BA
:10594000E0F515E51445157003025B268514828584
:105950001583A3A3127B1E60DD851482851583A3A6
:10596000A3A3A3A3A3A3A3E0A2E050CA85148285A6
:105970001583A3A3A3A3126D32851482851583A377
:10598000A3601F127B1EFA7901851482851583A3FB
:10599000A3A3A3126FA912276A8A128B1375110190
:1059A000800F125C00A3A3E0F512A3E0F5137511BC
:1059B00000E512451370030259298512828513836D
:1059C000A3E065087004A3E06509600F74FF650833
:1059D000700474FF650960030259298512828513DA
:1059E00083A3A3A3A3A3A3A312299585128285133E
:1059F00083A3A3A3A3A3A3E0FC7405122E2D12700E
:105A000074A9101241CF7402122B84E9703C8512E4
:105A100082851383A3A3A3A3A3A3A3A3A3A3122950
:105A200095851282851383A3A3A3A3A3A3A3A3A3F2
:105A3000E0FC7403122E2D127074A90F1241CF7462
:105A400002122B84E97003025929E50F2510C33394
:105A5000240AFA7B00123E218A0A8B0BEA450B705E
:105A6000030259078A828B8374D2F08516828517C8
:105A700083A3A312631C8A828B83A3A3E8F0A3E908
:105A800012794EA3E510127A5FE50FF0E510603C45
:105A9000EA2405FAE4350BFBE50A240AF8E4350BA1
:105AA000F98A828B831263267403122E2D125C05F1
:105AB000122B52AC10EC2CFCE433FD8A828B831247
:105AC0007074123DFD7403122B84800D8A828B83C7
:105AD000A3A3A3A3A3E4F0A3F0E50F70030258DF90
:105AE000A810E828F8E433F9E50A28F8E50B39F9B5
:105AF000E8240AFAE439FB850A82850B83A3A3A371
:105B0000A3A3A3A3A3125BC37401122E2D125C05E1
:105B1000122B52AC0FEC2CFCE433FD123DFD740350
:105B2000122B840258F1851882851983E0602712B0
:105B30006AEC122B5A7508E97509077808122B567A
:105B40007403122E2D126AF5122B5A90077812291F
:105B5000957508008029EEFAEFFB1234CDE9702F1D
:105B6000126AEC122B5A7508E97509077808122B8E
:105B7000567508007808122B5A90077812299578E4
:105B800008122B5A125BC91242FB7407122B847441
:105B900003122E2D126D32600B7403122E2D127013
:105BA00074123EC97401122E2D126D32600B7401F5
:105BB000122E2D127074123EC97405122B847F10A0
:105BC000022809EAF0A3EBF022E5162402FCE435F2
:105BD00017FDE5161267203517F583E0F97A067B85
:105BE0008022125BEAAA0AAB0B22E0FCA3E0FD22B2
:105BF000850A82850B83E0F8A385820A85830B22C0
:105C0000126FA9A322E0F50CA3E0F50D750E007844
:105C10000C2274F112258474F4122C188A088B0952
:105C2000ECFEEDFF740B122E2D7403F0122BF2120A
:105C3000490112342BEAFCEBFD7403122BF21248DB
:105C4000FBE9600FEE24131268D264036010E06475
:105C500001600B8518828519837484025DA48E828D
:105C60008F83A3A3A3A3A3A3A3A3E06018F4601549
:105C7000EE24131268D264037016EE24141268D254
:105C80006003F4700B8518828519837482025DA409
:105C900012781CE064217002A3E06003025D7B8542
:105CA0001882851983748C125E1A64036003025D86
:105CB000657401122BFA1264C0124C2BE9600302C6
:105CC0005D651241518A0A8B0BEA450B7003025D38
:105CD000A58E0C8F0D750E00780C122B527C157D45
:105CE00000123DFD7403122B84850882850983A36D
:105CF000A3E50A2415FCE4350BFD7409122AB2123F
:105D0000747BC0E0E50A241EF582E4350BF583D0F0
:105D1000E012632CC0E0E50A241FF582E4350BF5A0
:105D200083D0E0F0E50A2420F582E4350BF5837496
:105D300005F0EE240BFE50010FFAEFFB123AAF7D97
:105D4000007C007900EEFAEFFB1242B39081001262
:105D5000298D7A007B109007AAE0F9123F8974041C
:105D6000122B848078125DE2122B5A125DF4124CD1
:105D7000557401122B84E9702C8014125DE2122BF1
:105D80005A125DF4124C4F7401122B84E9700D8588
:105D90001882851983E4F0124121800985188285D3
:105DA00019837488F012747BF50A780A122B5A74DE
:105DB00001122BEA880A890B780A122B56E508246F
:105DC0000CF582E43509125DEC4480F50B780A127B
:105DD0002B561268521242A77405122B84740C02BF
:105DE0006F7DEE1264CDE0F50A780A22F583E0F5C6
:105DF0000AA3E022EE240BFCE43FFD8E828F83A3F6
:105E0000A3A3A3A3A3A3A3A31270B18E828F83A382
:105E1000A3A3A3A3A3A3A3E0F922F0127991E02204
:105E2000C082C08374F3122C18851882851983E40C
:105E3000F004122E2D125BC37403122E2DAA82AB16
:105E400083122FABAA18AB19122FE7740D122B84F3
:105E500002706374F61225841268DAFAA3E0F9EA94
:105E6000F89007BBE058F508A3E059F509E50845A7
:105E700009601C7808122B56900778122995126831
:105E8000CFFD7C001269A51243077404122B840213
:105E9000565274F412258474FF122C18EAFEEBFF9C
:105EA000851882851983E4F090098EE06021EE2444
:105EB0000B1268D2640160178E828F83A3A31263D2
:105EC0001CEE24151268D2687003A3E06960030217
:105ED0005F8612678012631AE8FAE9FB8882898379
:105EE000A3A3A3A3A3A3A3A3E0FC88828983A3A362
:105EF000A3A3A3A3A3A31279F8EC28F508E439F52A
:105F000009EC45096010EC9471E994085008900977
:105F10009AE06402700A851882851983748080383B
:105F20001230238A0A8B0BA80AA90BE84960218842
:105F3000828983A3A3A3A3E06016C394035011E84E
:105F40002412125F91E82414125F911241218009FA
:105F50008518828519837481F0125F8B126AF3129F
:105F60002B5A7401122BEA880889097808122B56DB
:105F700075081F7509807808122B56126786124221
:105F8000A77405122B847401026D24EE1278433F2E
:105F900022F582E439F583E508F0A3E509F02274DF
:105FA000EA12258474DB122C188A148B15751200E2
:105FB000751300127B16F50EAC18AD197A007B0034
:105FC000799C1231077A047900122FF9EAF50C85D1
:105FD0001882851983E02AF0F8E50EC39840030281
:105FE00061BEE0C3950EF509C3940440037509032F
:105FF000E50975F01AA4FAABF0123EC38A128B13AE
:10600000EA451370030261C1750D00AE12AF13852E
:106010000E08807E126229123E09850A82850B8352
:10602000A3A3A3A3E0702D850A82850B83126D3292
:10603000700C1271BEF0EE24181271C18010126241
:1060400037F0900567E014C0E0126211D0E01262F0
:1060500062E48034900567E004C0E0126211D0E091
:1060600012625AC39403EE40030261251264C9749C
:106070000212625A64017003026132EE2415126248
:106080003AF0EE241612623AF0EE241AFE50010F96
:10609000050DE50DC39509400302615DE508C39553
:1060A0000C400302613B85080AAA0A7B0012306B90
:1060B0008A0A8B0B05089005541262431249018528
:1060C0000A82850B8312631C12621FE8F0A3E91297
:1060D0006274850A82850B83A3A3A3A3A3A3A3A3AE
:1060E000A3A3E0C0E0126207D0E0F07401122E2DED
:1060F000E4F0850A82850B8312631C7402122E2D34
:106100001263267401122BF2122FD5E96401600389
:106110000260147404122E2DAC82AD8312622F1211
:10612000490102601A12623812625A640360030263
:10613000607BEE24151271C1026081E50CC3950EDF
:106140004005750800801DE50EC3950CF508801408
:10615000126237F0EE241AFE50010F050DE50DC353
:106160009509505D740E122BFA85080AAA0A7B0065
:10617000798712310705087418122E2D1262431206
:106180004901126229123E09EE2412F8E43FF97423
:106190000E122E2D12707488828983EAF0A3EB12FE
:1061A00062627403126274741D122E2DE0C0E0123C
:1061B0006207D0E0126FDB70971271BE809575098F
:1061C00000750A00780A122B5A7812122B56780999
:1061D000122B5AE50EF5097809122B5A7405122E66
:1061E0002DE0FD7C0012670C1243437405122B84D2
:1061F000E51245136007AA12AB13123EC9742512AB
:106200002B847F0E022809EE2419F582E43FF583E2
:106210002212621522EE2418F582E43FF58322EE65
:106220002412F582E43FF583227C087D0079FFEE9D
:10623000240AFAE43FFB22EE2414F582E43FF583BE
:106240007401221263208E828F83E8F0A3E9F07C30
:10625000687D05EE1269C03FFB221279B3A3A3A3A8
:10626000E022F0EE1271B57402F0EE2416F582E42D
:106270003FF58322F0EE2417F582E43FF5837402A4
:10628000F012621574FFF02274F612258474F9126C
:106290002C188A088B0912630D3509127AE0123E18
:1062A00015EAF8EBF9ECFAEDFB85188285198312F3
:1062B0002E16EE2404FE50010F8E828F83E0C0E084
:1062C0007404122E2DD0E0126FB2FA7405122E2D26
:1062D0007401F07406122E2D7401F0900782F09074
:1062E000078B041279CAA312631C900783126326DA
:1062F000EA90078C12632C900781F0AA18AB191250
:1063000030A7E960031230AD740702564FEA1263FA
:1063100012221268EF2212771939F58312632022B4
:10632000E0F8A3E0F922E8F0A3E9F022F0127928DE
:10633000E02274F212258474FF122C187508007E76
:10634000007F001233598A0A8B0B1233598A0C8B47
:106350000DA80CA90D80050508126316E84970F711
:1063600090099AE060076401600302643D123359AA
:106370008A0C8B0DA80CA90D8003126316E84960E6
:106380003688828983127074900554E06A7003A382
:10639000E06B600D12771939F583127074EA4B7057
:1063A000D98882898312631C900554E0687003A326
:1063B000E069700302643D7A167B00123EC38A0CCA
:1063C0008B0DAE0CAF0DEE4F607390055412631C35
:1063D0008E828F83126326900549E08E828F83A37D
:1063E000A3F01234B5E98E828F83A3A3A3A3A3F0F5
:1063F0009011261279A7F07C687D051264C01249BD
:1064000001AA18AB197941124A8785188285198328
:10641000E0600890077812631C800478FE79FF8E94
:10642000828F83A3A3A3A3A3A3A31263261264C88A
:10643000E50AF0A3E50BF08E0A8F0B050890078C98
:10644000E0F8E508C39850047A008022E508C39874
:10645000FAC3940640027A057900800DE50A1277A6
:106460001A350B125DECF50B09E9C39840EE75097E
:10647000007809122B5A780A122B56EAF509780986
:10648000122B5A90078CE0F5097809122B5AAD08A7
:106490007C007A837B07900781E0F912433D740505
:1064A000122B8490099AE060046401700BEE4F6037
:1064B00007EEFAEFFB123EC91230AD7401025768C5
:1064C000EE240BFAE43FFB22EE1264CD2212771A7F
:1064D0003FF58322EEFAEFFB7F0602280974EC12E7
:1064E000258474FF122C188A0A8B0B7E008E0E8E68
:1064F0000F12630D350B127B1CFFAC18AD197A001F
:106500007B00799D123107851882851983E0F8EFA9
:10651000C39840030265B8E0C39FFEC3940B4002DA
:106520007E0AEE75F007A4FAABF0123EC38A088B20
:10653000098A0E8B0FEA450F607C750C00801A8566
:106540000882850983A3A3A3A3A37403F0E5082409
:1065500007F50850020509050CE50CC39E5059AC1F
:1065600008AD09850C10E5102FFAE43400FB798B97
:10657000123107850882850983A3A3A3A3A3E0148E
:10658000600814601314601F80B585088285098334
:10659000A3A3A3A3A3E480B4850882850983A3A34E
:1065A000A3A3A3740180A5850882850983A3A3A35F
:1065B000A3A3740280967E007508007808122B5AF7
:1065C000780E122B56EEF5087808122B5AEFF508C4
:1065D0007808122B5A7405122E2DE0FD7C00E50A76
:1065E0001269C0350BFBE50A126720350BF583E015
:1065F000F91243497405122B84E50E450F6007AA72
:106600000EAB0F123EC97401122B847F0C022809B5
:1066100074EA12258474FE122C188A148B15750ADC
:1066200000750B00127B16F508AC18AD197A007BCB
:106630000079A3124C4985080C85188285198312AC
:10664000631CC3E50C98E499507D851882851983F5
:10665000E0C3950CFEA3E09400FFC3EE9404EF9416
:106660000040067E037F008004EE4F605AEEFAEF92
:10667000FBEA75F015A4FAA8F075F015EBA428FB59
:10668000123EC38A0C8B0D8A0A8B0BEA450B6037CE
:10669000750900750E00850E10C3E5109EE49F502D
:1066A0002BAC0CAD0D850E12850810E5122510FAE5
:1066B000E43400FB79A2124C49E50C2415F50C508A
:1066C00002050D050E80CF75098B7E00750C0078D4
:1066D0000C122B5A780A122B56EEF50C780C122B52
:1066E0005A7808122B5A7405122E2DE0FDAC0912AF
:1066F000670C12434F7405122B84E50A450B6007A3
:10670000AA0AAB0B123EC974020261FFE5141269BA
:10671000C03515FBE5141267203515F583E0F92225
:10672000240FF582E42274F612258474FF122C18CB
:10673000EAFEEBFF126780127860A3A3A3A3A3A3D2
:10674000A3A3E0F91230CBE9851882851983F0758F
:1067500008007808122B5A7401122BEA880889095C
:106760007808122B567508357509807808122B5653
:106770001267861242A77405122B84740102564FC9
:10678000EE1263123F227901126790FAE43FFB2276
:10679000EE2402FCE43FFDEE240F2274F412258463
:1067A00074FA122C188A088B09EA127720127730B3
:1067B000FFEEFAEFFB122FB1E9601312342BEAFC63
:1067C000EBFDEEFAEFFB1248FBE96401700A74017D
:1067D000122E2DE4F0A380097401122E2DEEF0A3E9
:1067E000EF1279E6A3A3A3A3A3E0F8A2E6500874EE
:1067F00003122E2D7401F0E8A2E750087404122E43
:106800002D7401F07405122E2DE4F004122BF212F7
:1068100030FBE9851882851983F07A007B001234F9
:106820004F750A00780A122B5A7401122BEA880A53
:10683000890B780A122B56750A34750B80780A1268
:106840002B561268521242A77405122B847406024A
:106850006D247901E5082402FCE43509FDE50824EE
:106860000FFAE43509FB2274F612258474FF122C0A
:10687000181268DAF509A3E0F508A9091230B9E998
:10688000851882851983F090099AE0700B74016570
:10689000087005A909124409EE240B1268D2702C65
:1068A0007508007808122B5A7401122BEA8808899F
:1068B000097808122B567508367509807808122B4E
:1068C000561267861242A77405122B8402677BEE6C
:1068D000240EF582E43FF583E0221268DE22EAFE10
:1068E000EBFF1268EE3FF583E01268F5E022EE243C
:1068F00013F582E422F8A3E0F98882898322C0821A
:10690000C08390099AE0700312440F02706374F41C
:1069100012258474EF122C18EAFEEBFF12576E90CA
:106920000778E065087004A3E065097052A818A90B
:1069300019880A890B780A122B56750A11750B00F3
:10694000780A122B567C007D007A817B00123F4D25
:106950007404122B84E97027750A00780A122B5AE6
:106960007401122BEA880A890B780A122B56AC089C
:10697000AD091269A51243017403122B848021759D
:106980000A11750B80780A122B567808122B5612B2
:1069900068CFFD7C841269A512430D7404122B8408
:1069A0007411026D241269A922EE1269C03FFBEE38
:1069B000240FF582E43FF583E0F922FCEFFDE508C2
:1069C0002402FAE42274F112258474EB122C1812BA
:1069D00068DAFCA3E0FAE4CAFBEC2AF508E43BF52C
:1069E00009900778E065087004A3E0650960030278
:1069F0006A9488828983A3A3E09410500F888289C7
:106A000083A3A3E085188285198380088518828571
:106A100019837410F0E0C0E07404122E2DD0E0123F
:106A20007851A3A3A982AA83890C8A0D750E0078D8
:106A30000C122B527407122E2DE0FC7D00740812EC
:106A40002E2DAA82AB83123DFD7403122B84740495
:106A5000122BEA880A890B780A122B56750A1175CF
:106A60000B00780A122B567C007D007A817B001285
:106A70003F477404122B847404122E2DE09007B348
:106A80006005E0D2E48003E0C2E4F0851882851955
:106A900083E480088518828519837484F0E0C0E05F
:106AA0007401122E2DD0E0F07402122E2DE508F0A4
:106AB0007403122E2DE508F0125F8B126AF3122B6D
:106AC0005A7402122BEA880889097808122B567525
:106AD00008147509807808122B56790312678812FA
:106AE00042A77405122B847415026F7DE516127887
:106AF000433517F583E0F50878082274F4122584ED
:106B000074E0122C188A088B09AC18AD1912429542
:106B100090099AE0640270337402122E2DAE82AF97
:106B20008312342BEEFCEFFD1248FBE9601D12349A
:106B3000318A0A8B0BA80AA90B851882851983E074
:106B4000687003A3E0697003026D221235E77402D6
:106B5000122E2D12706A1234FDE964017003026D69
:106B6000227418122BF212343D7402122E2DAC82B4
:106B7000AD837418122BF21248FBE96032123437DD
:106B80008A0A8B0BA80AA90B851882851983E068ED
:106B90007003A3E069601885188285198312631C4D
:106BA00090054A1263267A4A7B05794B124A8D90EA
:106BB000099AE0600764016003026C6012763FC0CE
:106BC00082C0831234318A088B09D083D082E06579
:106BD000087004A3E06509605C7402122E2DAA827D
:106BE000AB831230238A088B09A808A909E84960F9
:106BF0002688828983A3A3A3A3E06401600D888211
:106C00008983A3A3A3A3E06402700C7402122E2D47
:106C1000AA82AB8312302F9005E8126D3260169075
:106C2000098EE06401700E12706E9005E9E0F58344
:106C3000888212276A1234318A088B09A808A909A8
:106C4000851882851983E0687003A3E06960117478
:106C500002122E2D12706A123005E96003124121D2
:106C60007402122E2D12706A1235D5790012706ED0
:106C700012324B740B122E2DE4126D36F8A3E0F98C
:106C8000740C122E2D126326740B122BF2122FD5B8
:106C9000E9603F7C087D0079007418122BF2123EE7
:106CA00009740E122E2DAC82AD837418122BF212C1
:106CB00048FBE9601D7402122E2DAC82AD83740E68
:106CC000122E2DAA82AB83122FAB740B122BF21251
:106CD0002FE77402122E2DAC82AD83740E122E2D6E
:106CE000AA82AB83122FAB740B122BF2122FDBE9AB
:106CF0006030740C122E2D12631C85188285198346
:106D0000E0687003A3E06960198518828519831211
:106D1000631C740C122E2D126326740B122BF212AC
:106D20002FE77420122B847F04022809F582E438AF
:106D3000F5831271F522F0851882851983E022749B
:106D4000F112258474F6122C18EAFEEBFF75080088
:106D500090081F126D3270507A377B00123EC3903C
:106D6000081FEAF0A3EB12752A60197C377D0079C1
:106D700000123E09EEFCEFFD90081F1270741242E3
:106D800065E9700B8518828519837488026EE61296
:106D90007824126F857401F07C717D429004D312C7
:106DA0007074124CB5026F7BE0C8126F857402F0EC
:106DB000EEFCEFFD127480124265E9700C851882BA
:106DC0008519837488F0750801750AE9750B0778D1
:106DD0000A122B5612708412299512782424281234
:106DE0007473FC1270B71278242414127473F9129D
:106DF00041C97404122B84126F92126FB82431129D
:106E000074736043127514FAE433FB123EC39008A6
:106E10001FE02432126FCD6022750CE9750D0775E5
:106E20000E00780C122B52127514FCE433FD127014
:106E3000A2123DFD7403122B84800C8518828519E3
:106E4000837488F0750801780A122B561270781234
:106E500029951278242411127473FC1270991278F7
:106E600024242B127473F91241C97404122B841256
:106E700078242434126FB824341274736035127578
:106E80000BFAE433FB123EC390081FE02435126F67
:106E9000CD6042750CE9750D07750E00780C122B4C
:106EA0005212750BFCE433FD127090123DFD740319
:106EB000122B84E508A2E04025126F9212747370C1
:106EC0000890081F1274D760157B007A00790012B1
:106ED000426B026F7B8518828519837488F0851850
:106EE000828519837486F07409122E2D740212762D
:106EF00083126FA1122E2DE8F0A3E9126FB2F508EC
:106F00007808122B5A7401122BEA8808890978082C
:106F1000122B567508207509807808122B567901B6
:106F20007406122BFAEEFAEFFB1242A77405122B2D
:106F3000841274C670427409122E2D7402F0126FFE
:106F40009B122E2D127531122B5A7401122BEA88C6
:106F50000889097808122B56750820750980780869
:106F6000122B5679017406122BFA90081F127074B6
:106F70001242A77405122B8412425F740A122B84EA
:106F80007F07022809126F8922242EF582E438F542
:106F9000832290081F12749C24312290081F126FC4
:106FA000A9A3A3126320740122E0F8A3E0F583886B
:106FB0008222127683A3E022F582E438F583126FF1
:106FC000C3C822E9F090081FE0F8A3E022F8A3E08C
:106FD0003400F988828983EAF0A3EB12785A12719F
:106FE000F522C082C08390081F126D326075E0C820
:106FF0002435126D2C6006127090123EC91278244E
:107000002432126D2C60061270A2123EC91278242E
:107010002412126D2C6009127078127074123EC91D
:107020001278242415126D2C60061270B7123EC916
:107030001278242429126D2C600912708412707445
:10704000123EC9127824242C126D2C6006127099FD
:10705000123EC990081F127074123EC990081FE4B6
:10706000F0A3F0D083D082022B36AC82AD8385189A
:10707000828519831270B1221274992412F582E468
:1070800038F583221274992429F582E438F5832295
:1070900012749924351270AB22127499242C127038
:1070A000AB2212749924321270AB22F582E438F5C7
:1070B00083E0FAA3E0FB2212749924151270AB222C
:1070C00074F1122584EAFEEBFF8C088D09750A0124
:1070D0008C0C8D0D750E00780C122B527C177D00D8
:1070E000123DFD7403122B84EE24121271C1F0A321
:1070F000F0EE24151271C1F0A3F012763FE0603A71
:10710000EE2412F8E43FF9880C890D127668123EDD
:10711000C31271E26021E50824121271D5122B52BC
:10712000E50824111271C9126220127074123DFD1B
:107130007403122B848003750A00E50812764D60F3
:1071400035EE2415F8E43FF9880C890D12766812A3
:107150003EC31271E26055E50824151271D5122B59
:1071600052E50824141271C91271B1127074123DE3
:10717000FD7403122B84E50AA2E0402BEE2412F5E5
:1071800082E43F126D30600912621F127074123E69
:10719000C9EE2415F582E43F126D30600AEE1271DB
:1071A000B1127074123EC9A90A026F80750A00807C
:1071B000CB1271B5222415F582E43FF58322EE242B
:1071C00014F582E43FF583E422127814E025E0FC14
:1071D000E433FDEE22127814E0F50CA3E0F50D780F
:1071E0000C22850C82850D83125BC3850C82850D74
:1071F000831271F522E0F8A3E0F9E8492274EE1257
:10720000258474ED122C18890A8A0E8B0F750C00D8
:10721000750D00750BFF7510FF7511FF7508007572
:107220000900851882851983E412752A6017740392
:10723000650A60067402650A7010E0C82430127492
:1072400073650F600579000274697C717D427A0074
:107250007B00124CB57401650A700A851882851985
:10726000837485803DE50A60067403650A70199091
:10727000081F1274A6F07403650A7029E50E6029D0
:10728000851882851983801A7402650A701BE50EC1
:1072900090081F70051274A680081278271274BD1A
:1072A0007402F08004E50A601E1274AC7019127446
:1072B000D06005126F95800A1274D7600A12782484
:1072C000243412747314F01274D0602212559CF599
:1072D00009127514F8E433F990081FE0FAA3E0CA24
:1072E00024321274E8241D12748D2425802E127409
:1072F000D7602E90081FE02417F508A3E03400F5AE
:107300000912750BF8E433F990081FE0FAA3E0CAFC
:1073100024351274E8240612748D240E127473F549
:107320000B7409122E2D7402126D3660030273D78E
:10733000E508450970030273D71274AC70047E220D
:1073400080027E21850882850983126FA1122E2D6D
:10735000126326900823E0C0E01278242430F582DE
:10736000E438F583D0E0F07412122E2D7403F0ACE3
:107370000CAD0D740A122BF21249018508828509A1
:1073800083A3E0F50C780C122B5A780B122B5A744D
:107390000C122BEA880C890D780C122B56781012DF
:1073A0002B56E5082406F50CE43509F50D780C128A
:1073B0002B5612747BF97409122BFAEEFA7B001229
:1073C00043197408122B847C717D429004D312708F
:1073D00074124CB5027467126F9B122E2D12753108
:1073E000122B5A7401122BEA880889097808122B8B
:1073F000567508207509807808122B567901740695
:10740000122BFA90081F1270741242A77405122BE7
:10741000841274C6704E1278242419F582E438F56B
:1074200083126FA3122E2DE8F0A3126FBE2418F55D
:1074300082E438126AF3122B5A7401122BEA88087C
:1074400089097808122B567508207509807808126A
:107450002B5679017406122BFA1274801242A7740B
:1074600005122B8412425F79017413122B847F0A58
:10747000022809F582E438F583E022127938E02207
:1074800090081FE02417FAA3E03400FB22F50CA3B8
:10749000E03400F50D1274992290081F1274A02296
:1074A000E0F8A3E0C8221274B674012290081F12FB
:1074B00074B6E06401221274A01274BD22242FF568
:1074C00082E438F58322127499126F89E0640222F3
:1074D00012751A90081F221274DB221274A0243431
:1074E000F582E438F583E022F582E43AF583E0287A
:1074F000F8A3E039F9E824FEF582E934FFF583E0EA
:10750000F510A3E0F51190081FE02290081F1274F7
:10751000DB25E02212751A25E02290081F1274A0C4
:107520002431F582E438F583E022126FC4F9E8498A
:1075300022E8F0A3126FC3F5838882A3E0F50878F0
:107540000822C082C0837B007A85790112426B02D7
:10755000706374F41225848C088D09EA240F127963
:10756000EC12794212631C8C828D83A3A3126326D2
:10757000EA240E1279ECA3F01277271276741278AF
:107580003650010FFCEFFDE5082406FAE43509FB4F
:10759000124901EE2408FE50010F8E828F83E0C055
:1075A000E0127934D0E0127735F8127924E81278B5
:1075B0003A50010FE5082412127647A3F0E508249B
:1075C0001512764712767DA30EAF83C0E012763F88
:1075D000D0E0F06028E508241212765F123EC31254
:1075E00079FF6019E5082412127652127641E0F90B
:1075F0001241ED8A0A8B0BAE0AAF0B8007E5082417
:10760000111276478E828F83E0A3AE82AF83C0E0F3
:1076100012770BD0E0F0601FE508241512765F1298
:107620003EC31279FF6010E50824151276521276D7
:107630004DF91241ED800512770BE4F0026D27E55C
:1076400008241112781422127814E4F0221277110F
:10765000E022127814125BEAEEFAEFFBE50822F85A
:10766000E43509F9880A890BE012766D2225E0FAE3
:10767000E433FB22FF12799C8C828D8322A3127645
:1076800083E022F08E828F832274F61225848C0888
:107690008D09127727FFEEFCEFFDAA08AB0912490E
:1076A00001EE2408FE50010F8E828F83127A4D1254
:1076B0007735850882850983A3A3A3A3A31278360F
:1076C00050010F8E828F83E0F8E508127720E812D0
:1076D000782B7403687026EEFCEFFDE508240BFAA6
:1076E000E43509FB1249018E828F83A3A3A3A3A3D0
:1076F000A3A3A3E0C0E012770BD0E0800A127918B0
:1077000012780EE8F0A3E9F0025652E5081277115C
:107710002212771A3509F58322E82414F582E4222F
:10772000126312127817221279C412772E22F5836F
:10773000E0FEA3E0221279631279A02274F21225EE
:1077400084EAFEEBFF750A00EE24101268D2C3949F
:107750000C400D12798D127827240B127473F50AE0
:10776000A80AE828F8E433F9E8240DFAE439FB1212
:107770003EC38A088B09EA4509700302780512673F
:107780008012797C8A828B8312795F7078EEFCEFAD
:10779000FDEA2403FAE43509FB124901EE2408FE50
:1077A00050010F8E828F8312799885088285098314
:1077B00012783950010F12780CE4F0E50A6046E5C2
:1077C00008240DF8E43509F98E828F83E0C0E012B9
:1077D000780CD0E012791FC0E012781CD0E012784B
:1077E0002B850A0B8E828F83E0FCA3E0FBEC888262
:1077F0008983127849500109EE2402FE50010F15C9
:107800000BE50B70DFAA08AB090264D8E508240B6E
:1078100012781422F582E43509F58322E508240C58
:107820001278142290081F12749C2212782F2212B0
:10783000796B0EAF8322A3A3A3A3F0A3E9F0EE24F8
:1078400002FE22240EF582E422125BC4E82402F830
:10785000221278552212785AA322F0888289832234
:107860001270AF8A828B83227F0102280974F21280
:1078700025841279C012559A850882F583E0F50DAA
:10788000A3858208858309A3A3E0F50C12797734D8
:1078900000FB123EC38A0A8B0BAE0AAF0BEE4F60A1
:1078A000378E828F83E50DF0850882850983E0FAA3
:1078B0001279D3850882850983A3A3A3A982AA8309
:1078C00089088A09880A7808122B521279723FFBBC
:1078D000123DFD7403122B840264D474F7122584C4
:1078E000EA2413F8E43BF988828983E0FAA3E0F5FF
:1078F000838A821279F21279131268F5A3E0FA886A
:10790000828983A3A3E0F9EA8C828D83A312632783
:1079100002786812785AE0221279A0F8E50822125B
:10792000782FE02212792822E508240FF582E43529
:1079300009F5832212793822E5081278433509F5D2
:107940008322127947A322F08A828B83A3221279A1
:107950005222F08A828B83A3A3A322A3A3A3A31200
:1079600079632212796BAE82AF8322F08E828F838D
:10797000A322AC0C7D00EE2404FAE42212798022CA
:10798000F583E0FEA3E0FF8E828F83E022127991DF
:10799000221268EE3FF583221279A0228E828F8315
:1079A000E0FAA3E0F9EA22E08E828F83A3A3A3A3E7
:1079B000A3A322F0850A82850B83A3228C088D095C
:1079C0001279C422EA1268EF3B22F0850882850909
:1079D00083A3221279F8EA8E828F83A3F0A3E9129F
:1079E00079E6E50CF02212796BA3A322F582E43B41
:1079F000F583E08C828D8322A3E0F8E4C8F9228528
:107A00000A82850B83125BC3850A82850B83127100
:107A1000F52274F61225841279BCF583127A461287
:107A2000767412783A50010F1269BB3509FB12497E
:107A3000018E828F83A3A3A3A3A3A3A3A3127A4D32
:107A4000A3A3F0025652126320E8FEE922127AF351
:107A5000A3A322127A5722E0FA1279F8EA28221216
:107A60007952A3A3A3A32274F61225841279BC121F
:107A70007AE0123E15EAF8EBF9ECFAEDFB850882A4
:107A8000850983122E16EE2404FE50010F8E828F7C
:107A900083E085088285098312795BC394065005CB
:107AA000127AF88037850882850983A3A3A3A3E00F
:107AB00064FE600E850882850983A3A3A3A3E0F476
:107AC000701B127AEB12782B850882850983A3A399
:107AD000A3A3E0F47007127B05F0A3E9F00256526D
:107AE00012772EFF7904EEFAEFFB228E828F83123B
:107AF0007AF322127AF8A322E0850882850983A30B
:107B0000A3A3A3A32212799C850882850983A3A33A
:107B1000A3A3A3A3A322EA1263123515F583126F60
:107B2000A9E02274EE12258474FC122C18851882A8
:107B3000851983EAF0A3EBF0127F0EE0F50AF50851
:107B4000127F00F87402122E2DE8F0A3E4F0740204
:107B5000122E2DE07003027EE2740D650A704674E9
:107B600002122BF2795312475D7402122E2DE0643B
:107B7000FE7003A3E0F47003027E1D7402122E2D2A
:107B8000E0F47003A3E0F47003027E1D127F3DA3B6
:107B9000A3E07003027E1D851882851983E0FEA391
:107BA000E0FF027DB27405650A701585188285199B
:107BB00083E0F8127F4379002421F8502E09802BAE
:107BC0007407650A7031127F3DE0700F7402122E47
:107BD0002DE0241BF0A3E03400801B85188285195A
:107BE00083127F4375F021A4F8A9F07402122E2DA0
:107BF000E028F0A3E039F07402122E2DE0FAA3E0A1
:107C0000FB123E218A088B09AE08AF09EE4F704780
:107C1000740C650A6003027EE2127F507003027EDC
:107C2000E2A2AFE433F508C2AF127F2D123893748D
:107C300002122E2DE0FAA3E0FB123E218A0C8B0DDE
:107C4000AE0CAF0DEE4F7009E508A2E092AF027ED8
:107C5000E2E508A2E092AF851882851983E0F50C71
:107C6000A3E0F50D750E00780C122B52850A081250
:107C70007F00FC7D00EEFAEFFB123DFD7403122B3A
:107C8000847405650A6003027D0C127EF6EE2403FF
:107C9000F510E43FF511851082127F21122B527CE2
:107CA000217D00AA08AB09123DFD7403122B8485C7
:107CB0001082851183E508F0A3E509F0127EEC85BA
:107CC0000882127F21122B528E828F83A3A3A3A33B
:107CD000A3A3A3A3E0FC7D00851082851183E0248B
:107CE00021FAA3E03400FB123DFD7403122B8485BE
:107CF0001082851183E02421F8A3E03400F985087F
:107D000082850983E8F0A3E9F0027DB27407650A71
:107D10006003027DB29010AE127F567003027DB2F6
:107D20009010AEE0F510A3E0F5119010AEE4F0A3D2
:107D3000F08E828F83A3A3E07031127EECEE240BD1
:107D4000F8E43FF9850882850983E8F0A3E9F08526
:107D5000100C85110D780C122B527C1B7D008508B0
:107D600082850983E0FAA3E0FB8038127EF68E82DA
:107D70008F83A3A3A3A3A3A3A3A3A3E508F0A3E5D1
:107D800009F0880C890D780C122B528E828F83A3F8
:107D9000A3A3A3A3A3A3A3E075F021A4FCADF0AA21
:107DA00008AB09123DFD7403122B84AA10AB11120B
:107DB0003EC99010B1127F566010EEFAEFFB127FB1
:107DC0001B12276AE96003027ED1740D650A600305
:107DD000027E81127F5EF988828983A3E054E0FAF3
:107DE00088828983E05403C394025031127F5EF588
:107DF000838882E01313543F540FF8900544E068E1
:107E0000701BEA7018851882851983E0F8A3E0C812
:107E1000241BF582E438F583E064026007AA18ABFE
:107E200019027EDFEE2413F8E43FF9E8241CFAE49B
:107E300039FBE8241DF582E439F583E0F9124AFFA5
:107E4000851882851983E0F8A3E0C8241CF582E434
:107E500038F583E0F47003A3E0F47069127F5EC824
:107E60002406F582E438F583E0C394024057EEFA25
:107E7000EFFB1233E9E9606AAA18AB191238938054
:107E800061740C650A703E127F0EA3E0641A6035BF
:107E90008E828F83127F53602C8E828F83A3A3A345
:107EA000A3E0C8240EF582E438F583E0A2E0501583
:107EB000EE240CFAE43FFBEE240DF582E43FF5835B
:107EC000E0F9124AFFEEFAEFFB9005A1E0F9123E4D
:107ED0002D740C650A700B127F506006127F2D12F4
:107EE00038937404122B847F0A022809EE2409F5C2
:107EF00008E43FF50922EE240BF508E43FF50922DA
:107F000074DB2508F582E43451F583E49322127F73
:107F10001222851882851983E0F8A3E0F583888210
:107F200022F583E0F50CA3E0F50D780C228518828C
:107F3000851983E02403FAA3E03400FB22127F12A8
:107F4000A3A322A3E0C82408F582E438F583E02245
:107F5000127F12A3A3A3E0F8A3E0F9E84922127F5D
:107F600012A3A3E0F8A3E022C082C08390099AE0A4
:107F70006004640170051233D180027900D083D08F
:107F800082022B367900022B3674F6122584E9FE24
:107F9000EAFCEBFD9010B0E060548C828D83E0F839
:107FA0007900EEC3943250047E328008EEC3946FA1
:107FB00040027E6E9010B0E0640170228E08E508E9
:107FC00024CEF508E434FFF509E88508F0A4C8AA32
:107FD000F08509F0A42AF97A3C7B0012232FC3E92B
:107FE0009401400474FF8001E88C828D83F07F024D
:107FF000022809FFFFFFFFFF851A87C2AF022B3659
:1080000024035400650078006100730020004900DB
:108010006E0073007400720075006D0065006E00E4
:1080200074007300240354004900200043004300FF
:10803000320035003300310020005500530042006B
:1080400020004300440043000B4B8738D532BB4C23
:10805000A32EE93F7B416D494F4947450000000091
:108060000000000000000000000000000000000010
:108070000000000000000000000000000000000000
:108080000030313233343536373839414243444594
:10809000460000000000000000000000000000009A
:1080A0000000FFFFFFFFFFFFFFFF000800040002CA
:1080B0000001FFFFFFFFFFFFFFFFFFFFFFFFFFFFCD
:1080C000FFFF0205020008017400000000000082AA
:1080D000003A003B0000000000000002000206021F
:1080E00019E0FCFF3C000000100E0000040000003E
:1080F000E71F030080510100F8FF000009433886A4
:10810000E8030000E204000058020000BC02000086
:108110003200000000F8FF0760EA000000000000E5
:1081200030000000E90300000B0000000100000027
:108130000A0000000200000097511800FEFFFFFF38
:108140001F000000080000006AAEE7FF965118000B
:108150009F020000E9FFFFFF0000FF00FFFFFFFF9D
:1081600064000000000000FFFA000000040309049E
:1081700000000000000000000A74F7122584E99056
:1081800005A1F0900556E4F01248D79005B5E4F04B
:10819000A3F09005A2F0A3F012358D90099AE0604B
:1081A0000464017006122FF31231B51248DD9005F8
:1081B00017E4F0A3F0124AC902B1B374F012258497
:1081C000EAFEEBFF548060689005A1E0F9123E39A9
:1081D0008A088B09EA4509604F7C0080010CEC7528
:1081E000F003A4F8A9F0747A28F582745139F58364
:1081F000E493F4602CE493F88508828B83E0687044
:10820000DCAA08EC75F003A4F8747B28F58274519D
:1082100039F583E493C0E0740193F583D08212278B
:108220006AAA08AB09123E27EEFAEF64800284AC1A
:10823000EF5420601E1233EF8A088B09EA4509606B
:108240000A12330BAA08AB09123E27EEFAEF64209C
:108250000284AC90099AE064027024EEA2E0501F00
:1082600090055BE0640F701179001232DBE9600960
:1082700090111712D3971232F3EE64010283B2EE1B
:1082800054207003028383750C007A207B009005D4
:10829000A1E0F9123F9BEA4B4C4D701790813412CC
:1082A000298D7A207B009005A1E0F9123F8F74049C
:1082B000122B847C0079047A007B001233B98A087F
:1082C0008B098018850882850983A3A3A3A3A3A390
:1082D000A3A3A37401F0850A08850B09E5084509E5
:1082E00060777C007904AA08AB091233B98A0A8B3B
:1082F0000B750C01E5082404F8E43509F988828936
:108300008312EF8812EADD70CD850882850983A388
:10831000A3A3A3A3A3A3A3A3A3E0640170A68508BA
:1083200082850983A3A3A3A3A3A3E0540470958526
:108330000882850983A3A3A3A3A3A3A3A3A374066D
:10834000128BAE700374B7F0E0FA8508828509835A
:1083500012868A1232ED0282D61233897C007901AC
:108360007A007B001233B98B09EA45097010E50CDD
:10837000700C7A207B009005A1E0F9123F95EE6425
:1083800020802FE0600764016003028482EE5410B5
:1083900060081231F1EE64108018EE54406008124B
:1083A0003269EE6440800BEE5480600B1230BFEEF9
:1083B0006480FAEF0284ACEF540160169005D41289
:1083C000CBDD600612C64712276AEEFAEF6401029F
:1083D00084ACEF540860471231C190098AE064010F
:1083E000703490098BE0602EF508E4F509F50AF584
:1083F0000B908100780C122DD67808790C12241F6E
:108400007808122B4E7A007B089005A1E0F9123F04
:108410008F7404122B84EEFAEF64080284ACEF54DC
:108420001060129005B3E06005E4F01231C1EEFA7D
:10843000EF64108077EF544060489005DE12CBDD8A
:1084400060399005E412CBDD603190098EE0640163
:1084500070299005DE12C64412276A9005E412C600
:108460004412276A90811812298D7A007B4090056A
:10847000A1E0F9123F8F7404122B84EEFAEF6440EE
:10848000802AEF5402600A123557EEFAEF64028038
:108490001BEF5404601912CAE712C8F9790190055C
:1084A0005412D39712313DEEFAEF6404FB80047A44
:1084B000007B0002C184C082C08374EA122C187C45
:1084C000167D007900AA18AB19123E097408122E05
:1084D0002D7402F090054A1297D41284F574091293
:1084E0002E2D12C8F97413122E2DE412CA43124A0B
:1084F000B77416800EE8F0A3E9F090055412D15835
:10850000227408122B8402C1BC74F712258474DF14
:10851000122C18EAFEEBFFEE4F602DAC18AD1912CD
:1085200034137406122E2DE0601E7417122E2DE0E7
:10853000FD7401122E2DE0FCEEFAEFFB7900122FF4
:1085400057E9600479A480027900742102B1B07403
:10855000F4122584EAFEEBFF8E828F83A3A3A3A3EC
:10856000A3A3E054406016128BA21234CDE9600739
:108570007AFF7BFF02865112C64002864490099A18
:10858000E060076401600302862A900541E0A2E1F1
:10859000400302862A8E828F8312868412CA09A320
:1085A000A3A3A3E0FA88828983A3A312D56A8E824B
:1085B0008F83A3A3A3A3A3A3A3E0541060047940D3
:1085C00080027900750AFE750BFF780A122B56128D
:1085D000B678122995AC08AD09128BA21231C77476
:1085E00004122B84E5086A7003E5096B600B12B670
:1085F0007D6A7003A3E06B704E750A00780A122B37
:108600005A79028E828F8312B268AA08AB0912359A
:108610000F7401122B847508CDAA088E828F8312E5
:10862000868A1232EDE9604C805790099AE0640224
:10863000600FE06004640170DD900541E0A2E1405C
:10864000D590054A12D39774FE6A700374FF6B606D
:10865000C512C64012DA8B1234CDE98E828F836048
:108660000512AA9E800312AAB312AABC124ABDE93F
:10867000F50870A5EE4F60097901EEFAEFFB1233B1
:108680009502BF51E0F812B2AA2212EE53E0F9228D
:1086900074F6122584E9FEEAFF7A0F7B00123E2170
:1086A000EA4B601F8A828B83740CF0EEA3A3F0EF79
:1086B0008A828B8312AEF19005A1E0F9123E2D79EA
:1086C00000802FEEF91233BF8A088B09A808A90988
:1086D000E849601C88828983A3A3A3A3A3A3A3A3BF
:1086E000A3740612E6CDE0F912327BEEF912339B49
:1086F000791002C53074F412258490055BE0640F94
:108700007030EA4B602C900556E064086005E06428
:1087100004701F8A088B09E4F50AF50B7808122B00
:108720004E7A017B009005A1E0F9123F8974041292
:108730002B840298BF74F2122584EAFEEBFF8C08AA
:108740008D09890A740E122E2D1297EE850C82F572
:1087500083E4F0A312C8FFE0F91234A9E9602612FD
:10876000D38A1234CDE96402701B8E828F83A3A357
:10877000A3A3A3A3A3A3A312B910850C82850D8381
:1087800012C8F98003750A0012B0A21460251460A3
:108790003A14605B14606314603F14607D24FE70C3
:1087A0000302883414700302884814700302885B43
:1087B000028869780C122B56AC08AD09EEFAEFFB73
:1087C0001231D97402122B84028864AC08AD09EE10
:1087D000FAEFFB1231DF02887312D38A1234CDE92B
:1087E0006003028869EEFAEFFB12322D028873A94A
:1087F0000AEEFAEFFB123515806A12BBB8640270FC
:1088000068E50A700A12DB447003A3E0697064EE45
:10881000FAEFFBA90A12349D804A12DB447003A3CD
:10882000E069704512BBB86402703EEEFAEFFB12CD
:108830003485803F9005D612CBDD6037EEFAEFFB32
:1088400012C64712276A802B12DB447003A3E0692B
:108850007017EEFAEFFB1235218018EEFAEFFBA944
:108860000A12352DE9F50A800A750A007AD37B00D1
:108870001244E1A90A02D16974F412258474DB124E
:108880002C188A088B098A828B83A3A3E0F9123300
:10889000BF8A0A8B0BAE0AAF0BEE4F70030289A999
:1088A000850882850983A3A882A983E0C0E012C855
:1088B000C7D0E012E6E464F160338508828509835D
:1088C000A3E064CD6027850882850983A3E0641A4C
:1088D000601B850882850983A3E064E9600F850831
:1088E00082850983A3E064E16003028A9390099A78
:1088F000E06007640160030289C28E828F83A3A3B4
:10890000A3A3A3A3A3E0540870030289C28E828F9D
:1089100083A3A3A3A3A3A3A3A3A37405F090099A7D
:10892000E0600464017053850882850983A3E064D4
:10893000E960479005DA12CBDD600612C6471227C0
:108940006A9005DC12CBDD6031900541E0A2E15078
:108950002912CDB5A3A3A312B0B88882898312D3FC
:10896000971235BDEA4B6012850882850983A3E022
:10897000F99005DC12C64412276A8E828F83A3A366
:10898000A3A3A3A3A3A3A3E0640270108E828F838A
:10899000A3A3A3A3A3A3A3A3A37406F0850882851E
:1089A0000983A3A3E0F912339B12338990099AE05B
:1089B0006402700990111B12D3971232F3742502CE
:1089C00098BC7900123395E97003028A9390099A52
:1089D000E0600764016003028A68900541E0A2E15B
:1089E0004003028A6812CBD8607E8E828F8312D3B6
:1089F000977404122BFA12CDD21234138508828593
:108A00000983A3E064E97020128B91122B5A850828
:108A100082850983A3E0F50A780A122B5A12D57BC6
:108A20001234497402122B84740D122E2D12CBCEE7
:108A300012EA0912C8F97409122E2DE06004794077
:108A400080027900740F122E2D12B0B8740D122E00
:108A50002D12D3971231D3E9600E8E828F83A3A398
:108A6000A3A3A3A3E04420F0EE2404F50AE43FF519
:108A70000B8E828F8312AD4AE0F9850A82850B83C3
:108A800012D3971248E9850A82850B83EAF0A3EB9B
:108A900002891C850882850983A3E0C0E074021264
:108AA0002E2DD0E012A530EEF0A3EF128BAEC0E079
:108AB0007403122E2DD0E012E2DEE0AA18AB19707A
:108AC0002E12311990099AE0600464017024740236
:108AD000122E2DE0701C128BA21234CDE97036904C
:108AE00005DA12CBDD602E12C64712276A80031208
:108AF00034A37402122E2DE064E97019128B9112C6
:108B00002B5A750AE9780A122B5A12D57B1234496E
:108B10007402122B8490099AE060076401600302DA
:108B2000897A900541E0A2E1400302897A8E828F22
:108B300083A3A3A3A3A3A3A3A3A3E0640270398E7A
:108B4000828F83A3A3A3A3A3A3E05404602A128B60
:108B5000A21234CDE98E828F83700F12C64474FF47
:108B6000F0A312AD65740502899BA3A3A3A3A3A3DD
:108B7000A3A3A3740302899B850882850983A3E0CC
:108B800064E9600302897AEEFAEFFB123533028959
:108B90007A8E828F8312D158E8FAE9FB750A017840
:108BA0000A228E828F8312B283FAA3E0FB22F0E5C1
:108BB0000812EE493509F583E02274F4122584EA9F
:108BC000FEEBFF7508007509008E828F83A3A3A3B7
:108BD000A3A3E0603B75080812D38A79FF122EAF79
:108BE0008B0BEA450B601075082C8E828F83A3A334
:108BF000A3A3A3E0D2E0F08E828F83A3A3A3A3A3B9
:108C0000E0540364016003028CC4430811028CC465
:108C1000EE241812BBBB6049EE241A12BBBB6003E2
:108C2000F4701D12DB447003A3E06970067508221E
:108C3000028CC4900556E064046003028CC4801C5E
:108C4000EE241BF582E43F12B6A0241A12BBBBFA35
:108C5000EE241912989412323FE970687509018068
:108C60006312D38A1234CDE96402700375080112CD
:108C7000DB447003A3E0697006E508D2E1F508E57E
:108C80000860158E828F83A3A3E07006E508D2E505
:108C90008004E508D2E6F50812D38A1234CDE964DF
:108CA000017006E508D2E0F5088E828F83A3A3E069
:108CB000601212B0A2F91234A9E964016006E50855
:108CC000C2E0F50890099AE0600464017012E508BA
:108CD000A2E1400CE509A2E04006E508D2E7F5086C
:108CE00002BF5174EC12258474CD122C18EAFEEBED
:108CF000FF851882851983129BB0751000751100CD
:108D000075090090099AE06402701C8E828F83A31B
:108D1000A3A3A3E0601190111912CBDD600990119B
:108D20001912D3971232F37405122BFA8E828F83A5
:108D3000A3A3A312CBD012D395123413E97003026C
:108D40008E6679017407122E2DE0C394024001193A
:108D50007409122E2DE0C3940240027900740E12A1
:108D60002E2DE064F87003A3E0F47003028E6674A5
:108D70000E122E2DE064F97003A3E0F47003028E4E
:108D800066740E122E2DE064FA7003A3E0F47003F3
:108D9000028E66740E122E2DE064FB7003A3E0F4C5
:108DA0007003028E667408122E2DE0F8900544E0E0
:108DB000686003028E66E9A2E04003028E6612B983
:108DC000077424122E2D12CA32241C12B90A7412EE
:108DD000122E2D12C8F9740B122E2DE0601D741C7A
:108DE000122E2DE0FD7406122E2DE0FC8E828F8354
:108DF00012D3957901122F57E9703D7405122BF2A9
:108E0000123305E9F508740B122E2DE0702E900533
:108E10003EE06028742255086422602074425508A0
:108E2000644270147422122E2D1297AB600E7422BD
:108E3000122E2D1297B160047ACF802CE9A2E65051
:108E40006E90099AE0600464017025900541E0A2EB
:108E5000E1501D7422122E2D12B0AB122A1A0101FC
:108E60000A878E00668E7AD37B001244E102978FC8
:108E70007422122E2D12B0AB24FD600B1460082456
:108E8000FD600424FD70DF7422122E2D1297F670FF
:108E90000E7422122E2D12C646A3E0640D601074CB
:108EA00005122BF2123509E96401700302978FEE67
:108EB000242DF582E43FF583129E887003A3E069B8
:108EC000701E750A00780A122B5A780A122B5AEE75
:108ED000242F1298941297C21234497402122B84D0
:108EE000740B122E2DE07003028F8D1297C2123573
:108EF000BD8A0A8B0BEA450B70030290367406128A
:108F00002E2DE0F88E828F83A3A3E028F8A3E0340F
:108F100000F9E8240D129799F88A828B83A3A3A302
:108F2000E068600FE88A828B83A3A3A312DC281277
:108F300097FCF079047406122E2D12A31FE02AF874
:108F4000A3E034008882F583A3AA82AB83123E1586
:108F50008A0C8B0D8C0E8D0F850A82850B83A3A343
:108F6000A3A3780C122B11400302978F90812C78C9
:108F70000C122CBF850A82850B83A3A3A3A3E50C47
:108F8000F0A3E50DF0A3E50EF0A3E50FF090099A2C
:108F9000E064026015E06007640160030290D09015
:108FA0000541E0A2E150030290CA900556E0640436
:108FB0006008E06409600302978FE508A2E54003BA
:108FC000029071EE242F12BBBBC0E07402122E2D52
:108FD000D0E012981CC0E07403122E2DD0E012983D
:108FE00014C0E07404122E2DD0E0F07416122E2D51
:108FF000E0640170267410122E2D1297B77003A32F
:10900000E0697017740E122E2D12D3971234CDE929
:10901000640270077416122E2DE4F012980A1229B9
:109020008D7406122BFA7409122BF212311F74047C
:10903000122B8402978F90059BE064016003028FDE
:109040008D7422122E2D1297AB7009E508A2E650FE
:1090500003028F8D7412122E2DE0F47003A3E0F43E
:10906000600CEEFCEFFD7405122BF2123311029727
:109070008FA2E650527422122E2D12CDCC7016748F
:109080001C122E2DE06402703E7405122BF2790042
:1090900012349D80327422122E2D1297B1701474E6
:1090A0001C122E2DE06404701E7405122BF2123473
:1090B0009180147422122E2D1297F6700A79007482
:1090C00005122BF212351502978F90099AE0601362
:1090D000E06401600302978F900541E0A2E1400344
:1090E00002978F7416122E2DE0601CEE240212B629
:1090F00067129D511412AEE7129D51C0E074161212
:109100002E2DD0E0F07006E508C2E7F508E508A2CC
:10911000E35061751110A2E25018740A122E2DE06E
:1091200054E3F0740A122E2DE0131313541FF8E0C9
:10913000802CA2E4502A740A122E2DE01313543FFF
:109140005407F86009740768600B18E87007C3E5F6
:1091500008C2E7F508E8333354FCF8E054E348F07C
:10916000740A122E2DE0C0E08E828F83A3A312AE6C
:1091700037D0E0F0900556E064046008E0640960D0
:1091800003029250740E122E2D12DB517003A3E0D5
:1091900069601F740E122E2D12D3971234CDE9641C
:1091A00002600F740A122E2DE05403640160030262
:1091B000978F7407122E2DE07041EE242F12BBBB47
:1091C000C0E07402122E2DD0E012981CC0E074038F
:1091D000122E2DD0E0129814C0E07404122E2DD05F
:1091E000E012980512298D7406122BFA7409122BBD
:1091F000F212311F7404122B8480527422122E2D0D
:1092000012CDCC7016741C122E2DE06402703E74C8
:1092100005122BF2790012349D80327422122E2D09
:109220001297B17014741C122E2DE06404701E7419
:1092300005122BF212349180147422122E2D1297E3
:10924000F6700A79007405122BF212351502978F09
:10925000746155087003029357E508A2E0506D123F
:10926000B0AF7405122BF212326FE9705C12344306
:10927000E9F5097416122E2DE0700F7410122E2DC0
:109280001297B77003A3E0696042A90912B0AF74E6
:1092900005122BF2123275E96024E508A2E3500CA6
:1092A00085188285198374FFF0A3800C740E122E2A
:1092B0002D1297D4E8F0A3E9F0751004800EE508AC
:1092C000C2E5F508750900800353089FE508A2E58B
:1092D000503FEE242F12BBBBC0E07402122E2DD0E3
:1092E000E012981CC0E07403122E2DD0E0129814E6
:1092F000C0E07404122E2DD0E012980512298D744E
:1093000006122BFA7409122BF212311F7404122B5D
:1093100084E508A2E6400302962AA818A919880A3B
:10932000890B780A122B56A9091297A2122BF21256
:1093300032F97402122B84E9F509700302962A743B
:1093400022122E2D12B0AB6401600302962A741013
:109350004510F51002962A7407122E2DE064017054
:109360005D7422122E2D12B0AB6405701EA818A9D0
:1093700019880889097808122B561297A0122BF227
:109380001232F97402122B8402978F7422122E2D3E
:109390001297F67029740E122E2D12D397123011D7
:1093A000E9601BA818A919880A890B780A122B569C
:1093B0001297A0122BF21232F97402122B84741637
:1093C000122E2DE070257407122E2DE06401700C12
:1093D0007422122E2DE0F81297F6600CEEFCEFFDD1
:1093E0007405122BF212331102978F12338FE9603A
:1093F0000302978F741D122E2DE070030294A57442
:1094000020122E2D12B0B8741F122E2DE0FA741EE9
:10941000122E2DE0F912323FE9607D741F122E2DBD
:10942000E0701E740E122E2D1297D412BC9EFAA359
:10943000E0FB12301D8B0BEA450B60030296248083
:10944000517420122E2D12D397741F122E2DE0F975
:1094500012323985188285198312DA8B7808740DD7
:10946000122E2DE060027810740C122E2DE0600494
:10947000740828F8740A122E2DE0600108088E8204
:109480008F83A3A3E028FAA3E034008A82F583E067
:1094900014F07510400296247508007808122B5AB3
:1094A000790B0295DD740E122E2D12C8F574091277
:1094B0002E2DE060030295F8E508A2E35003029523
:1094C000F87407122E2DE06401607A790085188205
:1094D00085198312D3971232938A0A8B0BA80AA993
:1094E0000BE849601C88828983A3A3A3A3A3E0643B
:1094F00001605288828983A3A3A3A3A3E0640260CE
:1095000044EE242D12B0B285188285198312D397A8
:109510001235BD8A828B83E5824583600FA3A3E069
:10952000F91235DBE96005C3940840197410122E56
:109530002D12D397123011E970030295D3740912DA
:109540002E2D7404F0E4F5097809122B5A741E12BA
:109550002E2DAC82AD83740F122E2D12D397740A68
:10956000122E2DE0F91232A57401122B84E9600F3E
:109570007510208E828F83A3A312B0AB543FF0747A
:109580001D122E2DE06023740E122E2D12B0B87411
:109590001E122E2DAA82AB8312340D8518828519D6
:1095A0008312DA8B74404510F5107407122E2DE0EB
:1095B0006401601579007410122E2D12B0B8740E6B
:1095C000122E2D12D397123245E508A2E3503779B7
:1095D0004080357508007808122B5A7902740F12F2
:1095E0002E2D12B0B87411122E2D12D39712350FE2
:1095F0007401122B8402978FE508A2E340030295C1
:1096000045744002954679007410122E2D12B0B8A0
:10961000740E122E2D12D3971231D3E960067420E6
:109620004510F510123443E9F50985188285198330
:10963000E064FE7003A3E0F4700375090090098DE7
:10964000E0640160030296DDEE241312BBBBF470EC
:1096500003A3E0F470030296DD740E122E2DC3E016
:1096600094F9A3E094FF507512B9077410122E2DCF
:10967000E0687003A3E06960647410122E2D12D3A9
:109680009712301D8A0A8B0BA80AA90BE849604D76
:1096900088828983A3A3A3A3E06401600D888289E3
:1096A00083A3A3A3A3E0640270337426122E2D7447
:1096B0000112E001F8A3E0F97431122E2D12C8F95D
:1096C0007426122BF2122FE1E960127429122E2D4A
:1096D000AA82AB8312302FE96003124121E508A270
:1096E000E7400302978FE509700302978F8E828F00
:1096F00083A3A3A3A3E0FA7B00123EC38A0A8B0BC9
:10970000EA450B700302978FEE2404F512E43FF54F
:10971000138E828F83A31297E4122B5285128285B7
:109720001383E0FC7D00123DFD7403122B8474074B
:10973000122E2DE0C0E07402122E2DD0E0F0740342
:10974000122E2DE4F0A3F07402122BEA880C890D7E
:10975000780C122B567810122B56E509F50878086C
:10976000122B5A12CAD9122995851282851383E0C9
:10977000F97407122E2D12B0B8AA0AAB0B123401DD
:109780007407122B84E96007AA0AAB0B123EC97456
:1097900033122B847F0C022809F582E412E82E2272
:1097A000790012CADD12B0BC74072212B2836406BB
:1097B0002212B28964072212D158EE241312B68401
:1097C0006822EE242BF582E43FF58312B6A624131B
:1097D0001298AF22E01297D922F8A3E0F9851882F7
:1097E00085198322A31297EE750E00780C22E0F5FE
:1097F0000CA3E0F50D2212B289640322A3E4F0A3C6
:10980000F0A3F0A322F012980A22EE2425F582E4B8
:109810003FF58322F0EE243112B68422F0EE24309C
:1098200012B6842274F4122584EAFEEBFF8C088DB4
:109830000990098AE0600F12DB447003A3E06970AD
:10984000051231C1804C790012D38A1232938A8278
:109850008B83E58245836032A3A3A3A3A3A3E05433
:10986000186027E508241C12C8DC122995E5082495
:109870001312C8DC122995EE2418129894129899A4
:109880001232AB7404122B8480087900129899125A
:1098900031EB802B12B684F9228E828F83A3A3A38F
:1098A000A3A3A3A3A3A312B6A6240B1298AF22F5D9
:1098B00082E43FF58312EA04FB227418122B847FA2
:1098C0000402280974F012258474EA122C188A0AFA
:1098D0008B0BEA2402F50EE4350BF50F0A0AFB1296
:1098E00030238A088B09AE08AF09750801850A8202
:1098F000850B83A3E0F509750C01AC0EAD0F740B5D
:10990000122E2DAA82AB831249017413122E2D122E
:109910009BB07415122E2D7402F07408122E2DE4D3
:10992000F09010BFE0700EEE4F700AE509700675FA
:1099300008C3029B04900556E0640860067508C2DF
:10994000029B00850A82850B83A3A3A3A3A3A3A3E1
:10995000A3A3A3E0A2E1500EA2E35005750C04807E
:109960000C750C038007A2E35003750C02EE4F70D8
:1099700003029A108E828F83A3A3A3A3E0640460E2
:109980000D8E828F83A3A3A3A3E06403700C7404E1
:10999000650C602C7403650C60268E828F83A3A3F4
:1099A000A3A3E06402600D8E828F83A3A3A3A3E030
:1099B000640170357402650C60067401650C701CDE
:1099C0008E828F8312D3971234EBE970438E828F8D
:1099D0008312A69B122E2D12C8F980348E828F839B
:1099E000A3A3A3A3E06402600D8E828F83A3A3A32D
:1099F000A3E06401700A8E828F8312A80212276A84
:109A0000E50A2402FAE4350BFB12302F7E007F00BA
:109A10007413122E2DE064FE7003A3E0F4704E1256
:109A20002FEDE97048E5096023900593E06402702A
:109A30001B9010C612D3971234EBE9700F9010C62A
:109A400012A69B122E2DE8F0A3E98020850A8285BC
:109A50000B83A3A3A3A3A3A3A3A3A3A3E05402F9EB
:109A60001231FD7413122E2DEAF0A3EBF0741312D1
:109A70002E2DE064FE7003A3E0F470057508C78026
:109A80007FE509F50D780D122B5A850A82850B8327
:109A9000A3A3A3A3A3A3A3A3A3A3E0F9E50A24027A
:109AA000FCE4350BFD7414122E2D12D397123143A2
:109AB0007401122B84E97048A90CE50A2402FCE425
:109AC000350BFD7413122E2D12D397122FFF8A0E11
:109AD0008B0FAE0EAF0FEE4F601E74026509700D56
:109AE0008E828F83A3A3A3A3A3E0D2E3F074151205
:109AF0002E2DE4F0F50880087413122E2D129BB061
:109B0000E5097009AA18AB19124A99800AFCA90C38
:109B1000AA18AB1912348BE9F8EE4F6053E50960CF
:109B2000208E828F83A3A3A3A3A3E0D2E6F07402C6
:109B30006509700D8E828F83A3A3A3A3A3E0D2E552
:109B4000F0850A82850B83A3A3A3A3A3A3A3A3A346
:109B5000A3E0A2E6500D8E828F83A3A3A3A3A3E06C
:109B6000D2E7F08E828F83A3A3A3A3A3A3E004F084
:109B7000E5087003E86034FC7D007A017B10124830
:109B8000E3EE4F600CE50A2402FAE4350BFB1230D9
:109B90002F7413122E2DE064FE7003A3E0F4600B0B
:109BA0007413122E2D12A80212276A741602C18194
:109BB00074FEF0A304F02274F712258474F7122CBB
:109BC00018EAFEEBFF900556E06403600DE06401C7
:109BD0006008E064096003029CE18E828F83A3E049
:109BE0006003029CB77C007D007A027B001248E390
:109BF000129CE68A828B8312B91090054712C8F92D
:109C00007953124A8D790090055412D39712313D41
:109C1000900556E06409600990055412D3971235F7
:109C2000B7851882851983740112CA437942124A92
:109C30008D9005567404F07401122BF2794A124A81
:109C4000877401122BFA7A4C7B0512490190099A0C
:109C5000E060046401701F90054AE064FE7003A395
:109C6000E0F4602A79007401122BFA90054A12D3AD
:109C700097122FFF8018E06402701390054712B00E
:109C8000B87A037B001248E312A5C21248E390059C
:109C900041E0A2E35004D2F08002C2F012CA397946
:109CA00052124A8D90099AE0640270329011171294
:109CB000D3971232F380278E828F83A3AE82AF8335
:109CC000FC7D007A037B101248E38E828F83E0F9DB
:109CD00090055412D39712313D900556E4F012339B
:109CE0005F740902B1B0EE2402FAE43FFB22C082A5
:109CF000C08390051712CBDD701F900556E01460ED
:109D00000924FC600A14600C800F900520803490B8
:109D1000051C802F90051E802AE8496008900518D0
:109D200012A328700C8A828B83A3E0F9123125805C
:109D30001D900517129D516402700512354B800E5F
:109D40009005D812CBDD600612C64712276A02C101
:109D5000BCE0F8129D5722A3E0C82406F582E4383F
:109D6000F583E02274F412258474FB122C188A08FF
:109D70008B097A0F7B00123E218A0A8B0BAE0AAF49
:109D80000BEE4F7003029E838E828F83740212CA81
:109D9000437950124A87850882850983A3E06003CE
:109DA000029E66900554E0F47003A3E0F4604490D2
:109DB0000554E064FE7003A3E0F4603785188285E3
:109DC0001983129E887003A3E06960278508828545
:109DD0000983A374EAF07A477B057953124A8D7A96
:109DE0004A7B05794B124A8D7A547B057950124A89
:109DF0008D807385188285198312DC1512C8F97A53
:109E0000477B057953124A8790054712AD5B12C80C
:109E1000F97A4A7B05794B124A877A497B0579E1C1
:109E2000124A8790055BE0C3940F501D900549E0EE
:109E3000C0E07402122E2DD0E0F07404122E2D74A6
:109E400001F004122BF2124AB1750A00780A122BA3
:109E50005A780A122B5A90114DE0F912AA4A12347C
:109E6000497402122B8485088285098312D6AAA31D
:109E7000F09005567403F0EEFAEFFB9005A1E0F9BF
:109E8000123E2D74050298BC12DC19E0682274F4AD
:109E900012258474E8122C18EAFCEBFD8C828D8369
:109EA000A3A3A3A37808122DD67808122D689005D5
:109EB000577808122CF87F7F7E7F790090055778BD
:109EC00008122DD6E97808122BB9E508A2E050292E
:109ED00078009005A28014850882850983A3A3E0F9
:109EE00069700108E508241412C8DC12A72570E780
:109EF000E8C39F5004E8FFE9FE09E9C3941B40BC96
:109F00008C828D83A3A3A3A3122E0AE8494A4B6037
:109F10007DEC2404F508E43DF509850882F58312FB
:109F20002E0A900557122E167C187D007900AA186B
:109F3000AB19123E09850882850983122E0A8518FD
:109F400082851983122E167404122E2D7401F0903E
:109F5000055DE0C0E07405122E2DD0E0F07407120C
:109F60002E2DE412CA43124AA5807090055412D3D4
:109F7000971231738A0A8B0BA80AA90B900554E833
:109F8000F0A3E912CBEA687003A3E069602D9005A5
:109F9000A212A7256025850882850983129E8870F4
:109FA00003A3E069700C850882850983A3A3E06E92
:109FB00060B9E508241412C8DC80D6EE900549F09B
:109FC000123341E96015900556E4F090052212CB5A
:109FD000DD600879C412C64712276A0298BA74F481
:109FE00012258474E8122C188A828B83A3A3A3A35E
:109FF000A3A3A3A3A312B910E8FAE9FB7900900583
:10A00000577808122DD6E97808122BB9E508A2E096
:10A010005031EA29F582E43BF583E0F89010C5E081
:10A02000C398501F750801750900750A00750B006B
:10A03000E97808122AF27808122D689005577808F6
:10A04000122CF809E9C3941B40B4900557122E0A4C
:10A05000E8494A4B604E7C187D007900AA18AB197C
:10A06000123E09900557122E0A851882851983120F
:10A070002E167404122E2D7401F07407122E2D74F6
:10A0800001F090055DE0C0E07405122E2DD0E0F0E7
:10A090007407122E2DE412CA43124AA59005567475
:10A0A00006F0801E900556E4F0FCFD7A047B101249
:10A0B00048E390052212CBDD600879C412C647122E
:10A0C000276A0298BA74F512258474D1122C188A62
:10A0D000088B098A828B8312B914741C122BFA8A9A
:10A0E000828B83A3A3A3A3A3A3A312B25F12D392D1
:10A0F000123371741C122E2DE0702C850882850994
:10A1000083A3A3A3A3A3A3A3A3E0C3940B40188E8C
:10A11000828F83A3A3A3A3A3A3A3A3E064027007D6
:10A1200012C8C7E0F4600302A31A900556E0640267
:10A13000700302A1FCE06406700302A1FC90051705
:10A1400012CBDD600812A328700302A231900556DD
:10A15000E064086008E06404600302A31A741E123D
:10A160002E2D12A31FA3A3A3A312B914900517E0C9
:10A17000F8496007129D5764026077900554E06EBD
:10A180007003A3E06F600302A31A74016A6016747F
:10A1900023122E2DAC82AD837A687B051248FBE931
:10A1A000600302A31A7A007B029005A1E0F9123F36
:10A1B0009BEA4B4C4D600302A31A900557122E0ADE
:10A1C000851882851983122E1690055DE0C0E07413
:10A1D00004122E2DD0E0F07405122E2D7401F074AF
:10A1E00006122E2D740212CA431230A7E960030230
:10A1F000A317EEFAEFFB12354502A31A90051712CA
:10A20000CBDD702D7508007808122B5A7808122BB8
:10A210005AEE2410F582E43FF58312CBD1A3A3A319
:10A22000A3A3A3A3A3A312AE2C1234497402122B2E
:10A23000848E828F8312B9107407122E2DE8F0A33A
:10A24000E912AD6512B9107409122E2D12CA32240A
:10A250000D12BBBBC0E0740B122E2DD0E0F012C863
:10A26000C712AD3E740F7808122DB8740C122E2D43
:10A27000E508F07420122E2DE0C0E0740D122E2D92
:10A28000D0E0F07422122E2DE0C0E0740E122E2DBC
:10A29000D0E0F0741D122E2DE0C0E07410122E2DAF
:10A2A000D0E0F0741E122E2DE0C0E0740F122E2D9F
:10A2B000D0E0F0EE241012BBBBC0E07411122E2DC2
:10A2C000D0E0F07421122E2DE0C0E07412122E2D79
:10A2D000D0E0F0742E122E2DE0C0E07413122E2D5B
:10A2E000D0E0F07423122E2DA982AA8389088A094E
:10A2F000750A007808122B527C087D007417122E04
:10A300002DAA82AB83123DFD7403122B84740712B5
:10A310002BF212313780031230AD742F02EF97E029
:10A32000FA8E828F83A3A322129D5864012274F6B1
:10A3300012258474C9122C189005D212CBDD600648
:10A3400012C64712276A900556E06408700302A3FC
:10A35000EB900593E064027023905273E4939005B0
:10A3600038F0905273E493900536F090055F7401D5
:10A37000F01297FC04F0A3E4F0A3806C900567E072
:10A38000F874B928F582E4340AF583E0FA900538C8
:10A39000F074BA28F582E4340AF583E0F9900536C2
:10A3A000F07508FF7509FFEA7808122D44E508F4F6
:10A3B000FCE509F4FD3395E0FE90055FECF0A3EDBC
:10A3C000F0A3EEF0A3F07508FF7509FFE9C39A78D2
:10A3D00008122D44E508F4FCE509F4FD3395E0FE90
:10A3E000A3ECF0A3EDF0A3EEF0A3F07C237D0079C5
:10A3F000007414122BF2123E09900567E070097484
:10A400001E122E2D74018006741E122E2DE412A52C
:10A4100030740FF09010C412CA437946124A8D74FA
:10A4200001122E2DE4F0901126E0C0E07402122EED
:10A430002DD0E0F0900544E0C0E07403122E2DD042
:10A44000E0F07404122E2DE4F07405122E2DE4F0C9
:10A450007407122E2DE4F0900567E0C3940F500CA2
:10A46000E0C0E07406122E2DD0E080077406122E94
:10A470002D740FF07C687D057408122E2DAA82AB16
:10A48000831249017C037D0079FF7410122E2DAADE
:10A4900082AB83123E099005A0E0C0E07413122E37
:10A4A0002DD0E012C83B7401122BF212336B7AA448
:10A4B0007B057945124A8D12347990055BE0C0E046
:10A4C000741C122E2DD0E0F090055CE0C0E0741DED
:10A4D000122E2DD0E0F0900549E0C0E0741A122E43
:10A4E0002DD0E01284F97418122E2D12C8F97420A0
:10A4F000122E2DE4F090055EE0C0E0741F122E2DA8
:10A50000D0E0F07434122E2DE4F07429122E2DE4D4
:10A51000F07A477B057953124A8D7A4A7B05794B4D
:10A52000124A8D7414122BF2124AAB743702C52DE5
:10A5300012A53422F085188285198322C082C08337
:10A540008A828B83A3E09005566004E4F0807074E7
:10A5500008F0900567E0702890052212CBDD6008B6
:10A56000790012C64712276A90055412B0B87A05CE
:10A570007B001248E390055412D3971235B7801828
:10A58000790012313190054712B0B87A067B00127B
:10A5900048E312A5C21248E39005DE12CBDD601F2E
:10A5A00090098EE06401701790811812298D7A004D
:10A5B0007B409005A1E0F9123F897404122B8402BC
:10A5C000C1BC90054A12B0BC7A047B002274F4121C
:10A5D000258474EA122C18EAFEEBFF129CE6123076
:10A5E000238A088B09EA4509700302A6968A828BA2
:10A5F00083A3A3A3A3E0640160278A828B83A3A320
:10A60000A3A3E06402601A8A828B83A3A3A3A3E0BE
:10A610006403600D8A828B83A3A3A3A3E064047008
:10A6200075EE2402FCE43FFD740B122E2DAA82ABC2
:10A630008312490185088285098312A69B122E2D5B
:10A6400012C8F97415122E2D7401F07408122E2DF3
:10A65000E412CA43124A9F890AAC0A7D007A077B3A
:10A66000001248E3850882850983A3A3A3A3A3E07E
:10A67000C2E012C128A3A3740112E2ED5001097ACD
:10A68000027B00122327E8850882850983A3A3A300
:10A69000A3A3A3A3A3F074160298BC12D1587413F9
:10A6A0002274F212258474F8122C18EAFEEBFF8C47
:10A6B0000A8D0B890C9080BAAC18AD197408122A57
:10A6C000B2F50DEEFCEFFDAA18AB191248FBE970CC
:10A6D00003750D019005A2801AEEFCEFFDE508243C
:10A6E0000BFAE43509FB1248FBE97023E508241452
:10A6F00012C8DC12A7256024E50DA2E040DB850826
:10A7000082850983E0650A7004A3E0650B70DD852E
:10A710000882850983A3A3E0650C70D0AA08AB0961
:10A72000740802D16612AD42E508450922C082C014
:10A73000839005A202C1B974F71225849005A21274
:10A74000EA04800C12D42312B917123EC9EEFAEFB4
:10A75000FBEA4B70EF9005A2E4F0A3F002B1B374F2
:10A76000F4122584EAFEEBFFEE241312BBBB640354
:10A77000700CEE240BFAE43FFB123023800EE064F1
:10A7800002707C12C8C712D39712301D8A088B0939
:10A79000E508450960698E828F83A3E0700F850804
:10A7A00082850983A3A3A3A3A3A3E4805164F160DA
:10A7B0000A8E828F83A3E064E17027850882850971
:10A7C00083A3A3A3A3A3A3E06401701685088285D5
:10A7D000098312A80212276AEE240BFAE43FFB1247
:10A7E000302F850882850983A3A3A3A3A3A3E060D8
:10A7F0000E850882850983A3A3A3A3A3A314F00253
:10A8000098BF1298B590053012C90D2274F1122527
:10A81000848A088B09ECFEEDFF890A12D697EEF8C0
:10A82000EFF9A30EAF838A828B83A3A3E0C454F015
:10A83000FA88828983E04A12A8ED12D6AB12A8E802
:10A84000E0333354FCF88E828F83E04812A8E8A3EB
:10A85000E033333354F8F88E828F83E048F0EEF81B
:10A86000EFF9A30EAF838508828B83A3A3A3A3A3D1
:10A87000A3E0A2E0E4331313FA88828983E04AF06C
:10A88000E5082407F50CE43509F50D750E00780C84
:10A89000122B527C087D00EEFAEFFB123DFD740393
:10A8A000122B84EE2408FE50010FE508240FF50C4E
:10A8B000E43509F50D780C122B527C037D00EEFA7D
:10A8C000EFFB123DFD7403122B84E50AC3940F4085
:10A8D00012E5082412F582E412DF218E828F83A311
:10A8E000A3A3F07F0702280912A8EDA322F0850890
:10A8F000828B83A3A3A32274F1122584EAFEEBFFCB
:10A90000890A8C088D098E828F83E08C828D831258
:10A91000B6B6AE82AF83E012BF5612C144C412BFB6
:10A920005612A9C1E054038C828D8312C142A2E267
:10A93000E4338C828D8312C141131313541F12BF51
:10A940005612C140A2E7E4338C828D83A3A3A3A354
:10A9500012A9C18E0C8F0D750E00780C122B527C33
:10A96000087D00E5082407FAE43509FB123DFD7473
:10A9700003122B84EE2408FE50010F8E0C8F0D78ED
:10A980000C122B527C037D00E508240FFAE43509F4
:10A99000FB123DFD7403122B84E50AC3940F40158E
:10A9A0008E828F83A3A3A3E0C0E0E508241212C81F
:10A9B000DCD0E08008E508241212C8DCE4F002A82C
:10A9C000E3A3A312B6BA0EAF832274F51225848ACC
:10A9D000088B098A828B83A3AE82AF83E0F91231A0
:10A9E0005B8E828F83E064EB602485088285098317
:10A9F000A3E064E16018850882850983A3E064F11F
:10AA0000600C850882850983A3E0641A70098508B3
:10AA100082850983A3E4F090111712D3971232F3C1
:10AA2000750A01780A122B5A850882850983A3E0EA
:10AA3000F5087808122B5A790012AA4A1234497480
:10AA400002122B8412338902EF9A90055412B0BC83
:10AA500090054A1298B522C082C083E99005B4706F
:10AA600003E4800274018065E0F902C1BC74F7124E
:10AA70002584EAFEEBFF8E828F8312CA0B12DA70F6
:10AA800012DA8B1234CDE98E828F83600512AA9E72
:10AA9000800312AAB312AABC124ABD02B1B312AA11
:10AAA000A5E4F0A322E0F8A3E0C8240DF582E43881
:10AAB000F5832212AAA57401F0A3E422F07CE17DC3
:10AAC000328E828F831298B522EAF0A3EBF002C196
:10AAD000BC74F61225849005B4E0701B7C007901EB
:10AAE0007A007B001233B9EA4B600C8A828B8312A6
:10AAF000CBDD60031232E702C530C082C083790427
:10AB00001233B3E9F8905280E493C398401079FF70
:10AB10001233B3E9F890527FE493C398500479015B
:10AB20008002790002C1BC74F01225848A088B0966
:10AB3000890B750C008A828B83A3A3A3A3A3A3A371
:10AB4000A3E0F91233BF8A0E8B0FAE0EAF0F750A5A
:10AB500001EE4F600302ABF785088285098312ADD1
:10AB60004AA3A3A3A3A3A312BC9012D3971233A703
:10AB70008A0C8B0DAE0CAF0DEE4F700302AD308E14
:10AB8000828F83A3A3A3A3E4F0A3F0E508240CFA27
:10AB9000E43509FB8A828B83E0C0E012E2E3D0E077
:10ABA000F01234D9EE240D12DA85E50812DF1335E0
:10ABB0000912B90E12B67812C8F9750C01EE240606
:10ABC00012BBBF547FF0A3E054FC12E6E4540460CF
:10ABD0000302AC6E90111FE0F50875090074077848
:10ABE00008122D448E828F83A3A3A3A3A3A3E045C1
:10ABF00008F0A3E04509F08E828F83A3A3A3A312DC
:10AC0000AD3C74077808122DB8E5085407F508E53F
:10AC10000B606B8E828F83A3A3A3A3A3A3A3A3A381
:10AC2000740212C14512B027600B90054212AD5B51
:10AC3000A3A312C8F9E508700302ACFCEE240612C7
:10AC4000EE1C547FFCA3E054FCFDE50824FFF5084E
:10AC5000E434FFF50974077808122D44EC4508F830
:10AC6000ED4509F98A828B8312C8F902ACFC8E8209
:10AC70008F83A3A3A3A3A3A3E0448002ABF6E508BC
:10AC80007005750A0080758E828F83A3A3A3A3A38A
:10AC9000A3E05420600C123E1BEA547F7900245F2D
:10ACA00080198E828F83A3A3A3A3A3A3E054106073
:10ACB0001A123E1BEA540F7900240A5001098E82B1
:10ACC0008F83A3A3A3A3F0A3E9800D8E828F83A318
:10ACD000A3A3A37401F0A3E412AD657404F07A2079
:10ACE0007B009005A1E0F9123F9BEA4B4C4D700CA4
:10ACF0007A207B009005A1E0F9123E63E50CA2E00A
:10AD000050318E828F83A3A3A3A312D39BF9EEFAB3
:10AD1000EFFB1233ADE9601B12B1A812CBDB600967
:10AD200012B29712D397123EC9EEFAEFFB123EC948
:10AD3000750A00A90A02C1848E828F83A3A312AD73
:10AD40004222E0F508A3E0F50922A3A3A3A3A3A34D
:10AD500012B0BC850882850983A32212D1588E8245
:10AD60008F83A3A32212C8E9A3A3A32274F41225FC
:10AD70008474F7122C187E001233BFEA4B70030262
:10AD8000AE258A828B83A3A3A3A3A3A3A3A3A3E03B
:10AD90006406600302AE258A828B83A3A3A3A3A3C8
:10ADA000A3A3E0FF8A828B8312AE37E0C0E0740871
:10ADB000122E2DD0E012B27C12C8F61233DDEF5401
:10ADC00008606085188285198312B0B87A007B000C
:10ADD0001233A18B0BEA450B704912EF91124AD541
:10ADE0007C007D007A007B0080258E828F8312B0EC
:10ADF000ABF47003A3E0F4602A90055412AE2C1259
:10AE00004ACFE9641A601C7C007D00EEFAEFFB1269
:10AE100033A18A0A8B0BAE0AAF0BEE4F70CC7900D0
:10AE2000124ADB7E01EEF974090298BC12B0BC8EA6
:10AE3000828F831298B52212B90212AE3E222408E4
:10AE4000F582E438F58322C082C083EA4B70059016
:10AE500005B580068A828B83A3A312B05B60258A26
:10AE6000828B83A3A3A3A3A3A3A3E0540860E5EC70
:10AE70004D60158A828B8312B0AB6C7003A3E06DBA
:10AE800070D280047A007B0002C1BC74F212258467
:10AE9000EAFEEBFF890A8C088D097A117B00123ECD
:10AEA000C3EA4B603E8A828B83A3A3A3A3A3A3A37D
:10AEB000A3A3E412B270A3E50A12DC28A3A3A31291
:10AEC000F0728A828B83A3A3A3A3E4F0A312B291AE
:10AED00012AEF112DA7812B786E4F012AEE6A3A34E
:10AEE000F0A3F002D169A312AEEB22F08A828B8329
:10AEF00022A3F012EE483BF583E4F02274F412250D
:10AF000084EAFEEBFF89088C0A8D0BEE4F7003027A
:10AF1000AFB074016508701279011233B3E9F8908B
:10AF20005285E493C3985022801674046508701407
:10AF300079041233B3E9F8905280E493C398500A2D
:10AF40007911806E7402650870668E828F83A3A368
:10AF5000A3A3A3A3A3A3A3E50812BEC112D68F8EF9
:10AF6000828F83A3A3E4F0A3F09005B512CBDD603C
:10AF7000178003E0F8A312CA12A3A312B05B888261
:10AF80008983A3A370ED80039005B512DA7C7A2043
:10AF90007B009005A1E0F9123F9BEA4B4C4D700CF1
:10AFA0007A207B009005A1E0F9123E6379008002CF
:10AFB00079C10298BFC082C083E9F879009005B5D5
:10AFC000801D8A828B83A3A3A3A3A3A3A3A3A3E02F
:10AFD00068600574FF687001098A828B83A3A312DD
:10AFE000B05B70DE02C1BC74F7122584EA4B7005B9
:10AFF0009005B580068A828B83A3A312B05B602084
:10B000008A828B83A3A3A3A3A3A3A3A3A3E06970B2
:10B01000E4EC60108A828B83E012B02770D7800442
:10B020007A007B0002B1B312AAA6E0540422C082C7
:10B03000C0839005B580068A828B83A3A312B05B80
:10B0400060128A828B83A3A3A3A3A3A3A3A3E06913
:10B0500070E580047A007B0002C1BC1298B5EA4B0F
:10B060002274F7122584EAFCEBFD9005B580068A70
:10B07000828B83A3A312B05B60218A828B8312B080
:10B08000AB6C7003A3E06D70E68A828B83128686B8
:10B0900012CAF8A2E0E43370D680047A007B000282
:10B0A000B1B3EE241DF582E43FF58312B28322EEA4
:10B0B0002413F582E43FF58312B0BC2212B0C02203
:10B0C000E0FCA3E0FD2274F21225848A0A8B0B8C2B
:10B0D0000C8D0D750800750900EA450B6030900570
:10B0E000B580068E828F83A3A312B917EE4F601E20
:10B0F000AC0CAD0DEEFAEFFB850A82850B831227AF
:10B100006AE9640170DDEEF8EFF988088909AA0898
:10B11000AB0902D1697900022B3674F712258490AD
:10B1200005B512B9107C007D00800DE8FCE9FD88B2
:10B13000828983A3A312B910E8496030EA687002DB
:10B14000EB6970E79005B512D397E86A7002E96B76
:10B1500088828983A3A3700812B9109005B580096D
:10B1600012B9108C828D83A3A312C8F9804574F79D
:10B17000122584EAFEEBFFEE4F602B1233D712B29A
:10B180009D123EC98E828F8312D397123EC912B18F
:10B19000A812CBDB600912B29712D397123EC9EE08
:10B1A000FAEFFB123EC9800BEE240DF582E43F223C
:10B1B000122B847F0102280974F71225848A828B5E
:10B1C0008312B2689005B512B9107508007E008030
:10B1D0003388828983A3A3A3A3A3A3A3A3A3E06427
:10B1E0000570180E88828983E0FFA3E0F5838F82C3
:10B1F000E06C7003A3E06D7002050888828983A368
:10B20000A312B910E84970C990527C12E438500872
:10B2100090527812D2D8400F8A828B83A3A3A3A323
:10B220007401F0A3E4800C900542E0F812B25FE8EC
:10B23000F0A3E912B291740512B270E0440812B2A0
:10B240007CF47003A3E0F4600E90055412D59212C2
:10B250004ACFE9641A70057901124ADB02B1B3A33F
:10B2600012B660A3A3A3A32212B283FCA3E0FD2223
:10B2700012B2742212DC30A3A3A3A32212AEEB12EB
:10B28000B28322E0F812B28922A3E0F5838882E03B
:10B290002212B274A3A32212B1A8F5832212B2A47F
:10B2A0001298B3228E828F83E0F8A3E0C8241FF5A2
:10B2B00082E43822C082C083EAFCEBFDEC4D6017CB
:10B2C000EC24FBF582ED34FF12CBDB700712B30EDA
:10B2D000E0F46007123E27790580309005A1E0C0B8
:10B2E000E012B30ED0E0F0905270E493F97AB77B9D
:10B2F00005123E5DE9640170107A007B209005A183
:10B30000E0F9123E6379008002790402C1BCEC24AA
:10B31000FFF582ED34FFF5832274F4122584A2AF89
:10B32000E433F508C2AF9005B712B917EE4F603A93
:10B33000EE24FBF582EF34FF12CBDB7A007B20900A
:10B3400005A16007E0F9123E638005E0F9123E694D
:10B35000E4F50AF50B780A122B56EEFCEFFD7AB7EE
:10B360007B05123E577402122B84E508A2E092AFCF
:10B37000EEFAEFFB0298BF74F012258474DB122CF6
:10B3800018EAFEEBFF750B00750A007508FE7509DB
:10B39000FF12338FE9600302B653EE241512BBBBD4
:10B3A000604690113AE0C43354E0F8E0333354FC83
:10B3B00048C0E012D37CD0E012B6B612D39679FF23
:10B3C000122EAF8B0DEA450D6011750B017508FF4C
:10B3D00012B67D440412C916D2E0F090099AE060DA
:10B3E0000464017003750A408E828F8312D3951214
:10B3F00034CDE9600312C9E9EE241312BBBB700D12
:10B4000090527BE493C0E012CAD9D0E0F08E828FD4
:10B4100083E0A2E7500454038019EE241412BBBB4E
:10B420007012900533E0C0E012EDFAD0E0F0900524
:10B4300033E004F012EE137019901128E0600D90C3
:10B44000053EE0700D8E828F83E07006EE241112AF
:10B45000C9EC90099AE0600464017048900541E0ED
:10B46000A2E15040E50BA2E040218E828F8312D3EF
:10B47000951234CDE9602D8E828F83E0600DEE242D
:10B480000B12B0A5F91234A9E9601912B68C700339
:10B4900002B604EE241312EE16600302B60412B6CE
:10B4A0007D54FBF08E828F83E06401700DEE240BDF
:10B4B00012B0A56402700312B69912B68C60030232
:10B4C000B57DE50BA2E0500302B57D90099AE060DE
:10B4D000076401600302B57D900541E0A2E14003ED
:10B4E00002B57DE50AF50B780B122B5AEE2406FC0B
:10B4F000E43FFD8E828F8312D395EE24121298942E
:10B500001232A57401122B84E9600612C9E912B641
:10B51000928E828F83A3A3A3A3A3A3E0603CEE2417
:10B5200002F50CE43FF50D850C8212B6A02407FA53
:10B53000E43FFB12340D8A088B09850C82850D834C
:10B54000E065087004A3E06509700C8E828F83A308
:10B55000A3A3A3A3A3E4F012B6998E828F83E06421
:10B56000016008A90A12B6AB123245A90A8E828F71
:10B570008312B6AB1231D3E9600312B692AC18ADA8
:10B5800019EEFAEFFB1234078A0A8B0B74FE65087A
:10B59000700474FF6509700312AD38EA450B70033F
:10B5A00002B6578E828F83E0C0E07401122E2DD038
:10B5B000E0F07402122E2D12DA7C7401122BEA884C
:10B5C0000C890D780C122B5612B678122995EE24A0
:10B5D0000E12BBBBF50C780C122B5A9005471229A2
:10B5E000957407122E2DE0F9AC08AD0912340174E0
:10B5F00007122B84E9FE74106E705EAA0AAB0B1260
:10B600003EC98055EE241312BBBBC0E07415122E48
:10B610002DD0E012EE77740D122E2D12CA322404B2
:10B6200012B66712B910740F122E2D12CA322414DA
:10B6300012BBBBC0E07416122E2DD0E012E2D9125C
:10B64000B66012B0B87404122BF2123275E96003BE
:10B6500002B4A4791180047E10EEF9742502C18130
:10B66000E0F98A828B832212B66B22F8E43FF9E874
:10B67000FAE9FB8A828B8322EE12C9FE2212B6817E
:10B6800022EE240FF582E43FF583E02212B68154C6
:10B69000402212B6814420F02212B6814440F022AA
:10B6A000F58312B6A62212B0C0EE22A3A3A3A31262
:10B6B000D3A71298B52212B6BA22F08E828F83A336
:10B6C00022C082C08374DC122C188A828B83A3A3CD
:10B6D000A3A312B910740E122E2DE8F0A3E912D113
:10B6E0004F740C122E2D12C8F912B786E0C0E07408
:10B6F0001A122E2DD0E0F012B7903B12B90E742022
:10B70000122E2D12C8F9EA12D3843BF583E0C0E073
:10B710007408122E2DD0E0F0EA241CF582E43B12CE
:10B72000B90E7412122E2D12C8F9EA2411F582E412
:10B730003BF583E0C0E07409122E2DD0E0F0EA243E
:10B7400012F582E43BF583E0C0E07407122E2DD0A1
:10B75000E012A53074FFF07401122E2D74FFF07406
:10B7600002122E2D74FFF090811C12298D74041288
:10B770002BFA7407122BF212311F7404122B8479E6
:10B78000007424028503EA240DF582E43BF583224C
:10B79000EA12EE492274EE12258474EF122C188AF4
:10B7A0000E8B0F8C088D09890C750A107A217B008D
:10B7B000123EC312D1AFE849700302B8FB750B000B
:10B7C0007C217D007900851882851983E0FA123E7C
:10B7D000097426122E2D12B91790099AE06004649C
:10B7E00001703EAA08AB0912301D8A108B11A810F7
:10B7F000A911E849602388828983A3A3A3A3E064F5
:10B8000001600D88828983A3A3A3A3E06403700968
:10B81000EE5440700474044FFFEF54046003750B42
:10B820000190055412D39785188285198312B902A5
:10B830002409F582E43812DA897423122E2D12B904
:10B8400010740F122E2DE8F0A3E912B91D12EE3F6D
:10B8500012B91D12AE3E740212BC9A12C645E5081A
:10B86000F0A3E50912B91D12EE0AE50CF0742512D9
:10B870002E2DE0F50885188285198312EE4FE50814
:10B8800012B91D241FF582E438F583E50EF0A3E517
:10B890000FF07406122E2D12DA7C7408122E2DE58C
:10B8A00008F07428122E2D12C644C082C083740C76
:10B8B000122E2DAC82AD83D083D0827403122AB2B3
:10B8C000A90BAA18AB19123395E9640170219009EC
:10B8D0009AE0600464017012E50BA2E0500CA90824
:10B8E0001233BFEA4B60031233E3750A00800C8504
:10B8F000188285198312D397123EC9A90A741102BE
:10B90000BECE12D15DC822EE2413F582E43FF5834A
:10B9100012D15822A3A3A3E0FEA3E0FF2212D1BEBE
:10B92000C82274EE122584EAFEEBFF8C088D098E86
:10B93000828F83A3740812CA25E060088E828F83E9
:10B94000A37410F012BBB860098E828F83A3E02429
:10B9500008F0EE241512BBBB60088E828F83A3E033
:10B9600004F08E828F83A3A3A3A3A3A3E060198E08
:10B97000828F83A3A3A3A3A3A3A3E0C3332402F8CA
:10B980008E828F83A3E028F0EE241112BBBB6005EA
:10B99000750B0E8003750B008E828F83A3E0F8EE8B
:10B9A000240D12BBBB28250B8C828D83F0EE241155
:10B9B00012BBBB601190053FE0F9122F5D85088234
:10B9C000850983E029F0850882850983E0C39475A1
:10B9D000400975080075090002BBB1E0FA7B00124E
:10B9E0003EC38A088B09EA4509700302BBB18E8207
:10B9F0008F83E0FA90054412BBC97402780C122DB3
:10BA000044EA450CFAAB0DEE241212BBBB5403F50D
:10BA10000C750D007406780C122D44EA450CFCEBF5
:10BA2000FDEE241512BBBB6004780180027800EEA5
:10BA30002416FAE43FFBE8F9ED49FDEE241112BBB0
:10BA4000BBF50C7409780C122D44ED450DFD8A826E
:10BA50008B8312BBC9740B780C122D44ED450DFD80
:10BA600012BE9E12BBC9740C780C122D44ED450D0C
:10BA7000FD8E828F83A3A3A3A3A3A312BBC9740AC1
:10BA8000780C122D44ECF8ED450DF9E88508828517
:10BA90000983F0E9A3F0EE240212BBBF850882857A
:10BAA000098312BBEDF0EE2404F8E43FF9888289A3
:10BAB0008312C0EFA312BBEDA3A3F0EE241312BBBD
:10BAC000D0F0EE241412BBD0A3F0750A088A828B42
:10BAD00083E06015EE241812B0B2E5082408FAE4F9
:10BAE0003509FB124901750A1012BBB8601BEE2420
:10BAF0001A12B0B2850A0CE508250CFAE43509FBE8
:10BB00001249017408250AF50A8E828F83A3A3A324
:10BB1000A3A3A3E06058EE2407F510E43FF51185D8
:10BB20001082F583E0C0E012C8D5D0E012BBDDE0A2
:10BB3000C0E012C8D5D0E012BBDD1297E4122B5240
:10BB4000851082851183E025E0FCE433FD850A0C35
:10BB5000E508250CFAE43509FB123DFD7403122BB0
:10BB600084851082851183E0C333250AF50AEE240B
:10BB70001512BBBB6008C0E012C8D5D0E0F012C8F7
:10BB8000C71297E5122B52EE240D12BBBBFC7D00B1
:10BB9000850B0A8E828F83A3E0F8E50828F8E43548
:10BBA00009F9E8250AFAE439FB123DFD7403122B6A
:10BBB00084AA08AB0902BED1EE241712B68422F87B
:10BBC000E43FF988828983E022E0F50C750D0022BC
:10BBD000F582E43FF58312BBF6A3A3A322F0050A86
:10BBE0008E828F83A3A3A3A3A3A3A3A322A3A312A1
:10BBF000E00712BBF62212C0F3A3A32274F41225AD
:10BC00008474FD122C188A088B09ECFEEDFF740178
:10BC1000122BEA880A890B780A122B567402122B0F
:10BC2000FAEEFAEFFB1232217402122B84E97057FC
:10BC3000851882851983E0850882850983F074015F
:10BC4000122E2DE0F812BC90A3A312BC9E60291402
:10BC5000850882850983A312BC9A12D770740112D9
:10BC60002E2DE028F8A3E039F9E824FEF582E93426
:10BC7000FFF58312EA04800C850882850983A3E41A
:10BC8000F0EEFAEFFB80047AFE7BFF74030298BCAF
:10BC9000A3E0F98508828509832212BCA622E8F078
:10BCA000A3E912BCA62212BCAA2212A534E0227477
:10BCB000EE1225848A0A8B0BECFEEDFF750F01E96D
:10BCC000C39408500302BE368E828F83E912AEE71A
:10BCD00012C11A123419E96003750F0012C0FC8EEC
:10BCE000828F8312C14CEE12B7913F12C136C0E071
:10BCF000EE2411F582E43FF583D0E012C12EC0E0BE
:10BD0000EE2412F582E43FF583D0E012B6B6740853
:10BD100012BEC1A3A3A3E06018E50A2408F8E43525
:10BD20000BF912CAD912C8F98E828F83A3E02408B6
:10BD3000F08E828F83A3A3A3A3A3A3A3A3E0601C7D
:10BD40008E828F83A385820885830912C10FEE241A
:10BD50001512E2BBA3E912CBEA2408F08E828F838E
:10BD6000A3A3A3A3A3E0600F12BEA88E828F83A318
:10BD7000A3A3A3A312BEC8EE241912C9ECEE241B80
:10BD800012C9ECA3F0EE241812BBBB700302BE264E
:10BD900012BEA8FAEE2419F582E43FF583EA12BE3A
:10BDA000C8F8E50A28F582E412E2B2F812CBEEE810
:10BDB00012BEC8E8C39AEE5068241912BBBBF890B3
:10BDC000526FE493C398500575110C8008EE241946
:10BDD00012BBBBF5118E828F83A3E0F8E50A28F52C
:10BDE0000CE4350BF50D750E00780C122B52AC11CE
:10BDF000EC2CFCE433FD7A597B0F123DFD740312E9
:10BE00002B84EE241BF582E43FF5837459F0A37470
:10BE10000FF0E511C333F8850882850983E0288097
:10BE20000412C9E5E4F08E828F83A3E0F88E828F3E
:10BE300083E0C398500479008062A3E0FAE50A2801
:10BE4000F8E4350BF9EE241D12E2BBA3E912C1455B
:10BE5000C39AC0E012BE9ED0E012C8E4603CEE245B
:10BE600017F8E43FF9880889098882F583E024F20D
:10BE7000F0EE241D12BBBF240EFAA3E03400FB88B1
:10BE800082898312DA8B90053FE0F9122F5DE9F881
:10BE9000850882850983E0C398F0A90F8033EE24DA
:10BEA00017F582E43FF583228E828F83A385820873
:10BEB000858309E0F8E50A28F582E4350BF583E08F
:10BEC0002212B6BAA3A3A32212CBF804F022122B9B
:10BED000847F0A02280974F41225848A088B09EAEF
:10BEE00012BF5DF0EA1313543F12BF56A3A3A3F091
:10BEF000EAC4131312BF5DA3A3F0EB12BF6812BF15
:10BF0000707409780A122DB812BF6612BF6F740AD6
:10BF1000780A122DB8E50A5401C0E0EC2418F58225
:10BF2000E43DF583D0E012BF75740B780A122DB88A
:10BF300012BF66A312BF6F740C780A122DB812BF1D
:10BF400066A3A3A3A3A3A3A3A3F0740D7808122D43
:10BF5000B8A9080298BF540F8C828D832254038C99
:10BF6000828D83A3A322E50A54018C828D8322A3B0
:10BF7000A3A3A3A3A3F08A0A8B0B22C082C0837958
:10BF8000008A828B83A3A3A3A3A3A3E090053E60B2
:10BF90000EE070228A828B83A3A3E070198016E0E2
:10BFA00060148A828B8312D38E900547E06A7003F7
:10BFB000A3E06B60010902C1BC74F01225848A0AF7
:10BFC0008B0B890C8C088D098A828B8312C11A1203
:10BFD000341912C0FC85088285098312C14CE5081A
:10BFE00012B791350912C136C0E0E508241112C814
:10BFF000DCD0E012C12EC0E0E508241212C8DCD06B
:10C00000E012EEA2740812C128E0601EE50A2408BE
:10C01000F8E4350BF9E508241312C8DC12C8F985D9
:10C020000882850983A3E02408F0850882850983B6
:10C03000A3A3A3A3A3A3A3A3E0601B8508828509F0
:10C0400083A312C10BE508241512C8DCE8F0A3E9AC
:10C0500012C1452408F0850882850983A3A3A3A300
:10C06000A3E06019850882850983A3AE82AF83129D
:10C07000BEB385088285098312C14004F0AA08ABCB
:10C080000912341FE9F50D7061850882850983A3C3
:10C09000A3A3A3A3A312C0EF701AE0FAE50A2AF83B
:10C0A000E4350BF9E508241D12C8DC12C8F9E50CCB
:10C0B000C39A802A12C10BE8240EF8500109E50842
:10C0C000241D12C8DC12C8F990053FE0F9122F5D5B
:10C0D0008E828F83E0F8E50CC39824F2C399C0E008
:10C0E000E508241712C8DCD0E0F0A90D02C18412C3
:10C0F000C0F322E0850882850983A322850A828510
:10C100000B83A3A312C162E0F9EA22AE82AF83E0FF
:10C11000F8E50A28F8E4350BF922E0FAA3E0F8E4A0
:10C12000C8F9EA28E439FB2212EE85A3A32212C142
:10C1300075A3A3A3E022F583E812C16EA3A3E022B6
:10C14000A3A3A3A3A3F08E828F83E022A3A3A3A320
:10C15000A3A3A3A3A312C16E12C162A3A3E0F9EA31
:10C16000F822E0FA850A82850B83A3A3A322F0A319
:10C17000E912C17522F0850A82850B83A3A3A3A3CC
:10C1800022122B847F08022809C082C0837AC57BD3
:10C190000579E2124A877AC57B058020C082C08378
:10C1A0009005478014C082C08390054A800BC082EE
:10C1B000C083794A124A87800312D397D083D082F2
:10C1C000022B3674F61225849005CDE0FE04F0EEC5
:10C1D000F91233BF8B09EA450970EDEE60EAF90206
:10C1E000C53074EE122584EAFEEBFF8C0E8D0F89AC
:10C1F0000A750B00750C001235BD8A088B09741284
:10C20000122E2DE0F5107413122E2DE0F50DEA45D7
:10C21000097017E50D600302C306A90AAC0EAD0F45
:10C22000EEFAEFFB1235E102C414E50D700302C211
:10C23000CC90099AE060046401700E9005DA12CB8C
:10C24000DD600612C64712276AE510700B8508826A
:10C25000850983E4F002C30190099AE06007640154
:10C26000600302C329900541E0A2E1400302C32913
:10C270009005DC12CBDD600CA910AA08AB0912C630
:10C280004712276A850882850983E0FA12E2CE50B8
:10C290000109C3EA98E499A2D265D0335009850810
:10C2A00082850983E004F0850882850983E0F8909F
:10C2B0005286E493687072750B01EEFAEFFB12324E
:10C2C000B1850882850983A3E4F0805DE5107021C3
:10C2D000EA2402F582E412DF21850A0E250EF8E435
:10C2E000340013E813F070098A828B83A3A37401CE
:10C2F000F08A828B83A3A3E0F890114DE0C398509D
:10C3000028750C0180237401650D701DE5106019FE
:10C3100090099AE060046401700F900541E0A2E189
:10C320005007EEFAEFFB1232B190099AE064026016
:10C330000FE060046401702A900541E0A2E1402210
:10C340007401650D701CE5109005EC6013E004F0BD
:10C35000901120E0F89005ECE0C3984005750B01C2
:10C36000E4F0E50CA2E092F0E50BA2E072F04003ED
:10C3700002C41490099AE060046401704190054180
:10C38000E0A2E15039EEFAEFFB12301D8A088B096A
:10C39000A808A909E8496026E50CA2E0500D8882AA
:10C3A0008983A3A3A3A3A3E0C2E0F0E50BA2E0501E
:10C3B0006388828983A3A3A3A3A3E0D2E0F0E50B63
:10C3C000A2E0505090099AE060046401701D90054D
:10C3D00041E0A2E15015EEFAEFFB12300BE9600BE1
:10C3E000EEFAEFFB7900123155802990054AE06E94
:10C3F0007003A3E06F701DEEFAEFFB790112315567
:10C4000090099AE06402700C7A017B009005A1E02B
:10C41000F9123F9502BED174F412258474016A4B5F
:10C42000700E7A017B009005A1E0F9123E6380371F
:10C4300090111712DA8BEA4B60218A088B09E4F518
:10C440000AF50B7808122B4E7A017B009005A1E0CB
:10C45000F9123F897404122B84800C7A017B0090BE
:10C4600005A1E0F9123F950298BFC082C0839011E8
:10C470001902AAC9C082C08390111B02AAC974F60E
:10C480001225847508337509057808122B567C6EC1
:10C490007D007A217B00123F3B7402122B84E9F568
:10C4A00008122F93E9420890099AE0600464017031
:10C4B00006123047E9420890071012CBDD600912DE
:10C4C000C64712276AE94208122ED3E9FE12446FCA
:10C4D000E9F8E5084E48F9805774F61225841248A9
:10C4E000DD7508337509057808122B5675086E75C9
:10C4F00009007808122B567C007D007A217B0012FF
:10C500003F477404122B84122F9990099AE060041B
:10C510006401700312304D90071212CBDD600612D9
:10C52000C64712276A122ED91244818003122B8427
:10C530007F0202280974F612258474FF122C187EDB
:10C54000007508337509057808122B567C6E7D003E
:10C550007A217B00123F3B7402122B84E9600302B4
:10C56000C6187808122B5675086E8E097808122B9B
:10C57000567C007D007A217B00123F4D7404122B03
:10C5800084E9600302C618900547E064FE7003A3C7
:10C59000E0F4700302C6180E900556E064086005CA
:10C5A000E06404706F851882851983EE12CA43799E
:10C5B00042124A8D7A5E7B057943124A8D7A5B7B03
:10C5C000057947124A8D7A4C7B05794A124A8D7A51
:10C5D0004A7B05794B124A8D7A547B057950124A71
:10C5E0008D7A477B057953124A8D7A5C7B057954A5
:10C5F000124A8D7A497B0579E1124A8D900541E016
:10C60000A2E35004D2F08002C2F012CA3979521269
:10C610004A8D80041248DD1E122F9F90099AE06017
:10C62000046401700312305F90071412CBDD6006C2
:10C6300012C64712276A122EE5EEF9740102C52DC3
:10C640008E828F83E0F8A3E0F58388822274F6124D
:10C650002584E9FEA2E0502675083375090578089F
:10C66000122B5675086E7509007808122B567C003F
:10C670007D007A217B00123F477404122B84EEA2C6
:10C68000E35003122FA590099AE06004640170083A
:10C69000EEA2E15003123065EEA2E2500E900716B2
:10C6A00012CBDD600612C64712276A02C53074F647
:10C6B00012258474EC122C187401122BFA9010C4F9
:10C6C000E0F97AA47B05123371900593E06402705F
:10C6D0007C7405122E2DE4F07407122E2DE4F07AEE
:10C6E00004F9122FF98A08905273E493FAC3E5080B
:10C6F0009AEB9400400302C783122FEDE960030216
:10C70000C78390526512C7DF60157A047903122F30
:10C71000F9905273E493FC90526512C7E950087483
:10C7200005122E2D7401F090526312C7DF60157A46
:10C73000027901122FF9905273E493FC9052631224
:10C74000C7E9503F7407122E2D7401803590055FA4
:10C75000122E0AE8494A4B600474018001E4C0E0EB
:10C760007405122E2DD0E0F0900563122E0AE849D0
:10C770004A4B600474018001E4C0E07407122E2D5E
:10C78000D0E0F09010C4E0F97CA47D057401122B78
:10C79000F212336B7AA47B057945124A8D74071225
:10C7A0002E2DE070117405122E2DE070098518826F
:10C7B000851983E480088518828519837401F090B7
:10C7C00010C0E0F89010BFE058F8851882851983F2
:10C7D000E05812CA437941124A8D741402C52DE4FF
:10C7E00093F8740193F9E84922E493F8740193F9FA
:10C7F000ECC398F8E499F9C3EA98EB992274F7121C
:10C80000258474ED122C18E9FE9005A0F0AC18AD4B
:10C81000199010C4E0F97AA47B05123371741212D6
:10C820002E2DEE12C83BAA18AB1912336B7AA47BDB
:10C83000057945124A8D741302B1B0F09010C4E02E
:10C84000F97CA47D052274F4122584EAFEEBFF90A6
:10C8500010C6E064FE7003A3E0F470687A167B00F3
:10C86000123E218A088B09EA450960588A828B8327
:10C87000740112C8E48A828B83A36004740280026C
:10C88000740112C8FFA3E08A828B83A3A3A3A3A38E
:10C89000A3A3A3A312C915FCA3E0FDEA2402FAE4B2
:10C8A0003509FB124901E508241312C8DCE4F0AA9B
:10C8B00008AB099005A1E0F9123E2D12C8C712D1AC
:10C8C0004812C8F90298BF12C8CB22EE240BF58299
:10C8D000E43FF58322850A0CE508250CF582E43552
:10C8E00009F5832212C8E9E022F08E828F83A3A388
:10C8F000A3A3A3A322E01297D9E8F0A3E9F022F0C2
:10C90000EE241DF582E43FF58312C90D2212D15D9C
:10C91000F583888222A3F0EE241512B6842274F2E5
:10C9200012258474FD122C188A088B09890A8C0B35
:10C930007401122E2D740412CA431234AF8A0C8B68
:10C940000DAE0CAF0DEE4F700302C9DAEE12B791C7
:10C950003F12CA097407F0A3A882A983E50824132B
:10C96000FAE43509FB8A828B8312CA1A8A828B8386
:10C9700012CA19E50812D38412DF21888289831232
:10C98000CA257401F0E508240BF8E43509F9EE1224
:10C99000C9E512CA3212EE2212342B12DA82EE24C8
:10C9A0001312EE247403650A60067401650A7007A9
:10C9B00012C9F57404800412C9F5E4F09010C6128F
:10C9C000AD5B12C8F97401650B7006EE241112C933
:10C9D000ECEEFAEFFB123095800279109010C6123F
:10C9E0009BB002D16412EE6E22EE2412F582E43F77
:10C9F000F583E4F02212C9FD7440F0A322EE12DFA9
:10CA0000133FF5832212EE483BF58312CA0F22E052
:10CA1000F8A3E0F98882898322A3E088828983F0E1
:10CA2000A308A98322F0EE2416F582E43FF58322C1
:10CA3000A3A3E8F0A3E9F0EE22A2F0E43385188284
:10CA4000851983F0AA18AB192274F4122584EAFE22
:10CA5000EBFF7A007B049005A1E0F9123F9512CA22
:10CA6000E712C8F99005567409F012342B8A088B26
:10CA700009AC08AD0912CAD912D3971248FBE96470
:10CA80000170537A0F7B00123E218A088B09EA4518
:10CA90000960438A828B837402F012CAF1FC888297
:10CAA0008983A3A3E0FBEC8A82850983A3A312DA1E
:10CAB0008C88828983A3A3A3E08A8285098312C913
:10CAC00015FAA3E0FB794A124A8DAA08AB09900532
:10CAD000A1E0F9123E2D0298BF12CADD22EE241306
:10CAE000F582E43FF5832290051912D15890111B6D
:10CAF00022EE241DF582E43FF58312CDC2E02274BC
:10CB0000F412258474FD122C188A088B0974011202
:10CB10002E2D740212CA431234AF8A0A8B0BAE0A4E
:10CB2000AF0BEE4F700302CBC912EE8D70088882F6
:10CB30008983A37420F0850882850983A3A3A3A316
:10CB4000A3E06401700988828983A3E0D2E6F085BE
:10CB50000882850983A3A3A3A3A3A3E06401700AA9
:10CB600088828983A3E0D2E7800312EE0412EE7E6E
:10CB70007019850882850983A3A312CBDD6006EEB8
:10CB8000241612EE2412EE6012C8F9850882850977
:10CB900083A3A3A3A3A3A3A3E06401700312EE35B0
:10CBA00085088285098312D3971234CDE960031278
:10CBB000EE2E12EE2112342B12CBE312CBCF12CA7F
:10CBC00030FAEFFB1230958002791002BC8BE0F84E
:10CBD000A3E0F98E828F832212B2A4F58312D1587A
:10CBE000E8492212CBEEEAF0A3EB12CBF822EE24B6
:10CBF0001AF582E43FF58322F0850882850983E0F7
:10CC00002274F512258474F3122C18890AEAFEEBBB
:10CC1000FF7508007509007C0D7D007900AA18AB2E
:10CC200019123E09EE12D7783FF58312CDAE741F6C
:10CC300058600C7AD37B001244E1790002CD00E801
:10CC4000A2E55008740C122E2D7401F0E8A2E750F2
:10CC500008740B122E2D7401F0E8A2E6740A500835
:10CC6000122E2D7401F08008122E2DE06401701335
:10CC70008E828F83A3A3A3A3A3A3A3E06032EE2499
:10CC80001380128E828F83A3A3A3A3A3A3A3A3E0E5
:10CC9000601EEE2415F582E43FF58312A72560108F
:10CCA000AC08AD097402122E2DAA82AB8312490181
:10CCB00012C8C712C8F5740A122E2DE0640170372D
:10CCC00012D38A1234CDE97035EE240B12B90A90D2
:10CCD000054AE0687003A3E0697023E50845096030
:10CCE0001612342BEAFCEBFD7402122E2DAA82AB35
:10CCF000831248FBE96007AA18AB1912314FA90A41
:10CD000002EF9574F712258474D2122C18EAFEEB08
:10CD1000FF8E828F83129D51A2E0400302CDA912A3
:10CD2000CDB5E054FE12E6DC740D122BFA12CDD212
:10CD3000123425E97073742A122E2D12CDCC70692D
:10CD40007C0D7D007900AA18AB19123E09741612E9
:10CD50002E2D12C8F5742A122E2D12CDAEA2E5503A
:10CD600008740B122E2D7401F0E8A2E75008740A23
:10CD7000122E2D7401F0E8A2E65004742080027493
:10CD800022122E2D12B0B87402122E2DAA82AB835D
:10CD90001249018E828F83A3A3E0C0E0740C122E8F
:10CDA0002DD0E012CA43123149742E02B1B012C91B
:10CDB0000DA3E0F8228E828F8312CDC2A3A3A3A37A
:10CDC000A32212D15DF988828983A32212B28364DF
:10CDD0000422EA241EF582E43BF583E0F9EA241FED
:10CDE000F582E43B1298B322E9F879007404686094
:10CDF0000A740A686005740368700109022B3674AE
:10CE0000F61225848A828B837420F0A3A37401F028
:10CE100012309B8A088B09AE08AF09EE4F60168E60
:10CE2000828F837401F0900594E0700912EE211254
:10CE3000342B12DA82EEFAEFFB02C530C082C083D7
:10CE400090054402AA68C082C0839010C502AA68F7
:10CE5000C082C083E99010C502AACDC082C0839071
:10CE600005B97401F0E9A2E350037403F0E9A2E10B
:10CE70005004E0D2E2F002C1BC74F61225847900BD
:10CE80007C008A088B09780812284FF8FF07AACE81
:10CE9000A8CEA8CEA8CEA8CEA0CEA4CEAACEA5CEEF
:10CEA0007C0480060C0C80027C089005B9E05C6074
:10CEB00003098003EC60010902C53074F412258473
:10CEC000EAFEEBFF89081230238A0A8B0BA80AA915
:10CED0000BE849604188828983A3A3A3A3E060365D
:10CEE000C39405503174016508601A88828983A350
:10CEF000A3A3A3E06401600D88828983A3A3A3A3F5
:10CF0000E06402700A8882898312A80212276AEEFE
:10CF1000FAEFFB12302F0298BF74F61225848A8232
:10CF20008B83E07012A312CBDD600C8A828B83129C
:10CF3000D396124C2580047A007B0002C530C08253
:10CF4000C083900593E06402700B900556E064087E
:10CF500070031234F102C1BCC082C0837C00EC12A9
:10CF6000D00B7003A3E06B7011905276E493C0E095
:10CF700012CFDAD0E0F079C580510CECC3940340B5
:10CF8000DD7C00EC75F003A4F8A9F074BD28F582EF
:10CF9000740512979C64FE7003A3E0F4600F0CEC20
:10CFA000C3940340DE7C00EC12CFCE7015EC12E38C
:10CFB0007512DA8B905276E49388828983F0790037
:10CFC00080090CECC3940340DE79C702C1BC75F044
:10CFD00003A4F8A9F012CFDAE02274BC28F5827419
:10CFE0000539F58322C082C0837D00ED12D00B701D
:10CFF00003A3E06B700912CFD56004790180090D9D
:10D00000EDC3940340E5790002C1BC75F003A4F8B8
:10D01000A9F074BD28F582740512E82E6A2274F214
:10D0200012258474DD122C18EAFEEBFF750A0090BD
:10D03000099AE060076401600302D142900547E06D
:10D040006E7003A3E06F701EEE4F700302D1369036
:10D0500005CE12CBDD700302D136750A0112C64728
:10D0600012276A02D14212301D8A088B09EA45094B
:10D07000700302D1368A828B83A3A3A3A3E0640149
:10D0800060108A828B83A3A3A3A3E06402600302DF
:10D09000D136851882851983E412D14F740B122E74
:10D0A0002DE8F0A3E912CA43122FE1E9700302D17F
:10D0B0003685088285098312D14812C8F979001291
:10D0C00031FD85088285098312DA8B7403122E2DB7
:10D0D000AC82AD837418122E2DAA82AB8312490143
:10D0E00085088285098312B9107420122E2D12C86A
:10D0F000F97422122E2DE4F07C02850882850983C2
:10D10000A3A3A3A3E0F9740D122BF212348B8508AC
:10D110008285098312B9107401122E2DE8F0A3E95B
:10D1200012CA43122FE7750A01E508240C12C8DC65
:10D130001297FDF0800C90055412B6A2FAEFFB1284
:10D1400035A5A90A7423801E12D1589010C6221248
:10D15000AEEB12D15622A3A312D15DF922E0F8A3BF
:10D16000E022A90A7403122B847F06022809C082D8
:10D17000C08374FE122C1890099AE0600464017058
:10D1800029790190052C12C64412276A12D1AF905A
:10D190000547E8F0A3E912CA437953124A8D85186E
:10D1A0008285198312D3971240C7740202850385C2
:10D1B0001882851983EAF0A3EB12D1BEF92212BCC2
:10D1C000AAF8A3E02274F512258474F3122C188AAD
:10D1D000088B09ECFEEDFF750A12EA450970057926
:10D1E0000002D2D2900547E065087004A3E065090B
:10D1F000701912342BEAFCEBFDEEFAEFFB1248FB40
:10D20000E97005750A018003750A00851882851981
:10D2100083E4F004122E2DE508F0A3E50912CA43B9
:10D22000122FD5E960297403122E2DAA82AB831226
:10D230002FB1E964017018750A017403122E2DAC28
:10D2400082AD83EEFAEFFB1248FBE9701E801F747B
:10D2500012650A7019900593E064027011EEFCEFFC
:10D26000FDAA08AB09123005E96003750A00EEFC5F
:10D27000EFFDAA08AB091235C3E9F8740A68700516
:10D28000750A01804274A0687037EEFCEFFDAA08B1
:10D29000AB091235D57E008023EE75F017A4F8A9EE
:10D2A000F012E8447004A3E06509700F12E98012DF
:10D2B0002FB1E9700612E51F1235B10E12D2D5401A
:10D2C000D87401650A70097900AA08AB0912350300
:10D2D000A90A02EF9590526EE493F8EEC398227477
:10D2E000F6122584EAFEEBFF890890099AE06004B3
:10D2F0006401701E1234F1E508F5097809122B5A01
:10D30000790DEEFCEFFD7AFC7BFF12350F740112F4
:10D310002B8402C53074F7122584EAFEEBFF8E825F
:10D320008F83A3A3A3A3A3A3A3A3E0601312D37C1F
:10D330001298A61234FDE96401700512C8C7802D49
:10D340008E828F83A3A3A3A3A3A3A3E0602912CA01
:10D35000D912D39BFAA3E0FB1234FDE964017017E4
:10D360008E828F83A3A3A3A3A3A3A3A3A312D39764
:10D370001234E579018002790002B1B3EE12D38450
:10D380003FF583222415F582E4228E828F83A3A3A6
:10D39000A3A3A3A3A3A3A31298B52212D3A7A3A3C5
:10D3A000A3A3A3A3A3E02212B0C08E828F83A3A362
:10D3B0002274F212258474FD122C188A088B09EC51
:10D3C000FEEDFF890B750A017401122E2D740412F3
:10D3D000CA431234AFEA4B60477411122E2DE0603D
:10D3E0001AEA2417F582E43BF583E412DC378A82DB
:10D3F0008B83E0D2E7F012D423E4F012CA05740361
:10D4000012D691EE88828983A3A3F0EF8882898364
:10D41000A3A312AEE6A3A312F072123095E9F50AA7
:10D4200002D162EA2414F582E43BF5832274F012FF
:10D430002584EAFEEBFF890A750B0112CAF1F50C8F
:10D4400088828983A3A3E0FA8882898312D56A122D
:10D45000BBB86404600A7AD37B001244E102D5654C
:10D46000E50C122A1A0200027AD4030B1AD5030C17
:10D4700001D50DD9D40E1AD518D590099AE06007B8
:10D480006401600302D51A900541E0A2E140030265
:10D49000D51A7900AB09123293EA4B60318A828B3C
:10D4A00083A3A3A3A3A3A3E05418602212C8C712A6
:10D4B00029958A828B83A3A312299579008E828F66
:10D4C0008312D5891232AB7404122B84802E790119
:10D4D000AA08AB09123161804190099AE0600464A6
:10D4E000017037900541E0A2E1502FAB091234DF03
:10D4F000AA08AB091234E5E964C5701E750B0080FB
:10D500001990099AE060046401700F900541E0A24F
:10D51000E150071240EB8002880AEE2409F50EE480
:10D520003FF50FAC08AD09A90C850E82F58312D327
:10D5300097123179850E82850F8312D3971234CDDD
:10D54000E96022EE241112BBBBC39402401712C83B
:10D55000C712DB517003A3E069600AE50BA2E0503B
:10D5600004A90A8002790002C184A3A3A3E0F8E41D
:10D57000C8F9EA28F508E439F50922E508240CF58C
:10D5800082E43509F58312B660A3A3A3A3A3A3A3E2
:10D59000A3A312B0BC8A828B831298B52274EE12B8
:10D5A000258474F5122C188A0A8B0B890C8C0E8D2D
:10D5B0000F7E01EE122E2D740AF0741D122E2DE036
:10D5C000F50DE9700FE50DC333240AC0E0EE122E0D
:10D5D0002DD0E0F0AA18AB191234AF8A088B09EAF3
:10D5E0004509700302D68612B790350912D8137414
:10D5F0000912D81F450D12D6B1AC0EAD0FEEFAEFE1
:10D60000FB124901EE2408FE50010FE50C70247C4A
:10D6100000741E122E2D12B9108012EC12DB3DE8A0
:10D620002AFAE93BFB12D697A30EAF830CECC39505
:10D630000D40E8E508241712C8DC7401F012342B01
:10D64000E508241AF582E4350912DA897403122BED
:10D65000FAAA0AAB0B122FBDE96019E508241612CD
:10D66000C8DC7401F07403122BEAE508241812C810
:10D67000DC12C8F985088285098312D68DAA08AB09
:10D6800009123095E9FEEEF9740B02BECEA3A3E5B4
:10D690000AF0A3E50BF0228A828B8312D6AB12D656
:10D6A000B18A828B8312D6AAF022A3E08E828F8366
:10D6B00022F0A3AE82AF832274F012258474F81294
:10D6C0002C188A088B0912D777350912D898F50BD0
:10D6D000880AA3AE82AF83EEFCEFFDAA18AB191245
:10D6E0004901EE2408FE50010FAC18AD197A687B91
:10D6F000051248FBE9607474E0550A7067AA0BEAEA
:10D700002AFA7B00123EC38A0C8B0DEA450D605B42
:10D710007C00801E8E828F8312C11AEC12D770E5B6
:10D720000C28F582E50D3912DA89EE2402FE50014B
:10D730000F0CECC3950B40DC780C122B56780B12B7
:10D740002B5A7403122BFA7900E508240B12C8DC5B
:10D7500012D3971235277403122B84AA0CAB0D1227
:10D760003EC980077AD37B001244E1740802C1816C
:10D7700025E0F8E433F922EA241DF582E42274F06E
:10D780001225848A0A8B0B890C8C088D099007E579
:10D7900012CBDD607B7410122E2DE0F50D12D770C8
:10D7A000E8240EFAE439FB123E218A0E8B0FAE0EEE
:10D7B000AF0FEE4F605A8E828F8374D4F0A3A3E52F
:10D7C0000AF0A3E50B12BEC1E50CF0AC08AD09EE02
:10D7D0002405FAE43FFB12490112B297E50DF074FB
:10D7E00011122E2D12DC217808122B52AC0DEC2CCC
:10D7F000FCE433FDEE240EFAE43FFB123DFD74031E
:10D80000122B84EEFAEFFB9007E512C64412276A4A
:10D8100002C184F583E0FEA3E0FF8E828F8322F0B5
:10D82000A3E50CC43354E02274F612258474F81274
:10D830002C18890812D7773B12D898F98809A3AE1B
:10D8400082AF837401697042EEFCEFFDAA18AB1938
:10D85000124901EE2408FE50010FAC18AD197A6888
:10D860007B051248FBE9602974E05509701C8E8223
:10D870008F83A3E0FA8E828F83A312C11C8E828FC6
:10D8800083E0F912353FA90880097AD37B0012445E
:10D89000E17900740802C52DF583E02401FEA3E0C0
:10D8A0003400FF8E828F83E0F8741F582274F612C2
:10D8B000258474DF122C18EAFEEBFF12CBD86050DF
:10D8C0008E828F8312D397AC18AD1912CDD2123439
:10D8D000137409122E2D12DB517003A3E06960301E
:10D8E00012C6401229957508FE7509FF7808122B9B
:10D8F00056741C122E2DE0F9740D122E2D12B0B894
:10D90000740F122E2D12D3971232AB7404122B8483
:10D91000742102C52D74F7122584E9FC7A007B007E
:10D920007E00800B12D9B7E02AFAA3E03BFB0E90F1
:10D93000527312D2D85029EE75F016A4F8ADF0ED5E
:10D94000F912E833F460E774CB28F582740A3912CF
:10D95000CBDB60DAEC60CD12D9B7E4F0A3F080CE77
:10D960007E00800B12D9A4E02AFAA3E03BFB0E1242
:10D97000D2D5502DEE75F017A4F8ADF0EDF912E9FF
:10D98000917003A3E0F460E6749E28F582740C396C
:10D9900012CBDB60D9EC60CC12D9A4E4F0A3F08008
:10D9A000CD02B1B3EE75F017A4F8EDF9749E28F529
:10D9B00082740C39F58322EE75F016A4F8EDF97433
:10D9C000CB28F582740A39F5832274EC12258489F8
:10D9D0000CEAFEEBFF9005A0E0C3950C503B12341F
:10D9E0007F9005D012DA7C90053AE0F508E4F5095D
:10D9F000F50AF50B9081607810122DD67808791011
:10DA000012241F7808122B4E7A007B029005A1E0A9
:10DA1000F9123F897404122B8402979474F612252C
:10DA200084EAFEEBFF9005BA801388828983E06E5A
:10DA30007003A3E06F603688828983A3A312CBDDD5
:10DA400070E87A047B00123EC38A088B09A808A9F3
:10DA500009E84960188882898312DA7C9005BA1235
:10DA6000DA70A3A312DA8B9005BA12C8F902C53096
:10DA70001298B588828983228A828B83EEF0A3EF85
:10DA8000F022EE241AF582E43FF583EAF0A3EBF0EE
:10DA90002274F41225847E009005BA80070E8882D5
:10DAA0008983A3A312CBDD70F4EE12DB3D123EC3DB
:10DAB0008A088B09EA4509607E7F009005BA8021BB
:10DAC0008882898312B0B8EF12DB3DE5082AF5821F
:10DAD000E5093BF583ECF0A3EDF00F88828983A381
:10DAE000A312CBDD70DA90059C12DB517003A3E02A
:10DAF000697808701C122B56EEF50A780A122B5A18
:10DB00007C687D05790090059C12D397123527809B
:10DB10001A122B56EEF50A780A122B5A7C687D05EC
:10DB2000790090059C12D39712351B7403122B8435
:10DB3000AA08AB09123EC91230AD0298BF25E0FA1F
:10DB4000E433FB228E828F83A3A3A3A3A3A3A3A367
:10DB5000A312D158900547E06822C082C08380128A
:10DB60008A828B83A3A312B9109005BA12C8F91246
:10DB70003EC99005BA12B05B70E602C1BC74F512E2
:10DB8000258490055412B9179005D012DC1512C8DF
:10DB9000F97AD07B057950124A8D9005D012DC219C
:10DBA000801512E3D365087004A3E06509600612CE
:10DBB000E5271235B1050A12DC0A5018E50A12E50C
:10DBC000137003A3E06F70DA749328F582740C125B
:10DBD000F06F80E19005D012B9179007E712CBDD06
:10DBE00060257A067B00123E21EA4B601A8A828BFE
:10DBF0008374D5F0A3A3E412DC280412DC37900769
:10DC0000E712C64412276A02EF9A90526EE493F824
:10DC1000E50AC3982212DC192212D15DF99005544D
:10DC20002212AD42750A002212DC2C2212DC3022B4
:10DC300012AEEBA3A3A32212DC2CA3EEF0A3EFF011
:10DC400022C082C0839005D27469F0A37435F0902D
:10DC500005D47463F0A37435F09005D67481F0A3F5
:10DC6000743502AACDC082C083900547E064FE707F
:10DC700003A3E0F4600E900541E0A2E150061235E6
:10DC8000C912356F02C1BC74F0122584900595E06D
:10DC90006053F50CE4F50DF50EF50F908100780852
:10DCA000122DD6780C790812241F123E1B8A088B7D
:10DCB00009A808A90990525FE49358F508A3E493D2
:10DCC00059F509E4F50AF50B780C7908122D0B7853
:10DCD0000C122B4E7A007B019005A1E0F9123F8FC8
:10DCE0007404122B8402C18474EE1225847E007F9A
:10DCF000008E0A8E0B1230718E0D803E850D08AAA3
:10DD0000087B0012306B8A088B09A808A909E8492A
:10DD1000602688828983A3A3A3A3E06004640470BF
:10DD20001788828983A3A3A3A3A3A3A3A3A3A3E088
:10DD3000F91235DBE960010F050D905273E493F899
:10DD4000E50DC39840B612359F8A0E8B0F8E0C805E
:10DD500023AA087B001235AB8A088B09A808A909F9
:10DD6000E849600EE8240F129799F91235DBE96053
:10DD7000010E050C850C08C3E508950EE4950F40CF
:10DD8000D0EF2EFE700302DE818E0875090074024A
:10DD90007808122D44AA08AB09123EC38A0A8B0BDD
:10DDA000EA450B700302DE7F750C008E08750900D2
:10DDB00074027808122D44AC08AD0979FF123E09AF
:10DDC000750D00805D850D08AA087B0012306B8AF6
:10DDD000088B09EA450960488A828B83A3A3A3A321
:10DDE000E06004640470398A828B83A3A3A3A3A395
:10DDF000A3A3A3A3A3E0F91235DBE96023050C7804
:10DE00000A122B56EEFD850882850983A3A3A3A3DE
:10DE1000A3A3A3A3A312DF271235757402122B84C8
:10DE2000050D905273E493F8E50DC3985006E50C88
:10DE3000C39F4091750C00850C08C3E508950EE45E
:10DE4000950F503DAA087B001235AB8A088B09EA72
:10DE500045096027EA12DF1312DF21F91235DBE9E9
:10DE60006019780A122B56EEFDE508240E12C8DC64
:10DE700012DF271235757402122B84050C80B87ED0
:10DE800000750E6290053FE0600CF9122F5DE9F815
:10DE90007454C398F50E75F003E50E84F50D9420C7
:10DEA0004003750D1F850A08850B09750C00E50EEA
:10DEB0006006750C20750E00E50DC39E5004AF0D75
:10DEC0008008EEFFE50CD2E6F50CAC08AD09AA0C13
:10DED000EFF912357BE9F50FE50CA2E6401A1F7841
:10DEE00000800BE5082404F5085002050908E8C382
:10DEF0009F40F0EFCEC39EFEE97006E50CA2E6500F
:10DF0000AAE50A450B6007AA0AAB0B123EC9A90F86
:10DF100002BED1240FF582E42274262508F582740E
:10DF2000103509F583E022E0FC850882850983121B
:10DF300098B52274F2122584EAFEEBFF89088C0959
:10DF40008D0A7C007D00740E122E2D12D3978C0B3F
:10DF5000800DEAFCEBFDEA2404FA50010B050BE509
:10DF60000BC3950A400302DFFE8A828B83E0F470C4
:10DF700003A3E0F46077EC4D600C8C828D83C3E0EA
:10DF80009EA3E09F50CC8A828B8312E342EE98EFEF
:10DF90009950BFEAF8EBF988828983E0F47003A313
:10DFA000E0F46010E82404F8500109050BE50BC308
:10DFB000950A40E3E8FCE9FDE824FCF8E934FFF9C0
:10DFC000888289831297EE8C828D83E50CF0A3E51D
:10DFD0000D12E0018C828D83A3A312E6D6E08C8221
:10DFE0008D83A3A3A3F0C3EA98EB9940C712DA7814
:10DFF0008A828B83A3A3E50912DC28E508F002D10D
:10E000006912E007A3E022F088828983A32274F2D8
:10E0100012258474FD122C1889088A09ECFEEDFF84
:10E02000750A0175F003E9A42402C0E07401122E00
:10E030002DD0E012CA431234AFEA4B607812CA0501
:10E040007408F0741F55084509A3F0E82402F8503D
:10E050000109750A0080388E828F83E08882898367
:10E06000F0A3A882A9838E828F8312CA198E828F11
:10E0700083A3A3E05407C4FC8E828F83A3A3A3E0F1
:10E0800054074C12CA1BEE2404FE50010F050AE58A
:10E090000AC3950840C18A828B83A3A374FCF0A3B2
:10E0A00074FFF0EA2413F582E43BF5837401F01267
:10E0B0003095E9F50A02D16274F11225848A0A8B3F
:10E0C0000B7508007AFE7BFF7CFE7DFFE50A12D708
:10E0D00078350B12CAF8F509741F5509F50CE824B8
:10E0E00002F8500109E509A2E7406FE50A2417F597
:10E0F00082E412E2B2FE75F003E50CA424026E7015
:10E1000059E50C600B88828983E0FEA3E0FBEEFA00
:10E11000750D00801DE05407F50EA3A882A983EEBB
:10E12000FC900547E06E7003A3E06F7003850E0856
:10E13000050DE50DC3950C502B88828983E0FEA365
:10E14000E0FCE4CCFDEE2CE43DFFE82402F85001B5
:10E150000988828983E0548860BB7AD37B001244AB
:10E16000E102E2A7E508700BA909123587E97003FF
:10E1700002E2A712E2C412D39712301D8A0C8B0D53
:10E18000AE0CAF0DEE4F605A8E828F83A3A3A3A374
:10E19000A3A3A3E4F090528693F88E828F83A3A367
:10E1A000A3A3A3A3A3A3E0C398402412E2CE5001EB
:10E1B000097A027B00122327E88E828F83A3A3A310
:10E1C000A3A3A3A3A3F0E508C39407500205088EF8
:10E1D000828F83A3A3A3A3A3A3A3A3A3E508F00211
:10E1E000E2A77CFF7DFF12E2C412D3971235938A17
:10E1F0000C8B0DAE0CAF0DEE4F704F1235998A0C93
:10E200008B0DAE0CAF0DEE4F700302E2A77C177DB5
:10E21000007900123E0912E2C412CBCE1284F58EB0
:10E22000828F83A3A3A3A3A3A3A3A312CA3012B66E
:10E230007974AA12E2ED5001097A027B00122327B9
:10E2400012B297E812E2D97401F0905286E493F882
:10E25000EE240D12BBBBC398401912E2CE50010947
:10E260007A027B0012232712E2B8E508C394075014
:10E2700002050812E93FE50812E2DEE4F0129CE62E
:10E28000122FB1E97021850A82850B83A3A3A3A372
:10E29000A3A3A3A3E06010E50A12D384350B12B642
:10E2A000A0129CE712490102A8E37426250AF58210
:10E2B0007410350BF583E022EE240DF582E43FF572
:10E2C00083E8F022E50A12EE49350BF583229052DD
:10E2D00086E49379002401F822F012E94322F01237
:10E2E000E2E322EE240CF582E43FF58322F0905223
:10E2F00086E49379002401F82274F7122584E9FE5C
:10E3000074FE6A700374FF6B603474605E646060F6
:10E310002DEEA2E5401CA2E6900547500DC3E09A01
:10E32000A3E09B5019790002B1B3C3E09AA3E09B2C
:10E3300040F390054712E342EC98ED9940E77901EC
:10E3400080E512D158C32274F71225847E0080071D
:10E3500012E51F1235B10E12D2D540F47E00EE1236
:10E36000E375129BB088828983E4F00EEEC39403B8
:10E3700040EC02B1B375F003A4F8A9F074BC28F81E
:10E38000740539F988828983A32274F71225847F62
:10E390000080010F90526EE493F8EFC398502DEF78
:10E3A00075F017A4F8A9F012E81F6A7003A3E06BD8
:10E3B00070E112E3D36C7003A3E06D600A74FF6C2C
:10E3C000700374FF6D70CC12E52780047A007B0027
:10E3D00002B1B312E3D722749328F582740C12E8C9
:10E3E0002E2274F61225847CFF7DFF7AFE7BFF12BD
:10E3F0003593EA4B703C7508008032E50875F017DC
:10E40000A4F8A9F0749828F582740C12979C600502
:10E4100012E8147016748928FE740C39FF8E828FEE
:10E420008312D3971232B1EEFAEFFB050812E435EE
:10E4300040C902C53090526EE493F8E508C39822B3
:10E44000C082C0837A007B007D00801012E9897051
:10E4500003A3E0F460050AEA70010B0D90526EE42C
:10E4600093F8EDC39840E502C1BC74F41225848A88
:10E47000088B09ECFEEDFF800B1235B1EEFCEFFDD1
:10E48000AA08AB09123593EA4B70EE0298BF74F6F6
:10E490001225847D007E0080020D0E12D2D5501808
:10E4A000EE12E98A7003A3E0F460EF8D08EA6508D4
:10E4B0004B70E612E52780047A007B0002C53074B9
:10E4C000F7122584EAFEEBFFEE4F601A7C177D0001
:10E4D0007900123E098E828F8374FEF0A30412AD80
:10E4E00065A314129BB202B1B374F7122584EAFE3D
:10E4F000EBFF7508008014E50812E5137003A3E034
:10E500006F600612E5271235B1050812E43540E7C1
:10E5100002B1B375F017A4F8A9F012E3D76E22EE9A
:10E5200075F017A4F8A9F0748928FA740C39FB2245
:10E5300074F41225848A088B09ECFEEDFF90099A89
:10E54000E0600464017020900554E06E7003A3E065
:10E550006F701412301D8A0A8B0BA80AA90BE849A8
:10E560006005E82408801AEEFCEFFDAA08AB09124A
:10E5700035938A088B09A808A909E8496009E824A5
:10E580000DFAE439FB80047A007B000298BF74F432
:10E590001225848A0A8B0BECFEEDFF7508007509C5
:10E5A000008034E50912E979122FB1E96027E50905
:10E5B00075F017A4F8A9F012E83E7004A3E0650B0B
:10E5C000700375080AEEFCEFFD12E9801248FBE9C2
:10E5D00060034308A0050990526EE493F8E509C36F
:10E5E000985004E50860BC02BF5174F61225847E81
:10E5F00000805C8E08AA087B0012306B8A088B09A9
:10E60000A808A909E849604688828983A3A3A3A32F
:10E61000E06401603988828983A3A3A3A3E0640234
:10E62000602CE82407129799FA74012AF090059655
:10E63000E0C39A501988828983A3A3A3A3A3A3A3A9
:10E64000A3A3A3E412E6CDA312E6DC1232B10E902E
:10E65000527312D2D8409C7E008059EE75F017A4F8
:10E66000F8AAF0EAF912E9917003A3E0F4604474A7
:10E670008928F8740C39F9E8240C129799F8740178
:10E6800028F0900596E0C3985029EE75F017A4F88D
:10E69000EAF9748928F8740C39F9E812DF1339F5AE
:10E6A00083E4F0E8240EF582E439F583E412E6DC35
:10E6B0001232B10E12D2D540A27B00EB12CFCE6047
:10E6C0000214F00BEBC3940340F102C53012E6D6FE
:10E6D000A3A3A3A3A32212E007A3A32212E6E4FAB2
:10E6E000A3E0FB22F088828983E02274F312258460
:10E6F0008A088B09ECFEEDFF750C007B007C017431
:10E700000D122E2DE0F50AA3E0F50B8010123E1B32
:10E71000E50CF5F0EA84ABF0750C007C007D008020
:10E72000010D90526EE493F8EDC398504912E989B7
:10E730007003A3E0F460EA12E8447004A3E0650902
:10E7400060DF12E81F6E7003A3E06F60D412E83E32
:10E750007004A3E0650B60C912E81460C4C3940799
:10E7600050BFEC050C70BAE50CC39B40B47489280B
:10E77000F582740C80787A0080010A905273E493D9
:10E78000F8EAC3985070EA75F016A4F8A9F012E8F8
:10E790004A64FE7003A3E0F460E012E84A65087082
:10E7A00004A3E0650960D312E84A6E7003A3E06F2A
:10E7B00060C812E84A650A7004A3E0650B60BB7488
:10E7C000C428F582740A12979C60AFC3940750AABC
:10E7D00012E833640160A3E06402609EEC050C70F3
:10E7E00099E50CC39B409374BB28F582740A39F5F4
:10E7F0008312D3978019E50C6011EB700E740165DC
:10E800000C600302E70D7B0102E7187AFE7BFF7FB5
:10E8100005022809749728F582740C12E82E22123A
:10E82000E82322748928F582740C12E82E2239F527
:10E8300083E02274BF28F582740A12E82E2212E8BF
:10E8400023650A2212E82365082274BB28F5827426
:10E850000A12E82E2274F51225848A088B09ECFE30
:10E86000EDFF750A008002050A12DC0A5022EEFC58
:10E87000EFFDE50A12E9791248FBE960EAE50A755D
:10E88000F017A4F8A9F0748928F582740C12F06FBF
:10E8900002EF9AE9F87907C3940D400479018019D1
:10E8A000E8C3940740047903800FE8C3940340044D
:10E8B00019198005E870027900022B3674F01225D0
:10E8C000848A088B098C0A8D0B890C1235998A0E63
:10E8D0008B0FAE0EAF0FEE4F60627C177D0079009C
:10E8E000123E098E828F8312F0728E828F83A3A3D1
:10E8F000A3A3A3A3A3A312D68DE50C600712B67839
:10E90000E50C800512B6787401F09005D412CBDDC9
:10E91000601590059BE06401700612E93FE4800CED
:10E9200012E93F7407800512E93F740112E2ED50CD
:10E9300001097A027B0012232712E2B802C1841275
:10E94000E94322EE240EF582E43FF5832274F712A8
:10E9500025847E00801BEE12E98A7003A3E0F46038
:10E960000F12E980122FB1E9700612E51F1235B1BE
:10E970000E12D2D540E002B1B375F017A4F8A9F099
:10E98000748B28FA740C39FB22ED75F017A4F8A9E2
:10E99000F012E82364FE22C082C0839005D874F38D
:10E9A000F0A37435F09005DA74F9F0A37435F090A3
:10E9B00005DC74FFF0A3743502AACD74F712258428
:10E9C000EAF8EBF990051712EA04CA2406F582E486
:10E9D0003AF583E0702B88828983A3A3A3A3A3A322
:10E9E000A3A3A312299590051712EA09122DFE88F8
:10E9F000828983A3E0F912316D7402122B841230E4
:10EA0000AD02B1B3E0FAA3E02212EA04F5838A82F0
:10EA100022C082C08390059E12EAD4F090059E1217
:10EA2000CBDD7005790112353902C1BC74F61225AF
:10EA30008474FC122C18E9FE905277E493700874E9
:10EA4000E16E600302EACFEA2408F8E43BF9888229
:10EA5000898312EAD412EADD700E90059EE4F0A3D9
:10EA6000F07901123539806790099CE06061FA9075
:10EA7000059E12E342EA98E4995054790012353920
:10EA80008A088B09AC08AD09ECF8EDF9E875F0647B
:10EA9000A4F8AAF075F064E9A42AF990059E12D3AF
:10EAA0009712232FE8941AE9940040239007DF126D
:10EAB000CBDD601B90059E12C8F57402122E2DEC62
:10EAC000F0A3ED12CA439007DF12C64412276A74FE
:10EAD0000402C52DE02401F0A3E034002212E6E494
:10EAE000F8A3E0F9E84922C082C08374F8122C1818
:10EAF00090809AAC18AD197408122AB2AC18AD19EE
:10EB00001248FBE9640170047900800279010285F2
:10EB10000174F6122584740C122E2D12B917743A52
:10EB20006E7001EF6006743B6E4F7023740A122EF4
:10EB30002D1229958C088D097808122B56EAFCEBCA
:10EB4000FDEEFAEFFB123F4D7404122B8480027924
:10EB50000A02C530C082C0839005DE7477F0A374CA
:10EB600030F09005E0747DF0A37430F09005E2740D
:10EB70001DF0A37436F09005E47423F0A37436F00E
:10EB80009005E67429F0A37436F09005E8742FF030
:10EB9000A37436F09005EA7435F0A37436F0741D52
:10EBA0004436600312361D02C1BC74F4122584740D
:10EBB000E9122C188A088B097404122E2D7402F0A5
:10EBC00004122BF21234AF8A0A8B0BAE0AAF0BEE93
:10EBD0004F700302EDF012EE8D700888828983A3D6
:10EBE0007420F0850882850983A3A3A3A3A3E0640E
:10EBF00001700988828983A3E0D2E6F085088285C6
:10EC00000983A3A3A3A3A3A3E06401700A88828954
:10EC100083A3E0D2E7800312EE0412EE7E70198522
:10EC20000882850983A3A312CBDD6006EE241612A9
:10EC3000EE2412EE6012C8F9850882850983A3A329
:10EC4000A3A3A3A3A3E06401700312EE3585088299
:10EC500085098312D3971234CDE9600312EE2E1288
:10EC6000EE2112342B12CBE3FAA3E0FB8E828F83CA
:10EC7000A3A312DA8B1234CDE9600312C9E9EE24A2
:10EC80001312BBBB700D90527BE493C0E012CAD943
:10EC9000D0E0F08E828F83E0A2E750045403801905
:10ECA000EE241412BBBB7012900533E0C0E012EDED
:10ECB000FAD0E0F0900533E004F012EE13701990F2
:10ECC0001128E0600D90053EE0700D8E828F83E08C
:10ECD0007006EE241112C9ECAC18AD19EEFAEFFB78
:10ECE0001234078A088B09EA4509700302EDE47AB9
:10ECF000217B00123EC37406122E2D12DA8B74068D
:10ED0000122E2D12CBDD700302EDD890099AE0602F
:10ED1000046401700812B678A3E04404F074011290
:10ED20002BF27950124A877401122E2D12B91074E9
:10ED300006122E2D12EA04CA2409F582E43AF5835C
:10ED400012C8F990054712B9107415122E2D12C869
:10ED5000F97406122E2D12B90212EE3FF07406124B
:10ED60002E2D12AE37740212EE777406122E2D126B
:10ED7000EA0912BC9EC0E07406122E2D12B90212CE
:10ED8000EE0AD0E0F0EE240E12EE1CC0E074061283
:10ED90002E2D12EE4FD0E0F07406122E2D12868426
:10EDA00012F070EE240F12B90A740C122E2D12C834
:10EDB000F98A828B83E0C0E0740E122E2DD0E0F031
:10EDC0007406122BF2123383E9F50A7406122E2D03
:10EDD00012D397123EC98003750A10AA08AB091214
:10EDE0003EC98003750A10EEFAEFFB123EC980039C
:10EDF000750A10A90A74170298BCEE2414F582E46F
:10EE00003FF5832212CADD740122241EF582E43804
:10EE1000F58322EE241112B68464012212B66BE04F
:10EE200022EE2417F582E43FF5837401F02212B636
:10EE3000814404F02212C9FD7401F0A3E4F022120F
:10EE4000EE4938F583740222EA240BF582E422129B
:10EE5000EE532212D15DC8240CF582E438F58322EA
:10EE600085088285098312D156EE12EE6E2224188F
:10EE7000F582E43FF5832212B6BA12D1572212EE80
:10EE800085E064012212EEA6A3A3A3A32212C8CB9D
:10EE900012CA0F7404F0A3E412EEA2A3A3A3E064C9
:10EEA000012212EEA622F0850882850983A322742E
:10EEB000F61225847E00801F7C047D0079FF8E0879
:10EEC0008D0974027808122D4474262508FA7410EE
:10EED0003509FB123E090E90527D12D2D840D9025C
:10EEE000C53074F512258474F7122C18750A008049
:10EEF0001E850A0875090074027808122D447428CA
:10EF00002508F582741012C8DF12EF88F0050A9008
:10EF1000527D12DC0D506D850A0875090074027867
:10EF200008122D4412DF19F47003A3E0F460DE85AB
:10EF30000A0875090074027808122D4474282508FF
:10EF4000F5827410350912CBDB70A67408122E2DD1
:10EF50007402F0850A087509007808122D44742699
:10EF60002508FE74103509FF8E828F8312C8F512B2
:10EF7000EF91124AD57C047D0079FFEEFAEFFB1287
:10EF80003E0980897409800FE024FFF0A3E034FF7C
:10EF90002212F0FF22740D122B847F0302280974C1
:10EFA000F012258474F7122C18EAFEEBFF8C088D02
:10EFB00009750CFF7408122E2D12F0F1124ACFE9D8
:10EFC000641A700302F06B750E00800B74FF650C01
:10EFD0007003850E0C050E90527DE493F8E50EC388
:10EFE000985048850E0A750B007402780A122D4459
:10EFF00012E2AAF47003A3E0F460D1850E0A750B47
:10F00000007402780A122D4412E2AA6E7003A3E083
:10F010006F70C2750F007402780E122D447428258B
:10F020000EF5827410350FF5838030E493650E7011
:10F030002D74FF650C602E850C0A750B0074027828
:10F040000A122D447426250AF87410350BF98882AB
:10F05000898312DA7C88828983A3A312F0727901F2
:10F06000740902C18112EF91124AD5790080F139F9
:10F07000F583E508F0A3E509F02274F41225847401
:10F08000F7122C18EAFEEBFF7408122E2D12F0F185
:10F09000124AD5750A008002050A90527D12DC0DD5
:10F0A000504C850A0875090074027808122D441224
:10F0B000DF19F47003A3E0F460DE850A0875090027
:10F0C00074027808122D4412DF196E7003A3E06FEA
:10F0D00070C67C047D0079FF8D0B7402780A122DB6
:10F0E000447426250AFA7410350BFB123E0902AE51
:10F0F00027740212A534EEF0A3EFF012F0FF229075
:10F10000055412B0C0AA18AB1922C082C08374F88B
:10F11000122C1885188285198312DA8B7402122E2C
:10F120002DE4F0A3F07404122E2D7401F074051276
:10F130002E2D7401F07406122E2DE4F07407122E99
:10F140002DE412CA4312361702850174EE1225848B
:10F150008A088B09ECFEEDFF750C00EE6508700364
:10F16000EF6509600C123F418A0A8B0BEA450B7070
:10F1700006750C0102F207EEFAEFFB123F418A0E10
:10F180008B0FAC0EAD0FEC4D6007EEFAEFFB123FAC
:10F1900053E4F50EF50F780E122B56AC0AAD0BEEBC
:10F1A000FAEFFB123F3B7402122B84E96059AA0A62
:10F1B000AB0B123EC38A0E8B0FEA450F6046780EEA
:10F1C000122B56780A122B567C007D00AA08AB0938
:10F1D000123F4D7404122B84E9701D780E122B56C9
:10F1E000780A122B567C007D00EEFAEFFB123F47A7
:10F1F0007404122B84E96003750C01AA0EAB0F1284
:10F200003EC98003750C10A90C02BED174F61225FC
:10F210008412F44F905281E493F508EC8508F0A431
:10F22000FCA8F08508F0EDA428FD79FF7A3A7B1060
:10F23000123E0990070A7437F0A3743AF090070C55
:10F240007431F0A3743AF090070E745BF0A3743A33
:10F25000F09007107473F0A3743AF0900712747969
:10F26000F0A3743AF0900714748BF0A3743AF09002
:10F2700007167491F0A3743AF0900709E4F0800344
:10F28000122B847F02022809C082C0837B00800188
:10F290000B905281E493F8EBC398500BEB12F2E021
:10F2A00070EE12F6FF80047A007B0002F862C082E2
:10F2B000C0837A007B007D008018ED12F2E06011BF
:10F2C000743F28F582741012F724F8EA28FAE43B18
:10F2D000FB0D905281E493F8EDC39840DD02F86293
:10F2E00012F712F42274EC122584890F8A0A8B0B10
:10F2F0008C108D087E007F00123AA9AA0AAB0B126F
:10F300003AAF8A0C8B0D850A82850B83A3A3A3A336
:10F31000A3A3A3A3E064017007750E018E09800505
:10F320008E0E85100974FE650C700474FF650D70F7
:10F330000302F41A7B007414122E2DE0F50AA3E0E8
:10F34000F50B80010B905281E493F8EBC398505970
:10F35000EB12F70E650F70EC12F6F0650E70E51209
:10F36000F837650C7004A3E0650D70D8743E28F57D
:10F3700082741012F724650970CA743A28FE74105A
:10F3800039FF750C00E50CC39508400302F41A120E
:10F39000F423123A43E9700D12F423123A4FE97044
:10F3A000047E007F00050C80DC123A2B8A128B133E
:10F3B000AE12AF13EE4F60628E828F83E50FF0A323
:10F3C000E50EF08E828F83A3A3E50CF0A3E50DF08C
:10F3D0008E828F83A3A3A3A3E509F0905282E493C6
:10F3E000C395085004E493F5088E828F83A3A3A3EA
:10F3F000A3A3E508F0850A0C850B0D750E00780CAB
:10F40000122B52AC08EC2CFCE433FDEE2406FAE49B
:10F410003FFB123DFD7403122B84EEFAEFFB7F0CD1
:10F42000022809A80CE828F8E433F9E50A28F5824F
:10F43000E50B12F724FCA3E0FDEEFAEFFB22C082FD
:10F44000C08312F44F79FF123E09790102F86290ED
:10F450005267E493FC740193FD2274F7122584EA49
:10F460004B60377E0080010E8A828B83A3A3A3A307
:10F47000A3E0F8EEC3985022EE25E0F8E433F9EA71
:10F4800028F582EB39F583A3A3A3A3A3A3E06C70B3
:10F4900003A3E06D70D179018002790002F57374E5
:10F4A000F5122584EA4B607B8A828B83A3A3A3A3F6
:10F4B000A3E0606FEA2406F8E43BF98A828B83A319
:10F4C000A3A3A3A3E0F509750800800FEA2405F5BE
:10F4D00082E412F65714F0604A0508E508C395095E
:10F4E0005031AE08EE2EFEE433FF12F52A6C7003A5
:10F4F000A3E06D60D7AE08EE2EFE12F52AFEA3E063
:10F50000FF88828983EEF0A3EFF0E82402F850C967
:10F510000980C68A828B83A3A3A3A3A3E060047996
:10F5200001800279007F0302280912F578E0227435
:10F53000F7122584EA4B6039905282E493F88A826C
:10F540008B83A3A3A3A3A3E0C3985025EA2405F8C3
:10F55000E43BF988828983E025E0FEE433FF12F57D
:10F5600078ECF0A3EDF088828983E004F0790180E3
:10F570000279007F01022809EA2EF582EB3FF5832C
:10F58000A3A3A3A3A3A32274F41225848908EAFEEB
:10F59000EBFF8C098E828F83A3A3A3A3A3A3A3A3B2
:10F5A000E0640170098E828F8312FEBD800B123AD7
:10F5B000978A0A8B0BA80AA90B74FE68700374FF64
:10F5C00069700302F6497D00801A12F650640170DA
:10F5D00012743C2AF582741012F657687003A3E087
:10F5E00069605A0D905281E493FAEDC39A505AED36
:10F5F00075F00EA4FAACF0ECFB743A2AF5827410A4
:10F6000012F657650870DC8E828F83A3A3A3A3A391
:10F61000A3A3A3E0640160B212F65070C6743C2A42
:10F62000F582741012F657687003A3E06970B47421
:10F630003E2AF582741012F657650970A6ECF9742B
:10F640003A2AFA741039FB80047A007B0002F774BE
:10F65000743B2AF58274103BF583E02274F4122582
:10F6600084EAFEEBFF8E828F83A3A3A3A3A3A3A3AD
:10F67000A3E06401700D8E828F83E0F508A3E0F5AE
:10F68000098007123A978A088B0974FE650870048E
:10F6900074FF65096057750A008021E50A75F00E50
:10F6A000A4F8A9F012F6F0701112F7087004A3E0A4
:10F6B0006509700612F6FF123A3D050A12F77950F5
:10F6C000258E828F83A3A3A3A3A3A3A3A3E0640196
:10F6D00070C9E50A12F84670E112F7087004A3E059
:10F6E000650960D080D4AA08AB09123A6D02F7749C
:10F6F00012F6F422743B28F582741012F724227457
:10F700003A28FA741039FB2212F83B65082212F7E6
:10F71000122275F00EA4F8A9F0743A28F58274103C
:10F7200012F7242239F583E022743A28F87410394C
:10F73000F922122B847F0602280974F41225848989
:10F740000B8A088B097E007F008E0A801EE50A1254
:10F75000F70E650B7013AC08AD09AA82AB83123AA1
:10F7600043E960050EEE70010F050A12F77940DDDE
:10F77000EEFAEFFB7F04022809905281E493F8E54A
:10F780000AC3982274F2122584890C8A088B098C8A
:10F790000D750A00750B008004050A050B90528157
:10F7A000E493F8E50BC3985035E50B75F00EA4F81B
:10F7B000A9F0743A28FE741039FF8E828F83E065B9
:10F7C0000C70D8AC08AD09EEFAEFFB123A43E960D1
:10F7D000CAE50AC3950D40C1EEFAEFFB80047A003A
:10F7E0007B0002F735C082C08374F3122C1874FEBC
:10F7F0006A700374FF6B603D7D008015ED12F84662
:10F80000600EE0700B12F8376A7003A3E06B60259E
:10F810000D905281E493F8EDC39840E0E4936D704D
:10F82000148518828519837404F0740B122E2D121E
:10F83000FD73122FC9802612F83B22743C28F582F2
:10F84000741012F7242275F00EA4F8A9F012F6F441
:10F85000640122740B122E2DE0FAA3E0FB740D124A
:10F860002B84D083D082022B3674F6122584E4F5E3
:10F8700008F5097808122B5612FB2D12FC03123FD3
:10F880003B7402122B84E9FE6003123A79EEF9020E
:10F89000F28374F612258474FE122C188518828562
:10F8A0001983E4F0A3F0A818A91988088909780831
:10F8B000122B567508027509007808122B567C0029
:10F8C0007D007A417B00123F477404122B8474023E
:10F8D00002F28074F212258474EE122C18EAFEEB08
:10F8E000FF8C088D09750A007A417B00123F418A1E
:10F8F0000C8B0DAC0CAD0DEC4D6011E5086C70037C
:10F90000E5096D60077A417B00123F53E4F50CF581
:10F910000D780C122B56AC08AD097A417B00123FD2
:10F920003B7402122B84E9640A700302FA777402B2
:10F93000122BEA880889097808122B567508027577
:10F9400009007808122B567C007D007A007B031298
:10F950003F4D7404122B84E9600302FA7785188204
:10F96000851983E4F0A3F0F50802FA007404122B61
:10F97000EA880C890D780C122B569052671229C216
:10F9800085080C12FC0C850CF0A4F8AAF0850CF08C
:10F99000E9A42AF9E82402FCE439FD7A007B031289
:10F9A0003F4D7404122B84E9600302FA7774041249
:10F9B0002E2DE0F460487404122BEA880C780C12A7
:10F9C0002B569052671229C27404122E2D12FEBDBE
:10F9D000905267E493F50C740193F50DE8850CF0F3
:10F9E000A4C8AAF0850DF0A42AFA850CF012FBFC3D
:10F9F000123F477404122B84E9707C12FCC905087D
:10FA0000851882851983C082C083905281E493F85F
:10FA1000D083D082C3E098A3E0940050218518825F
:10FA2000851983C082C0837402122E2D12FEBDD0B0
:10FA300083D082C3E098A3E099500302F96CA81820
:10FA4000A919880889097808122B567508027509C2
:10FA5000007808122B567C007D007A417B00123F13
:10FA6000477404122B84E9700EEEFCEFFD7A007BE4
:10FA700003123F53E96003750A01A90A741202F7E1
:10FA80003274F212258474FE122C18750A0012FBCF
:10FA90002DF508E439F5097A417B00123F418A0CC3
:10FAA0008B0DAE0CAF0DA818A919880C890D780C18
:10FAB000122B56750C02750D00780C122B567C001B
:10FAC0007D007A417B00123F4D7404122B847A0032
:10FAD0007B03123F41EA4B700CE5086E7003E509A9
:10FAE0006F700D8041EE4F602B12FEB7E849602425
:10FAF0007C007D037A417B0012363BE9F8880A706E
:10FB000025EEFCEFFD7A417B00123F53E960097559
:10FB10000A018012EAFEEBFFAC08AD09EEFAEFFB3A
:10FB2000123A7FE9F50AA90A740202F73290526785
:10FB3000E493F8740193F9905281E493F508E88511
:10FB400008F0A4F8AAF08508F0E9A42AF9E824024C
:10FB50002274F512258474FE122C188518828519DA
:10FB600083E4F0A3F0123A85E9707EA818A91988F9
:10FB70000889097808122B5675080275090078085B
:10FB8000122B567C007D007A417B00123F4D74049D
:10FB9000122B84E970537E007F008E0A803CE50AB8
:10FBA00012FCD97808122B569052671229C2850A86
:10FBB0000812FC0C8508F0A4F8AAF08508F012FBE6
:10FBC000FC123F4D7404122B84E9700CE50A12F20A
:10FBD000E060050EEE70010F050A12F779500A1267
:10FBE000FEB7C3EE98EF9940B5851882851983E07A
:10FBF000FAA3E0FB7402122B8402F525E9A42AF98A
:10FC0000E82402FCE439FD7A417B0022905267E44B
:10FC100093F8740193F9E82274F112258474F012B8
:10FC20002C18851882851983E4F0A3F0FE805DEE20
:10FC300012FCD985080CF50D750E00780C122B52AC
:10FC400012F44F7405122BF2123DFD7403122B8433
:10FC50007402122BEA880A890B780A122B569052EA
:10FC6000671229C28E0A12FC0C850AF0A4F8AAF0C9
:10FC7000850AF012FBFC123F477404122B8485089E
:10FC800082850983E0F4600312FCC90E905281E47E
:10FC900093F8EEC3984098A818A91988088909789C
:10FCA00008122B567508027509007808122B567C2D
:10FCB000007D007A417B00123F477404122B84744C
:10FCC00010122B847F07022809851882851983E08A
:10FCD0002401F0A3E03400F02275F00EA4F8A9F09E
:10FCE000743A28F508741039F50922C082C083746B
:10FCF000F3122C1812FECD70128A828B8312FE2B07
:10FD0000122E2D12FEC3122FD58017EAFCEBFD74C4
:10FD100003122E2DAA82AB83122FABAA18AB191295
:10FD20002FDB02F85374F712258474F3122C18ECAD
:10FD3000FEEDFF8518828519837404F0740B122E72
:10FD40002D12FD73122FE1E9F508601D8E828F835D
:10FD5000A3A3A3A3A3A3A3A37403F0122E2DAC8289
:10FD6000AD83EEFAEFFB124901A908740D122B8442
:10FD700002F573EAF0A3EBF0AA18AB1922C082C017
:10FD80008374F3122C188518828519837404F07417
:10FD90000B122E2D12FD73122FE1740102F855740F
:10FDA000F612258474F3122C18900709E0707785F9
:10FDB00018828519837404F090054712FE2B122EC9
:10FDC0002DE8F0A3E9F012342BEAFCEBFD740312EA
:10FDD0002E2DAA82AB83122FABAA18AB19122FE7D4
:10FDE0001234378A088B09A808A9097401122E2D2C
:10FDF000E0687003A3E069602774FE68700374FF15
:10FE000069601D7401122E2DE8F0A3E9F07403124D
:10FE10002E2DAA82AB8312343DAA18AB19122FE7FC
:10FE20009007097401F0740D02F280E0F8A3E0F984
:10FE3000740122C082C08374F3122C1812FECD8A82
:10FE4000828B83701112FE2B122E2D12FEC3122FE5
:10FE5000D5E970608027A3A3A3A3A3A3A3A3E06411
:10FE6000037023EAFCEBFD7403122E2DAA82AB83F0
:10FE7000122FABAA18AB19122FDBE97037AA18ABF7
:10FE800019122FE7802E8A828B83A3A3A3A3A3A397
:10FE9000A3A3E0640170128A828B8312FEBD740BEF
:10FEA000122E2DE8F0A3E9800A740B122E2D74FE99
:10FEB000F0A304F002F853851882851983E0F8A3B3
:10FEC000E0F922E8F0A3E9F0AA18AB19228518821C
:10FED0008519837404F08A828B83A3A3A3A3A3A3AD
:10FEE000A3A3E064022274F51225847800790088C7
:10FEF0000A7F0080010F905281E493FCEFC39C5075
:10FF000032EF75F00EA4FCAEF0EEFD743A2CF582E3
:10FF100074103DF583E0F460DCAC0A74012CF50A42
:10FF20008C08EA65084B70CDEF75F00EA4F8EEF979
:10FF300012F729E8FAE9FB02F525C082C083901187
:10FF40004CE060357480659E70FA439403E594A29A
:10FF5000E250FAE0640270081247CF1247E18011C4
:10FF6000E06401600312452FE59DA2E640031245BF
:10FF70002F90114CE4F0124865D083D082022B36CA
:10FF800074F6122584E9FEA2AFE433FFC2AF9011EC
:10FF90004CE0600312452F900A9DE0600312452F4C
:10FFA000900A9CE07012900A9EE0700C900AB1E0FA
:10FFB0007006900AB0E06009EFA2E092AF7900808D
:10FFC00028124877EE90114CF0EFA2E092AF5394D4
:10FFD000FEE594A2E240FA74016E600B74026E605A
:10FFE0000312452F1247D579017F020228097409AF
:10FFF000F5D575D49E7409F5D375D2A6022B36FFBC
:020000040001F9
:10000000C082C083123A259004E074A3F0A3744C1C
:10001000F09004E2749DF0A3744CF09004E47497A3
:10002000F0A3744CF09004E67491F0A3744CF002C9
:10003000A4B674F7122584E9FE9004D2E4F0EE90A1
:1000400004D1F090113712929612A9877C8F7D0906
:100050007AD57B04124901901139E09004DDF090CB
:1000600004DE747AF0A3740902B18874F412258452
:100070008A088B09EB5480700302813E9004D1E022
:10008000F9123E398A0A8B0BAE0AAF0BEE4F7003A2
:1000900002813512B874E0F912A94E9004F012B43E
:1000A0009BA3A3A3A3A3A3A3A3E0640270378A82A4
:1000B0008B8312A96980078C828D8312AB94EC4DDF
:1000C00060208C828D83E06A7003A3E06B70E88C03
:1000D000828D83A3A3E06970DE90113F12C5C3F047
:1000E000804C124C678E828F83E064017034EE2462
:1000F000181281A7122B5A12AE6612298DEE241205
:100100001281A7122B5A12BEEC122B5612A40B12FC
:100110002995EE241712BEF81239D1740A122B84D5
:10012000800CE064027007EEFAEFFB124B47EEFA28
:10013000EFFB123E27AA08E5096480FB8066900960
:100140009AE0600464017019EAA2E050149004E897
:1001500012B1AB600612C8AC12276AE508640180D0
:100160003AEA5402600C9010BD7401F0EA6402FA9D
:100170008032EA54086029124C6D8B0BEA450B70F3
:10018000169004F2E4F0A3F0A3F0A3F07A08FB9039
:1001900004D1E0F9123F95E5086408FAAB09800440
:1001A0007A007B00028BCF12BDE0F50A780A227438
:1001B000F4122584EA4B9004E86026ECF0A3EDF0FD
:1001C0008A088B09E4F50AF50B7808122B4E7A01A0
:1001D0007B009004D1E0F9123F897404122B8480D3
:1001E0000FE4F0A3F07A01FB9004D1E0F9123F95FF
:1001F000028BCF74F41225848A088B098A828B8340
:1002000012C74D12BDBB38F583E02409FA7B0012FA
:100210003E218A0A8B0BAE0AAF0BEE4F70030282AF
:10022000B98E828F837402F0A3E412B007A3A3A354
:10023000A3E8F0A3E912A98BA3A3A3A3A3A3A3F00C
:10024000E5082403F8E43509129AAE12BDBB3AF56D
:100250008312B494F0EE2409FAE43FFB8E828F837C
:10026000A3A312A210F5838882E0A2E58E828F8379
:10027000A3A3A3A3A3500474018001E4F0E5082420
:1002800003F88882898312A969EA12C5A93BF5831C
:100290001282BE122B52EA12BDBB3B12A4148E82F4
:1002A0008F8312A967123DFD7403122B84EEFAEFBF
:1002B000FB9004D1E0F9123E2D028BCFA3A3E0F511
:1002C00008A3E0F509750A0078082274F212258463
:1002D0008A088B09ECFAEDFB740E122E2DE0FC124D
:1002E0003A558A0C8B0DAE0CAF0DEE4F6031AC0859
:1002F000AD09123A43E96027AC08AD09EEFAEFFB0D
:10030000123A49E970158E828F83128324EEFAEF38
:10031000FB123A3DAA08AB09123A6D7900800279C6
:10032000B4800EA3A3A3E0F508A3E0F50922122BE5
:10033000847F0602280974EF12258474F7122C18A2
:100340008A0A8B0BECFEEDFF750DB3750C00751072
:100350000080020510905281E493F8E510C39840A4
:1003600003028445851008AA087B00123AB58A0862
:100370008B09EA450960DC8A828B83A3A3A3A3A32C
:10038000E0250CF50CF50EC3E50A950EE50B94007F
:1003900050C17C157D007900EEFAEFFB123E098515
:1003A0000882850983A3A3A3A3A3E0F8E50AC39564
:1003B0000C2825E0F8E433F9E50828F582E5093949
:1003C000F58312A97512342BEAFCEBFDEEFAEFFB74
:1003D000124901850882850983A3E06401700A122D
:1003E000AE66740112AF39803DAC18AD1985088234
:1003F00085098312A967123A9DE960307408122EAC
:100400002DE0C0E012AE66D0E0F07408122E2DE0B0
:100410006403700CAC18AD1912B482124901800C3F
:1004200085188285198312AE7612A9878508828580
:1004300009831299CAA3A312AF41C0E012BABBD07C
:10044000E0F0750D00A90D7409122B847F090228B4
:100450000974F7122584E9FE8A828B83A3A3A3A3E0
:10046000A3A3E0540860338A828B83A3A3A3A3A32E
:10047000A3E0540260218A828B83A3A3A3A3A3A336
:10048000A3A3A3E06406600F74E96E600A74CD6EE6
:10049000600574F06E7003124C8502ACD774E812DC
:1004A000258474F8122C187406122E2D12C787ECAE
:1004B000FEEDFF89177515001286E4123A618A0A6B
:1004C0008B0BEA450B7003028696EE241012B66081
:1004D000A90A12318B8A128B13EA45137003028624
:1004E00096EE2403F50CE43FF50DEE2406F508E442
:1004F0003FF5097C0085088212BE14123A678A1003
:100500008B11850C82850D831286D91298B68512BF
:1005100082851383A3A3A3A31294B11286D9A3A3A4
:10052000A3A312B89E851282851383A3A3A3A3A3BA
:10053000A312CB9E12AF2D122B5212BDBA3F12A4A2
:1005400014851282851383A312A961123DFD7403E1
:10055000122B847514007423122E2DE0F5167424CA
:10056000122E2D780C122DD602861B851082851135
:100570008312A967123AA3850882850983A3EAF04A
:10058000A3EB1286F5A3A312AA3512898FA2E65017
:100590000F850882850983A3A3A3A3A3E0D2E1F07A
:1005A000E515706685088285098312C0F5900547B8
:1005B000E0687003A3E0697051850882850983A310
:1005C000A3A312B6657510007810122B5A780C127E
:1005D0002B4EE516F5107810122B5A7426122E2D7C
:1005E00012299590055412299579007410122E2D18
:1005F00012A96D122E3D740A122B8485088285097A
:1006000083A3A3A3A3A3E04405F074012514FC1263
:1006100086E4123A678A108B110514E510451160C3
:1006200050851408C3E508950AE4950B5043E5147A
:1006300075F006A4F8A9F0E51228F8E51339F9E8F1
:10064000240CF508E439F509850882F583E412D80D
:1006500020E06401600302856B75150185088285C1
:10066000098374011286F512BB0DE8F0A3E9028537
:1006700082AA12AB131231917812122B56AD167456
:1006800024122E2DE0FCA917EEFAEFFB124C8B740E
:1006900002122B84803E8E828F83A3A3A3E0C0E04E
:1006A0007403122E2DD0E0F0EE241212BDD9C0E05A
:1006B0007404122E2DD0E0F0E50A450B7009740584
:1006C000122E2D74B980077405122E2D741012A4E9
:1006D00034122E377408028CFEE085128285138353
:1006E000A3A3A3228E828F8312BE228E828F83A326
:1006F000A3A3E0F92212D824A32274E8122584745B
:10070000F2122C18E9851882851983F08A0A8B0B5E
:100710008C168D177426122E2D129102AA0CFB1224
:10072000317FE9F514AA0CAB0D123185E9F515E519
:10073000147003028977751300800F8E828F83A354
:10074000A3A3A3A3E0D2E3F00513E50C12A942355D
:100750000DF583E0F8E513C398400302896EE514B4
:10076000700302896EE51375F006A4F8A9F0E50C94
:1007700028F8E50D39F9E8240CFEE439FF8E828F64
:1007800083A3A3A3A3A3E0A2E040BD750E0090093C
:100790009AE060046401704A8E828F83E070431295
:1007A000A96812301D8A088B09A808A909E84960C0
:1007B0003188828983A3A3A3A3E06401600D8882AA
:1007C0008983A3A3A3A3E0640370178E828F83A3FE
:1007D000A3A3A3A3E0D2E7F0750E01E51570030211
:1007E0008748750F00750808750900E517600375DF
:1007F0000F207C087D0079007401122BF2123E0953
:100800008E828F83E0603C900597E064017018E56C
:100810000FD2E3F50F75091012C0F17401122E2DDD
:1008200012A0CD74FF803A430F0C75080C8E828F96
:1008300083A312898512A9837401122E2D74FFF0EF
:10084000A3801E851882851983E06009E50FD2E632
:10085000F50F75080A12C0F17401122E2DE8F0A3ED
:10086000E9F07403122E2DE50F12BB40C0E07405B1
:10087000122E2DD0E0F07406122E2D7401F0122BE2
:10088000F2124B41740D122E2DE06003028949745F
:1008900009122E2D1298938E828F83A3A3A3A3F007
:1008A0007409122E2D1289981290F8E51612898F6C
:1008B0006011900597E0C0E07409122E2D12910E80
:1008C000D0E0F0850C82850D83A3A3A3E0C0E07483
:1008D00009122E2D12BE44D0E012AC41C0E07409C2
:1008E000122E2D129118D0E0F07409122E2D1289BB
:1008F0008512C76512BB4912A96912C746EAF0A35F
:10090000EB12BB2FC0E012C73ED0E0F07409122EEC
:100910002D128AC712897C129CE53B12BB1C12BDAA
:10092000B3128D127512007810122B5212A40FEA16
:1009300012A93B3BF58312A969123DFD7403122BEA
:10094000847401122BF2124B3B8E828F83A3A3A3DC
:10095000A3A3E0D2E0F0740D122E2DE06003028715
:100960003BE50EA2E05002151515140287487900E8
:10097000AA0CAB0D124C7F740E028CFEA3A3A3A392
:1009800012C0FAEA2212C0FA850A82850B8322126B
:1009900089932212C2EEE022129D0412AE6039F554
:1009A00083E508F0A3E509F02274F012258474E9C8
:1009B000122C18EAFEEBFF89088E828F83A3A3A373
:1009C000A3A3A3A3A3E0F91231A98A0C8B0DEA45D6
:1009D0000D7003028AC2E50870157C048E828F8335
:1009E000A3A3A3A3A3A3A3A3E0F91231AF804F7CD9
:1009F000088E828F83A3A3A3A3A3A3A3A3E0F912CA
:100A000031AF8A0A8B0BEA450B6033E508F50978AC
:100A100009122B5A850C82850D83A3A3A3A3A3A33C
:100A2000A3E0FD8A828B83A3A3A3E0FC8A828B834D
:100A3000A3128AC7E0F91239CB7401122B8412A4D5
:100A40000512B1A9607C8882898312A96574061297
:100A50002E2D128AD112A9697408122E2D128AD154
:100A6000A3A3E0C0E07410122E2DD0E0F0850C821C
:100A7000850D83A312A961740E122E2D12C78774DF
:100A800011122E2DE412898FFAA3E0CA241FF582D9
:100A9000E43AF583129AB9E0C413135403FC7002CC
:100AA0007C0488828983E0F9780C122B56742059D3
:100AB000FD744059F97402122BF2124C8B7402121D
:100AC0002B8474170296B212BE28850A82850B8386
:100AD00022EAF0A3EB129E89A3A32274F7122584C5
:100AE00074FA122C18E9FE7F018F087D00800475CE
:100AF00008000D1293BCE0F8EDC3985027ED75F097
:100B000006A4F8A9F0EA28F8EB39F9E812BB3A395B
:100B1000F583E0A2E050D8540C60D4E0A2E250D2B9
:100B20007F0080CE8A828B83A3A3A3A3A3A3E070BC
:100B30003EE508A2E0400574016E70338A828B8323
:100B4000A3A3A3A3A3A3740112C607E0C0E0740388
:100B5000122E2DD0E012C5FFE0C0E07404122E2D3D
:100B6000D0E0F07405122E2DEF12A434122E37743B
:100B70000602ACD4C082C0837901124C7F02A4B6B5
:100B800074F4122584EA4B602D900593E0640270A2
:100B9000259010BDE4F08A088B09F50AF50B78085A
:100BA000122B4E7A027B009004D1E0F9123F897437
:100BB00004122B8480129010BD7401F07A027B0025
:100BC0009004D1E0F9123F9580057402122B847FC6
:100BD0000402280974E812258474FC122C1874028B
:100BE000122E2DE4F0A3F09004F012B76B8518825A
:100BF000851983E4F0A3F0751401900541E0A2E3A8
:100C00005003028C8B123FAD8A088B098C0A8D0B26
:100C10008A0C8B0D8C0E8D0F9004F2780C122BD257
:100C2000128D067810790C122D8850077A017B00FE
:100C3000028CFC850C14850D15850E16850F177812
:100C4000147910122515A814A91590113FE0C39826
:100C5000E4995003E0F514128D06780C79101225F2
:100C600015E4F512F51378087910122CAB9004F204
:100C70007808122DC7801412C0F69004F012A987CC
:100C8000EEFAEFFB123EC9AE08AF09EE4F60658E7B
:100C9000828F83A3A3A3E0F8E514C3985029EE2420
:100CA00003F582E43FF583A814E0C398F060217453
:100CB00002122E2D12C2DA12B4B6EEF0A3EF12A673
:100CC000A7FEA3E0FF80C48E828F83A3A3A3E4F0DA
:100CD0008E828F83A312832385188285198312B194
:100CE000AB8E828F83A3A3A3A3608C12A2A2129ABD
:100CF000C2A380897402122E2D12A9697404122BCA
:100D0000847F1002280990113D128D12E4F512F52E
:100D10001322E0F510A3E0F5112274F21225848A63
:100D20000A8B0BE9FE7A007B009004F01283269078
:100D300004F012B1AB601E0A850882850983A3A363
:100D4000A3A312B1AB600E0AEA70010B88088909EF
:100D5000E8450970E390114012C0F6C3EA98EB9998
:100D60004003028E057A067B00123EC38A0C8B0D6F
:100D7000A80CA90DE8497003028E0588828983E5D5
:100D80000AF0A3E50BF0EE88828983A3A3F090110B
:100D90003F129D30A3A3129E84E4F0A3F09004F0D0
:100DA00012B18C600B85088285098312A983801F8C
:100DB0009004F012A987900541E0A2E34011123F90
:100DC000ADEAF8EBF9ECFAEDFB9004F2122E169076
:100DD0000541E0A2E3502E7A087B009004D1E0F9AF
:100DE000123F9BEA4B4C4D701C90113D12D259782A
:100DF00008122B4E7A087B009004D1E0F9123F8F45
:100E00007404122B8402833174F212258474F31259
:100E10002C18EAFEEBFF8E828F83A3A3A3A3A3A3C8
:100E2000A3A3A3A3E0F50A9010BDE0700579BA0270
:100E300090EC750801750900750C00750D007C08B3
:100E40007D007900AA18AB19123E097405122E2DE7
:100E50007401129124540460127402122E2DE0D2F7
:100E6000E612912454087003750803E054106006DC
:100E700074404508F508E0540860227402122E2DD3
:100E8000E044C01291245420600A7403122E2DE015
:100E9000D2E080087403122E2DE0D2E1F08E828F12
:100EA00083A3A3A3A3A3A3A3A3E070161234318545
:100EB000188285198312C7877402122E2DE0D2E2A0
:100EC000802C640F70107402122E2D12912C740459
:100ED0004508F508807B8E828F83A3A3A3A3A3A3D9
:100EE000A3A3E064028E828F83700612A050F0806C
:100EF00060A3A3A3A3A3A3A3A3E06403700DAC18F2
:100F0000AD19EEFAEFFB124C2B80468E828F83A335
:100F1000A3A3A3A3A3A3A3E064017035900597E066
:100F200060107402122E2D12912C750910750AFF93
:100F300080187402122E2DE0440C12B4B674FDF029
:100F4000A374FFF074044508F5088E828F83129114
:100F500002EE241512BDD9A2E0503F7402122E2DCC
:100F6000E0540C701B8E828F8312A969124457E9DA
:100F7000700579BB0290EC7402122E2DE0D2E5F0E0
:100F8000EE241512BDD9A2E050107402122E2DE0ED
:100F9000540C64047004E0D2E5F0EE241112BDD9C3
:100FA000C0E07404122E2DD0E012A434124B417410
:100FB0000C122E2DE060030290E57408122E2D1203
:100FC0008998EE241812BDD9C0E01290F8D0E01232
:100FD000BB24E0C0E07408122E2D12C75012BDD001
:100FE00038F583D0E012A05864017011900597E0A5
:100FF000C0E07408122E2D12910ED0E0F074081289
:101000002E2D12B4A52417FAE43FFB8A828B83E0CD
:10101000FCE8241CF582E439F583ECF0A3E412B17A
:10102000BBE0C0E0E82422F582E439F583D0E0F0AB
:101030007408122E2D129118E50AF07408122E2D44
:10104000129D00129CE539F583E50CF0A3E50D1225
:10105000BE68FCA3E0FD12C770ECF0A3ED12954C46
:1010600012AB981290F13912C162C0E0E8242FF55A
:1010700082E439F583D0E0F0EE241B12BDD9C0E044
:101080007408122E2D12C759D0E0F0EE241A12BDAA
:10109000D9C0E07408122E2D12C75012B65638F57A
:1010A00083D0E012C78D1282BF122B5212AE4C12A7
:1010B000AB98740B122E2D12A02E123DFD7403124C
:1010C0002B84EE241512BDD95440601290050012F5
:1010D000B1AB600AAA18AB1912C8AC12276AAA18D9
:1010E000AB19124B3B740C122E2DE0F9740D0283D8
:1010F0002EE82428F582E422E82412F582E439F56A
:10110000832212910622E0F50CA3E0F50D2212C70E
:101110005412BAA538F5832212C7542423F582E469
:1011200038F58322F0EE241512BDE022E0D2E3125E
:10113000C2EE1291362212A2AAE8F0A3E9F02274BC
:10114000F71225847E638A828B83E0600C79051216
:101150002F5DE9F87456C398FE90053FE0600CF9E6
:10116000122F5DE9F8EEC39824F2FEEEF902ACD737
:1011700074F612258474FE122C1885188285198342
:1011800012C787E9FEECFAEDFB90070A12B1AB60DB
:1011900035A818A919880889097808122B567D01E5
:1011A000740E122E2DE0FCEEF990070A12A51F1204
:1011B000276A7402122B848B09EA450960047900BE
:1011C000800679B2800279B60298BE74F71225843F
:1011D000E9FE9004E012B1AB601F7409122E2DE0FD
:1011E000F5087808122B5AEEF99004E012A51F12A8
:1011F000276A7401122B84800279B602ACD774F787
:101200001225848908ECFEEDFF79B5E508245F60BE
:101210000C14603114601224F86041804A9004D3A9
:1012200012BB01E8F0A3E9801990070C12B18C60A1
:101230003690070C12A51F12276A8E828F83EAF060
:10124000A3EBF080209004E212C002601AEEFCEFE3
:10125000FD9004E212A51F12276A800B9004DE1293
:10126000A96D124901790002ACD774F7122584E9FF
:1012700079B5245F600624F6600E80178C828D831A
:1012800012929612A98780099004DE12A969124968
:1012900001790002ACD712C0FA9004D32274F21282
:1012A00025848A088B09ECFEEDFF750A019005473D
:1012B000E065087004A3E06509701012342BEAFCA5
:1012C000EBFDEEFAEFFB124901802A1234378A0C4B
:1012D0008B0DE508650C7004E509650D7009EEFAE3
:1012E000EFFB12343D800EEEFCEFFDAA08AB0912B5
:1012F0002FBDE9F50AA90A02833174F5122584EAA3
:10130000FEEBFF8C088D09750A0112342BEAFCEB09
:10131000FDEEFAEFFB1248FBE96401700B90054704
:10132000129ACE12A987800EAC08AD09EEFAEFFB37
:10133000122FC3E9F50AA90A02CCF074F61225842B
:10134000EAFEEBFF7A0C7B00123EC3EA4B606AEECA
:10135000242012BDD98A828B83F0EE24211293C4FB
:10136000F0EE24221293C4A3F0EE24231293C4A31C
:10137000A312B66B1293CD12A983EE1290F23FF531
:10138000831293CDA3A3A3A3A3A3E8F0A3E912B66A
:101390007A8A828B83A3A3A3A3A3A3A3A3F0EE249F
:1013A0002F12BDD9C0E01293BCD0E012AC4AF8A312
:1013B000E0F98A828B8312A97E0298C3EA12A946B9
:1013C0003BF5832212BDE08A828B83A32212C0FAEE
:1013D0008A828B832274F6122584ECFEEDFF79B3AA
:1013E00090053EE0702A900570E064017022EE24C2
:1013F0001112BDD9F9122F458A088B09A808A9092D
:1014000012AE5412A987E84960047900800279A1DC
:101410000298C374F412258474FE122C18ECFEEDAD
:10142000FFEE241612BDD96405700DEE2406FCE40F
:101430003FFD124C31E96074AC18AD1912BAC512F7
:10144000445D85188285198312B1AB605BE875F045
:1014500009A4F8AAF075F009E9A42AF9747628F825
:1014600074F639F9E8FAE9FB8A828B837808122D41
:10147000D61296A47808122D9840298518828519CD
:101480008312B4A512AE551294B17808122DD690DD
:10149000812C7808122CBF8A828B837808122DC782
:1014A0007900800A79A2800679A1800279C8028B2E
:1014B000CA129139EE1296A92274F412258474FF8F
:1014C000122C18EAFEEBFF90053EE0706C90057060
:1014D000E06401706475083A7509007808122B56AB
:1014E0007402122BEA880889097808122B567C01AD
:1014F0007D007A007B0012360B7404122B84E97095
:101500003512AFD67401129629C0E012AE4CD0E06D
:1015100012954C743A12B89E900508122E0A129633
:10152000A4122E1690812C7808122DD690050878DA
:1015300008122D1E800312953E7401028BCCEE24FE
:101540000FF582E43FF583E4F0A3F022F0EE12AE53
:10155000592274F012258474F6122C18ECFEEDFF5B
:101560007402122BFA124C31E97003029624AC1863
:10157000AD197402122BF212445D8518828519830D
:1015800012B1AB7003029624E875F009A4F8AAF032
:1015900075F009E9A42AF9747228F874F639F9E8A3
:1015A000FCE9FD12AFD6E4129629F8A3E0F912AED9
:1015B0005412A9878C828D83122E0A1296A4122EA1
:1015C0001690812C7808122DD68C828D8378081283
:1015D0002D1E8C828D837808122DD6908100780C78
:1015E000122DD67808790C122515E50C450D450EFF
:1015F000450F7030851882851983129D0075F0099A
:10160000A4F8AAF075F009E9A42AF9747A28F582F9
:1016100074F639F5837401F07A007B089007AAE02C
:10162000F9123E63740A0296B2F085188285198316
:10163000E02274F01225848A088B09ECFEEDFF127B
:10164000953E90815C780C122DD61296A4780C12DF
:101650002C44604CEE240E12BDD964017005124C6E
:101660001F803FE07015124C13E960368E828F8325
:10167000A3A312A45A5403700C802764027013129F
:101680004C13E9601DEEFCEFFDAA08AB0912449370
:101690008010E064037005124C13800679A180026B
:1016A00079A38011EE1296A9222412F582E43FF567
:1016B0008322122B847F0802280974F6122584EAFB
:1016C000FEEBFFEE240AF508E43FF509850882F5F4
:1016D0008312AB98EC12AE603DF583E4F012AC38A7
:1016E000124C07850882850983E02406FCA3E034B8
:1016F00000FD8E828F8312A969124C318508828584
:10170000098312B1A070541298981248FBE9701D19
:1017100012342B8A088B09AC08AD099004DE12A99B
:10172000691248FBE97006124BD7E9602E8E828F52
:101730008312AB8E8E828F8312A969124499E9605D
:10174000158E828F83A3A3A3A3A3A3A312C74D12B5
:10175000B8A3E4F0A3F0129AEFE4F012B192701A79
:1017600012977D12A969124C0D8508828509831292
:10177000B1A0700612AFC874A1F00298C3EE240A9B
:1017800012984D8882F5832274F6122584EAFEEBC6
:10179000FFEE240A12984D7A187B00123EC385088A
:1017A00082850983EAF0A3EB1298B6E84970030238
:1017B0009847EEFAEFFB124BD112B1926072129879
:1017C0008564018E828F83A3A3A3A3A3A3700712B2
:1017D0009877740E802012B1AB700F12989812484F
:1017E000FBE97006124BD7E9600712986D740D8003
:1017F0000512986D740512AC4A5403640170071207
:1018000098567405800B90053FE0C0E0129856D0C2
:10181000E012A421F812C8ABA3E0F9122F5D8508ED
:101820008285098312C75012BADB38F583E9801A22
:1018300085088285098312A969123EC985088285B7
:101840000983E4F0A3800312A66EF08076F8E43FEB
:10185000F988088909228E828F83A3A3A3A3A3A357
:10186000A3A312986622A3A3129F93A3228E828F12
:1018700083A3A3A3A3A3A3A3A3A3A312C75412A6A2
:101880005F38F583228E828F83A3A3A3A3A3A3A390
:10189000A3A3A3129B01E0229004DE12AB9C8E82D4
:1018A0008F83A3A3A3A3A3A3A3A3A3A3E02406FAC4
:1018B000A3E03400FB2212A425F8A3E0F92274026D
:1018C000122B847F0202280974F11225848A0A8B64
:1018D0000B8C088D097A187B00123EC38A0C8B0D85
:1018E000AE0CAF0DEE4F70030299C28E828F8374DF
:1018F00001F0E508240DF8E43509F988828983E0D0
:10190000FAC3E49AFA95E0FBE50812C5A935091275
:1019100099CEFB8E828F83A3A3A3A312C6338E829C
:101920008F83A3A3F0EEFAEFFB122F0985088285BF
:10193000098312C5CC70098E828F83A3740580063B
:1019400090053F1299CAF0EE2417F8E43FF9880C8D
:10195000890D8E828F83A3E0F9122F5DE9850C82B9
:10196000850D83F0EE2416F8E43FF9E508240EFA1D
:10197000E43509FB8882898312A67CE5082410FAE5
:10198000E43509FB850C82850D83E0FC8882898320
:10199000E0F88A828B83E0C398C39C12C2E3F0EE26
:1019A000FCEFFDAA0AAB0B124C01E9F508700AEE38
:1019B000FAEFFB122F15E9F508EEFAEFFB123EC91C
:1019C0008003750810A90802AF5C12A99222F58362
:1019D000E02AFAA3E03B227901022B3674F41225A7
:1019E00084EAFEEBFF8E828F83A3A3A3A3A3A3A30A
:1019F000A312BE0AF58312C5CC702A1298857025F1
:101A0000129ADCE06405701D129ADCA3E0F8740100
:101A10006860057406687007129AEF7402800512F8
:101A20009AEF7403F012977D12A51FE4F0EE2408DC
:101A3000129AAB242DF582E43AF583E0C0E08508E4
:101A400082850983129AB9A3A3D0E012C637FAA3FC
:101A5000E0CA242AF582E43AF583E0C0E0850882F2
:101A6000850983129AC2D0E012C637F8A3E0C812E3
:101A7000A94238F583129ACE129AB912A983123468
:101A80002B8A0A8B0BAC0AAD0B850882850983E093
:101A9000240612A29112490185088285098312A9A0
:101AA00069122F1512A718F0028BCFF8E43FF988BE
:101AB000828983E0FAA3E0CA22E0FAA3E0F5838AF0
:101AC0008222E0FAA3E0F5838A82A3A3A322129ADA
:101AD000D22212C0FE850882850983228E828F83DE
:101AE000A3A3A3A3A3A3A3A312A035129F8F228E07
:101AF000828F83A3A3A3A3A3A3A3A3A3A3129B0146
:101B00002212A21BC8240EF582E438F58322EA12C1
:101B1000C5A33BF583220299D7C082C0839004F607
:101B200074CBF0A3744BF09004F874BFF0A3744B23
:101B3000F09004FA74B9F0A3744BF09004FC74C5EF
:101B4000F0A3744BF002A4B674F4122584EAFEEB01
:101B5000FF129B9EF5081234318A0A8B0BA80AA942
:101B60000B8E828F83129AB9E0687003A3E06960DC
:101B70002AE508A2E550248E828F83A3E0FB90041F
:101B8000F612A51F12276A8E828F8312C750240A6D
:101B900012B1A57006129B9EC2E5F0028BCF8E8219
:101BA0008F83129868A3E02274F4122584EA240833
:101BB000FCE43BFD8C828D83129D0012A665E0FE45
:101BC00074035EF50912A9413912B4A3888289838E
:101BD000F0A3A882A983E50960097402650960037E
:101BE000029C73740C5EF508601774086508601138
